:100000000056002001660000516500006165000097
:100010007965000091650000A965000000000000FE
:10002000000000000000000000000000C1650000AA
:10003000D165000000000000E1650000F1650000EE
:10004000396500000000000000000000DD1801001C
:1000500019180100891801000000000000000000CC
:10006000F546000051FD000031FD000005190100BA
:100070000000000000000000000000002519010041
:100080002DE9F843054689464FF00108154E164CF8
:10009000164F12E0236943F00403236187F832808E
:1000A000BFF34F8F00BF30BF87F83200236923F0C2
:1000B00004032361BFF34F8F62B600F01DF872B6E0
:1000C000735D33B900F014F80028E3D000BF30BFEF
:1000D000F2E700237355B9F1000F00D0C84762B6AC
:1000E000BDE8F883CC22002000ED00E000001050B5
:1000F0005FF800F0254600005FF800F08500010081
:10010000FFFFFFFFFFFFFFFFFFFFFFFFFFFFFFFFFF
:10011000FFFFFFFFFFFFFFFFFFFFFFFFFFFFFFFFEF
:10012000FFFFFFFFFFFFFFFFFFFFFFFFFFFFFFFFDF
:10013000FFFFFFFFFFFFFFFFFFFFFFFFFFFFFFFFCF
:10014000FFFFFFFFFFFFFFFFFFFFFFFFFFFFFFFFBF
:10015000FFFFFFFFFFFFFFFFFFFFFFFFFFFFFFFFAF
:10016000FFFFFFFFFFFFFFFFFFFFFFFFFFFFFFFF9F
:10017000FFFFFFFFFFFFFFFFFFFFFFFFFFFFFFFF8F
:10018000FFFFFFFFFFFFFFFFFFFFFFFFFFFFFFFF7F
:10019000FFFFFFFFFFFFFFFFFFFFFFFFFFFFFFFF6F
:1001A000FFFFFFFFFFFFFFFFFFFFFFFFFFFFFFFF5F
:1001B000FFFFFFFFFFFFFFFFFFFFFFFFFFFFFFFF4F
:1001C000FFFFFFFFFFFFFFFFFFFFFFFFFFFFFFFF3F
:1001D000FFFFFFFFFFFFFFFFFFFFFFFFFFFFFFFF2F
:1001E000FFFFFFFFFFFFFFFFFFFFFFFFFFFFFFFF1F
:1001F000FFFFFFFFFFFFFFFFFFFFFFFFFFFFFFFF0F
:10020000FFFFFFFFFFFFFFFFFFFFFFFFFFFFFFFFFE
:10021000FFFFFFFFFFFFFFFFFFFFFFFFFFFFFFFFEE
:10022000FFFFFFFFFFFFFFFFFFFFFFFFFFFFFFFFDE
:10023000FFFFFFFFFFFFFFFFFFFFFFFFFFFFFFFFCE
:10024000FFFFFFFFFFFFFFFFFFFFFFFFFFFFFFFFBE
:10025000FFFFFFFFFFFFFFFFFFFFFFFFFFFFFFFFAE
:10026000FFFFFFFFFFFFFFFFFFFFFFFFFFFFFFFF9E
:10027000FFFFFFFFFFFFFFFFFFFFFFFFFFFFFFFF8E
:10028000704700BF034613F8012B002AFBD1181A50
:100290000138704700487047FCCA01003D20704794
:1002A0000120704708B506F0DFF808BD08B506F074
:1002B0003FF943690148984708BD00BFFCCA0100E7
:1002C00010B50C4611461A46012807D010B1022875
:1002D0000BD010BDE0B200F047F8FAE7BDF80830E7
:1002E000C9B2E0B200F082F8F3E7E0B200F046F9FC
:1002F000EFE700BF054B00229A80DA805A819A818D
:10030000B42119811A765A769A767047C023002054
:10031000014B1878704700BFC023002010B404467A
:10032000034B0FCB84E80F00204610BC704700BF82
:10033000C42300200346054901F1140248691860EE
:10034000098B927999809A7118467047C0230020D2
:10035000044B187E012803D0987E003018BF01207E
:10036000704700BFC023002010B504461D4B1B780A
:1003700013F0030F02D010F00C0F15D114F0030F7F
:100380001CD113F0080F02D014F0040F22D113F087
:10039000040F15D014F0080F12D0124B00229A80CF
:1003A000DA80B4221A810BE006F05EF802690D4B88
:1003B0001A61FFF79FFF00F019F901E0FFF79AFFBC
:1003C000084B1C70084C204600F090FE204600F0C0
:1003D0003DFB10BD034B00229A80DA80B4221A81C3
:1003E000EEE700BFC023002004CB010010B5044697
:1003F00000F0A4FF042C00D010BDFFF789FF10F01F
:100400000C0F05D000F0ABFF4368984700F0F8F8F8
:10041000564C204600F0B8FE204600F0BDFB544B81
:100420001A78042A30D0082A46D0514B5B89B3F59C
:10043000616F05D34E4B0021598199890131998112
:100440004B4B99894EF66023994250D0484BD9883E
:100450004EF6602399424ED0454B99884EF6602364
:1004600099424CD012F0080F4DD1414B1B8BB3F584
:10047000807F76D03E4B9B7E13B1013B3C4A937606
:100480003B4B1A7E5A76B7E73949CB8801339BB28A
:10049000CB803849A1FB0301490901EB8101A3EBA2
:1004A000C1039BB2002BC0D1314B59890131598115
:1004B000196901311961B8E72D490B89013B0B819D
:1004C0008B8801339BB28B802B49A1FB0301490927
:1004D000C1EB0111A3EB81039BB2002BA5D1244BEF
:1004E0005989013159811969013119619DE7204B01
:1004F00000219981AAE71E4B0021D980ACE71C4B53
:1005000000219980AEE700F02AFF4368984703680E
:10051000984760B9164B1B7813F0080FA5D0134805
:1005200000F06CFE78B1124BB4221A819DE700F006
:1005300016FF4368984700F0B2FD0128EAD10C4B42
:10054000B4221A81E6E70A4B1B7813F0080F8CD00F
:10055000074B1B89002B88D105F0EAFF03689847F9
:1005600083E7034B06229A768AE700BF04CB01009B
:10057000C0230020CDCCCCCC8988888810B5072832
:1005800019D8DFE800F019041D201823262C05F0E7
:100590006BFF044605F0CCFFC3684FF48062002176
:1005A00020469847FFF7A6FE0E4800F09FFD04F195
:1005B000F00000F038FA10BD0A4800F0BBFDFAE781
:1005C000094B1975F7E7084B5975F4E7064B997510
:1005D000F1E7054BD975034800F088FDEBE7024BC6
:1005E0001976E8E704CB0100C023002008B580227B
:1005F0000021024818F0E3F908BD00BFDC23002009
:100600002DE9F04F85B082460022924911F8323030
:100610006FF3C71301F8323001EBC20358786FF360
:10062000C710587098786FF3C7109870D8786FF328
:10063000C710D87018796FF3C710187158796FF315
:10064000C710587198796FF3C7109871D8796FF304
:10065000C710D8710132102AD8D1DAF80030984783
:1006600003900023029345E04FF001084FF0140C73
:10067000B5423AD801974FF04C0933464646984662
:100680002BE04FF001084FF0140CF1E7425C42F010
:100690008002425402F07F0202EB0C0BBBF14C0FC4
:1006A0000FDD425C69F30602425401339BB29C4267
:1006B0000FD319461EF80320D209E7D0002EF4D03C
:1006C000E4E7624410F801B062F3060B00F801B0F1
:1006D000EBE70135ADB2A84507D3A742F9D8019B96
:1006E0005C4A02EBC50E7046E3E7029B01330293BE
:1006F0000A2B66D09DF80880DAF8283040469847E3
:10070000012805D0DAF82830404698470228ECD175
:10071000DAF80C30404698478146DAF81030404607
:100720009847834603014C4A82FB0326F218DE17E2
:10073000C6EBE2264FEAC903484A82FB03271F445F
:10074000DB17C3EBA727DAF8183040469847DAF8EA
:10075000083040469847002814BF10240424B6B23D
:10076000351B25EAE575ADB226440F2EA8BF0F262E
:10077000B6B2BBB21F1B27EAE777BFB21C44072CF7
:10078000A8BF0724A4B2DAF8083040469847A9F178
:1007900043091FFA89F940F2B23399453FF664AF35
:1007A000BBF16E0F7FF66DAF002814BF4FF0140C35
:1007B0004FF0010C002814BF4FF001084FF0000863
:1007C00056E70026234F1FE0043AE55C62F3060576
:1007D000E55404E0013AE55C62F30605E5540133B3
:1007E000082B0ED0C25CD209F9D1C25C02F07F02A4
:1007F000122AEFD8032AE7D8E25C6FF30602E2542C
:10080000EDE70136102E04D0002307EBC6000446A6
:10081000E8E7039B1BB1002421460E4D05E0FFF7DE
:10082000E5FEF8E70134102C0DD0002305EBC400E1
:10083000C25C02F07F02092A84BF013189B2013310
:10084000082BF5D1EEE7034BA3F8801005B0BDE807
:10085000F08F00BFDC230020E1000EE049D6B9F2A2
:100860002DE9F04F83B0064601911446036898477E
:1008700070B13E4A92F88230013382F88230A1464C
:10088000002C5ED00027B8469346DFF8E8A037E09A
:10089000FFF7ACFE4FF00008019B83F8008055E0A5
:1008A000F3682046984740B333692046984720B301
:1008B000F36820469847054633692046984700016B
:1008C0008AFB00230344C017C0EBE32080B2ED0095
:1008D000274B83FB05232B44ED17C5EBA325ADB2B6
:1008E0000BEBC000435D03F07F03122B05D808F12A
:1008F00001085FFA88F8019B1C7001374F4510D042
:10090000FCB2B36A204698470128C9D0B36A204692
:1009100098470228C4D0B36A204698470328ECD1F0
:10092000BEE7B8F1000F0CD0104BB3F88030402B6D
:1009300010D8B8F1010F09D012D90023019A137011
:1009400004E04FF00008019B83F80080404603B0AC
:10095000BDE8F08F4FF00008019B83F80080F5E7B9
:100960004FF00008019B83F80080EFE7DC230020B4
:1009700049D6B9F2E1000EE0431E9BB24FF6FD727C
:1009800093421CD84B1E9BB293421AD809010E4BBE
:1009900083FB01231944C1F3CF21C0000B4B83FB20
:1009A00000231844C0F38F20094B03EBC101085CFE
:1009B00000F07F0013288CBF002001207047012029
:1009C00070470120704700BFE1000EE049D6B9F240
:1009D000DC230020F8B506460F4C2568238903EB7D
:1009E00083035B00F4336B8005F0A2FD043523899B
:1009F00003EB830307690A22314605EB4300B8473E
:100A0000238901339BB22381226852789A4201D80C
:100A100000222281F8BD00BF60240020704708B585
:100A2000FFF7D8FF08BD10B5044605F081FDC36887
:100A30004FF44472002120469847034B1C60462324
:100A400063700A23237010BD6024002030B5A5B068
:100A50000446436898474F4B1B7913F0030F09D0A6
:100A6000A368984710F0080F21D1A368984710F0A9
:100A7000040F1CD1474B1B7913F00C0F09D0A3684E
:100A8000984710F0020F41D1A368984710F0010F6A
:100A90003CD1A36898473F4D2871E36804A8984764
:100AA000BDF81830EB8000236B8125B030BD0025E8
:100AB00001950295ADF80C5005F03AFDC3680A2285
:100AC000294601A898479DF80430022262F30203E8
:100AD0008DF80430E36810A89847BDF80430BDF8DD
:100AE000462062F30F13ADF80430E3680CA8984772
:100AF000BDF83E30ADF80630E36808A898470B9B78
:100B0000ADF8083001A8FFF765FFB3E700250195B0
:100B10000295ADF80C5005F00BFDC3680A2229467A
:100B200001A898479DF80430032262F302038DF870
:100B3000043063689847BDF80430028862F30B13F1
:100B4000ADF80430134A52891209C3F3072362F344
:100B500007138DF80530E36820A89847BDF8823068
:100B6000ADF80630E3681CA89847BDF87030ADF8C2
:100B70000830E36818A89847BDF86E30ADF80A3021
:100B8000E36814A89847179BADF80C3001A8FFF74D
:100B900021FF7EE7602400202DE9F04FA9B0044634
:100BA00043689847A368984710F0080F04D1A368DA
:100BB000984710F0040F39D0236898474368984746
:100BC000054600F06CFA80B123689847436898475F
:100BD0008146002704970597ADF8187002460A2150
:100BE00004A800F048FAB846EEE0284600F05BFAA8
:100BF0000028E9D163689847B0F86030002B40F0D6
:100C00007381B84BDD880135E36818A89847BDF8B3
:100C100068309D4200F0D781E3680EA89847B14B39
:100C2000BDF84020DA805A8901325A8129B0BDE8E6
:100C3000F08FF36828469847336928469847236819
:100C4000984743689847834600F035FAB0F1000AA8
:100C5000C0F2448163689847C388ADF80830636880
:100C600098470389ADF80A30636898474388BDF810
:100C700008201344ADF80C30636898478388BDF8AA
:100C80000A201344ADF80E305FFA8AFADBF80C3014
:100C9000504698470190DBF810305046984702AA1A
:100CA0000146019800F0C0F9002840F019814FF486
:100CB000C973ADF8083040F66A03ADF80A3040F267
:100CC000A623ADF80C3040F62413ADF80E30DBF857
:100CD0000C30504698470190DBF81030504698474A
:100CE00002AA0146019800F09FF9003018BF0120C8
:100CF0009DF8223060F345138DF8223063689847E1
:100D000090F86330C3F302039DF8242063F30202DA
:100D10008DF824206368984790F866A00AF0FD0AD1
:100D20006369984701280ED14AF0020A6368984720
:100D300090F86830FF2B06D06368984790F86830C9
:100D4000013380F868306368984780F866A063686C
:100D50009847BDF8243090F8662062F3C803ADF8D8
:100D60002430B368284698479DF8253060F3820305
:100D70008DF82530B369284698471F2828BF1F20C3
:100D8000BDF8223060F38A13ADF82230F3692846AB
:100D900098471F2828BF1F209DF8233060F3C70302
:100DA0008DF82330336A28469847C0F38F001F28F8
:100DB00028BF1F209DF8253060F3C7038DF825302C
:100DC00007A8FFF707FE0137D9F800309847FBB2B4
:100DD0008342BFF40FAFFBB228AA134413F8905C10
:100DE000CDF81C80CDF82080ADF82480D9F82830CB
:100DF00028469847012805D0D9F828302846984732
:100E00000328E0D123689847436898470646E3687B
:100E10000AA89847BDF82CA005F08AFBC3680A22EF
:100E2000414607A898479DF81C306FF302038DF8E0
:100E30001C30B36A28469847012814BF00200120BF
:100E40009DF81C3060F3C3038DF81C30BDF81C30D6
:100E5000BDF82E2062F30F13ADF81C304FEA1A12C2
:100E60009DF81E3062F303038DF81E309DF820308C
:100E70006AF303038DF82030F36828469847BDF8DD
:100E80001E3060F30F13ADF81E30336928469847C3
:100E9000BDF8203060F30F13ADF82030236912A89D
:100EA00098479DF822309DF8482062F301038DF8A1
:100EB0002230736A284698479DF8223060F38303F6
:100EC0008DF8223003F00C030C2B7FF4B2AE9DF8AA
:100ED000223043F00C038DF82230AAE6404607E7A3
:100EE000012005E76024002000230A930B93ADF84E
:100EF00030302368984743689847064600F0DBF88F
:100F0000051E4FDB05F014FBC3680A2200210AA866
:100F100098479DF82830012262F302038DF82830AB
:100F2000E36814A89847BDF82830BDF8562062F34E
:100F30000F13ADF828306368984790F8603013F0CD
:100F4000020F3AD16368984790F8603013F0040FAD
:100F500035D16368984790F8603013F0080F30D1AE
:100F60006368984790F8603013F0100F14BF0622A2
:100F700000229DF82A3062F303038DF82A30EDB287
:100F8000F36828469847BDF82A3060F30F13ADF890
:100F90002A30336928469847BDF82C3060F30F1388
:100FA000ADF82C300AA8FFF715FD636898470023B9
:100FB000A0F860301B4A538123E60122D9E70422BE
:100FC000D7E70522D5E700250A950B95ADF83050F7
:100FD00005F0AEFAC3680A2229460AA898479DF888
:100FE0002830042262F302038DF82830E36824A835
:100FF0009847BDF82830BDF8962062F30F13ADF87E
:101000002830E36820A89847BDF88E30ADF82A3024
:10101000E3681CA898471F9BADF82C300AA8FFF77F
:10102000D9FCF9E560240020134672B1128882428F
:101030000DD89A8882420CD3DA888A420BD358881A
:1010400088428CBF0020012070470020704700209C
:101050007047002070470020704710B504460846CE
:1010600011460023224600F0BBF90021204600F083
:10107000E4F9C0B210BD08B5002300F0B1F908BD15
:1010800008B500F0ADF908BD08B5002100F0D5F9AC
:10109000C0B208BD08B500F0D0F9C0B208BD08B5AF
:1010A00000F076F908BD08B500F086F908BD08B56E
:1010B00000F05AF908BD08B500F0E6F908BD0000D7
:1010C00010B5436898470488003418BF012405F020
:1010D0002FFA8368224603210220984705F028FA58
:1010E0008368224603210420984710BDF8B50746BF
:1010F0000F4B1B68BBB1002425460D4E56F825301A
:1011000053B156F82530984703682BB156F825306F
:1011100098470368384698470134E4B2254656F8A4
:101120002430002BEAD13846FFF7CAFFF8BD00BFD4
:10113000280F0020F8B50746124B1B68F3B10024B6
:101140002546104E56F825308BB156F82530984775
:1011500043683846984750B156F825309847C368D9
:101160002BB156F825309847C36838469847013464
:10117000E4B2254656F82430002BE3D13846FFF779
:101180009FFFF8BD280F00202DE9F04107461A4BBC
:101190001B68002B2DD000242646174D05E0013496
:1011A000E4B2264655F824301BB355F82630002B00
:1011B000F5D055F8263098474368384698470028B8
:1011C000EDD055F82630984790F81480BB689847C2
:1011D00018EA000FE3D055F8263098478368002BB3
:1011E000DDD055F826309847836838469847002860
:1011F000D5D0BDE8F08100BF280F00202DE9F041D7
:1012000007461C4B1B68002B32D000242646194D84
:1012100005E00134E4B2264655F824302BB355F8E6
:101220002630002BF5D055F82630984743683846CD
:1012300098470028EDD055F82630984790F814804C
:10124000BB68984718EA000FE3D055F82630984756
:101250000369002BDDD055F82630984703693846DE
:1012600098470028D5D0012000E00020BDE8F0819B
:101270000020FBE7280F002008B543689847007856
:10128000C0F3400008BD704730B587B0044603681E
:1012900098474368984702461F4903A800F0E9FCB5
:1012A0009DF8153013F0020F2ED0BDF80C30CD3B59
:1012B0009BB240F29D22934229D8BDF80E2040F601
:1012C0007B039A4225D99DF81430043BDBB2382BBE
:1012D00001D9002019E00023019302934FF002038B
:1012E000012565F387138DF8043005F021F9436873
:1012F00001A898476368984790F8603043F002036C
:1013000080F86030284600E0002007B030BD0020A3
:10131000FBE70020F9E700BF6C24002008B54FF47C
:101320009F7354224021024800F08EFC08BD00BF8C
:101330006C240020004870471CCB010010B51446F7
:10134000012802D0022805D010BD1A46204600F020
:1013500081FDF9E71946104600F04AFDF4E701481F
:10136000704700BF34CB010038B505460368984785
:1013700048B10024AB68E0B29847034630B9013465
:101380000A2CF7D100E00023184638BD0123FBE703
:1013900038B505460368984750B10024AB6AE0B2FF
:1013A0009847012806D001340A2CF7D1002000E02C
:1013B000002038BD0120FCE738B505460368984792
:1013C00050B10024AB6AE0B29847032806D001343C
:1013D0000A2CF7D1002000E0002038BD0120FCE7F6
:1013E0002DE9F84F824689461646984600252F4635
:1013F00009E07B1CDBB20AF807404B451BD01F46B7
:1014000001350A2D17D0ECB2B36A20469847002860
:10141000F6D0F368204698478346336920469847BC
:10142000B8F1000FE5D0424601465846FFF7FCFDF3
:101430000028DED1E4E7BDE8F88F2DE9F843074640
:1014400088460024264604E00136F6B201340A2C10
:1014500017D0E5B2BB6A284698470028F6D0FB684B
:101460002846984781463B6928469847B8F1000FBF
:10147000EAD0424601464846FFF7D6FD0028E3D1B0
:10148000E4E770B2BDE8F88338B5054603689847CD
:1014900060B10024AB6AE0B2984728B901340A2C45
:1014A000F8D14FF0FF3038BD60B2FCE74FF0FF30AD
:1014B000F9E7000008B5436898470078C0F3C0001A
:1014C00008BD064B43221A80BE225A8040F2F532F4
:1014D0009A8040F6B502DA80704700BF8824002069
:1014E000F0B585B0044643699847244DA876236833
:1014F000984743689847024605F1080102A800F0A2
:1015000078FA9DF80830022B03D00025284605B054
:10151000F0BDBDF80A70BDF80C602A463146384669
:10152000FFF782FD05460028F0D0002300930193C9
:101530004FF00203042262F38503012565F387134C
:101540008DF8003047FA02F38DF8023046FA02F3C4
:101550008DF8033006F00F0646EA07168DF8046092
:1015600004F0E6FF4368684698476368984790F838
:10157000603043F0080380F86030C7E7882400201B
:1015800010B584B00D4C46230393642302931E23AD
:101590000193032200921223012104F1080000F0BC
:1015A00001FA43232380BE23638040F2F533A380F6
:1015B00040F6B503E38004B010BD00BF88240020CE
:1015C000004870473CCB010008B543689847037852
:1015D00013F0240F14BF0120002008BD38B5436864
:1015E0009847C58804894188294482882244034B4E
:1015F0005D809C80D9801A8138BD00BFC024002046
:101600002DE9F04784B08046436898470378C3F3D8
:101610008009C3F34017D8F8143098473F4D85F838
:101620002600D8F80030984743689847024605F1ED
:10163000140102A800F0DDF99DF808A0BDF80A60C9
:10164000BDF80C40AA1C21463046FFF7EDFC30BB2C
:1016500005F10A0221463046FFF7E6FC0346002862
:101660005AD1184604B0BDE8F0872C4B1A700023FD
:10167000F7E71FB3294B1B78012B1FD00023F0E79E
:10168000D8F80430984790F8603043F0040380F8AD
:1016900060300123E5E70023E3E70023E1E70022D0
:1016A000BAF1010FE1D0BAF1020FF4D1B9F1000F94
:1016B000DFD01FB9194B1B78002BEED1002301930B
:1016C0004FF00203012262F3850362F387138DF862
:1016D0000030124D2B788DF8013033118DF8023027
:1016E00023118DF8033004F00F0444EA06168DF838
:1016F000046004F01DFF4368684698472B78002B70
:10170000BED0D8F80430984790F8603043F02003FA
:1017100080F860300123A4E70122C1E7C024002043
:1017200030B587B00546036904A898479DF8133083
:10173000FBB9264C4623039364230293242301938D
:101740000523009312230222114604F1140000F035
:1017500029F96B689847C588018942882A4483889B
:101760000B446580A180E28023816F2140F6F40262
:101770001FE0164C0A23039364230293242301934E
:101780000723009312230322022104F1140000F026
:1017900009F96B689847C588018942882A4483887B
:1017A0000B446580A180E280238140F22C4140F609
:1017B0006602064B43205881998140F2F531D98168
:1017C0001A8200221A7007B030BD00BFC02400206A
:1017D0000048704754CB010010B50446028B038AC1
:1017E0009A4202D90123C375037594F82730012B5F
:1017F00012D0A37C012B14D0A27D0D4B53F82230C4
:1018000020469847012811D0022814BF002002204A
:10181000A38D0133A38510BD0423E3750123237534
:10182000E7E70523E37501232375E5E70120EFE7EB
:10183000380F0020C289B0F91A30B0F922105B1AB3
:10184000002BB8BF5B42934218DCB0F91C30B0F9F2
:1018500024105B1A002BB8BF5B429A4210DBB0F930
:10186000282043889A4207DCB0F92C304089834213
:10187000CCBF002001207047002070470020704737
:101880000020704770B5044690F82650012D05D908
:10189000AB1EDBB2012B08D9002070BD01230375FC
:1018A0000020A0750323E375F7E7068D013636B2F5
:1018B0000685FFF7BFFF08B901232375032D01D06B
:1018C0000020EAE723889E42BCBF0123237563887A
:1018D0009E42C4BF012323750023A375627D237B31
:1018E0009A4201D00020D8E7B4F92A30A288934266
:1018F000BCBF01222275E2889342C4BF0123237535
:10190000B4F92C3022899342BCBF0122227562892E
:101910009342C4BF0123237500236385237D4BB10C
:1019200000202075A685E38B6383238CA38301238A
:101930006375B2E7002363750220AEE710B5044675
:1019400090F8263023B9438D01334385002010BD24
:10195000012B25D1FFF76EFF18B90223E375012390
:10196000237501222285637D1344DBB26375A27562
:10197000B4F92210E183B4F9242022843BB1237D01
:101980002BB9607D012814BF00200120DFE7002073
:1019900020750123A38560856183A2836375F0E7C9
:1019A0000020D4E730B4BDF80850BDF80C400280E8
:1019B000438001FB02F292B2AB1A8380A21AC2806A
:1019C000058144810173BDF81030C381BDF8143026
:1019D0000382002303754375438583850385C3759F
:1019E0004FF6FF7242838283C2830284837530BCC8
:1019F0007047F0B585B005460C46164600230193A6
:101A00000293ADF80C30898B608BFEF7B5FFD0B137
:101A10000A2201A93046FEF723FF012822D900231C
:101A2000237563756385A3852385E3754FF6FF7280
:101A30006283A283E2832284A3752B706B80AB80C8
:101A4000284605B0F0BD0023237563756385A38523
:101A50002385E3754FF6FF726283A283E2832284BB
:101A6000A375D5E79DF8047000B3F368384698472E
:101A70006084336938469847A084B36A38469847EB
:101A800084F82600B3693846984720833046FFF72C
:101A90000EFBA0B9002384F827302046FFF79CFEF8
:101AA000628BA38B28706A80AB80C9E74FF6FF7307
:101AB0006384A384002384F826302383E6E701238C
:101AC00084F82730E9E700BF70B504460E46157864
:101AD0008B6A28469847012801D0012070BD002359
:101AE00023806380A380E38023816381A381E381DA
:101AF00023746374227E02F0F80263F3C302227639
:101B0000F36828469847A081336928469847E081C2
:101B1000237C01332374E0E72DE9F04104460F46AE
:101B20001678CB683046984780463B6930469847E0
:101B30000546BB6A30469847032841D0A389A8EBE5
:101B400003031BB22380B4F902209A42B8BF1A469D
:101B500016466280B4F904709F42A8BF1F46A78052
:101B6000E089281A00B2E080B4F908208242B8BFA8
:101B700002462281B4F90A108142A8BF0146618160
:101B8000B4F9125001EB050C604553DA491B884249
:101B900050DD521B904203DC227E42F0020222768C
:101BA000EA1993424BDA7F1BBB4248DD721B93421A
:101BB000DEBF237E43F0080323760120BDE8F081D9
:101BC00000232374B4F90020E38A9A4222DB217EA9
:101BD00001F00801002914BF0020102059428A4258
:101BE00006DC227E12F0040F04BF40F00800C0B2F1
:101BF000B4F9062093420FDC237E13F0020F0BD1C1
:101C000040F00400C0B29142D8DB237E13F0010FF4
:101C100008D0D3E70020E1E7914207DB237E13F0F1
:101C2000010F03D140F00200C0B2C7E7002808BF8F
:101C30000120C3E7217E41F001012176A9E7227E40
:101C400042F004022276B1E741828282C3820023FD
:101C5000038043808380C380038143818381C38168
:101C600003744374027E02F0F80263F3C302027647
:101C700070472DE9F04186B004460D461646002314
:101C80008DF81730314903AA03C982E80300009395
:101C90000193ADF808300A2269463046FFF7DDF9B6
:101CA00080469DF800708DF81770B36A38469847E3
:101CB000002831D0B8F1010F2ED1B36938469847CA
:101CC000AB8A834228D3B3683846984720BBF36871
:101CD0009DF817009847804633699DF8170098478C
:101CE00007462B7C06AA02EB830353F80C3C0DF14C
:101CF0001702314628469847A989EA896B7C5E1C01
:101D00006E7421806280A4F80480E7802372607280
:101D1000204606B0BDE8F08100232B806B80AB80AD
:101D2000EB802B816B81AB81EB812B746B742A7EF2
:101D300002F0F80263F3C3022A7623806380A38053
:101D4000E380237201236372E2E700BF6CCB0100E2
:101D5000014B1888704700BF042500200A207047F7
:101D6000024B5B6803EB0010807B7047042500206A
:101D7000024B5B680001185C704700BF042500201F
:101D8000024B5B6803EB001040887047042500207D
:101D9000024B5B6803EB001080887047042500202D
:101DA000024B5B6803EB0010C088704704250020DD
:101DB000024B5B6803EB001000897047042500208C
:101DC000024B5B6803EB001040897047042500203C
:101DD000024B5B6803EB00108089704704250020EC
:101DE000024B5B6803EB001040787047042500202D
:101DF000014B198058607047042500200048704747
:101E000074CB010001EB4011024B1B6833F9110048
:101E1000704700BF0C25002001EB4011024B5B68AE
:101E200033F91100704700BF0C25002001EB401171
:101E3000024B9B6833F91100704700BF0C2500204E
:101E400001EB4011024BDB6833F91100704700BF12
:101E50000C250020014B43F8210070470C25002081
:101E6000014B03EB80007047A0CB0100704700BF1F
:101E70002DE9F043054683B0092002F04BFB804674
:101E80000A2002F047FB07460DF0CEFE0446194E2D
:101E900098F80000184902F04FFBDFF86C903246CA
:101EA0002046002103F080FBEDB298F800001349B2
:101EB00002F042FB2B4642462046494600960FF070
:101EC000CBF838780E4902F037FB32462046002125
:101ED00003F006FF38780B4902F02EFB00962B46E4
:101EE0003A4609F1240120460FF004F903B0BDE899
:101EF000F08300BFD14500008D570000515700000E
:101F0000415F0000495E0000280E0020002330B52C
:101F10000F4A104D83B0044629461268632000938F
:101F20008DF8043000F0CEFC0120FFF7A1FF0A4B32
:101F300029461A68632000F0C5FC01238DF80030A3
:101F400000989DF8043020602046237103B030BD16
:101F5000A0040020288C0100A404002038B50B4BFD
:101F60000B491A68632000F0ADFC0A4C04F1180517
:101F700054F8043B1B699847AC42F9D1064B04491D
:101F80001A686320BDE8384000F09CBCA004002023
:101F9000648C010028000020A404002010B50B4B25
:101FA0000B4C1A682146632000F08CFC094A0A4B4E
:101FB000127853F82230DB689847084B2146BDE879
:101FC00010401A68632000F07DBC00BFA004002010
:101FD000588C0100400F002028000020A40400209D
:101FE00010B50B4B0B4C1A682146632000F06AFCBD
:101FF0000021094B094A1B6811705B689847084B20
:102000002146BDE810401A68632000F05BBC00BFA9
:10201000A00400204C8C010028000020400F00206C
:10202000A404002000232DE9F041504D8CB004465B
:1020300002A800938DF8043007F062FE2B78002B85
:102040005FD04B4A4B4B1278684653F822309B685E
:1020500098472B789DF817209A4250D09DF817305A
:10206000DBB2002B2B700CBF02250125424B9DF8E3
:102070002A201978914204D09DF82A00C0B2187025
:1020800030B39DF8203013B101238DF800309DF856
:1020900021301BB10122394B83F82220012D1AD0A7
:1020A000022D0BD09DF8002082BB00989DF80430D3
:1020B0002060204623710CB0BDE8F08107232C4D31
:1020C0008DF800302B78052BEFD00527B8460BE0B4
:1020D0000AF07CFAD5E70623254D8DF800302B78E1
:1020E000042BE2D00427B846224E56F82330DB6892
:1020F000984756F828302F705B689847D5E7002539
:10210000B4E79DF81720002AA4D19AE7184D013AA8
:1021100029780B46062AC8D801A050F822F000BF43
:102120003D21000055210000AB2000004B210000A4
:10213000AB200000E1200000C72000000029B4D03F
:1021400001290CD00027B846CEE70329ADD00327DC
:10215000B846C9E70129A8D00127B846C4E700223C
:102160000748174602709046BEE700BF420F0020A6
:10217000400F002028000020410F0020BC0D00204F
:10218000B80D002038B5114B11491A68632000F0D2
:1021900099FB0AF099FF10B90E4B1A789AB90E4CB8
:1021A00004F1180554F8043B1B689847AC42F9D178
:1021B00000240A4B0A4A1C70126805496320BDE8D6
:1021C000384000F07FBB1870E9E700BFA004002092
:1021D000408C0100420F002028000020400F00200A
:1021E000A404002030B4184D0022D5F8014001327B
:1021F0002346186802EBC201294480B1586898B19F
:102200009868B0B1D868C8B1042A1BD0D1F80130A1
:102210000132186802EBC20129440028EED120687F
:10222000186058680028EBD16068586098680028EA
:10223000E8D1A0689860D8680028E5D1E068042A51
:10224000D860E3D130BC70474004002030B4184D52
:102250000022D5F8014001322346186802EBC20182
:10226000294480B1586898B19868B0B1D868C8B1AD
:10227000042A1BD0D1F801300132186802EBC201E8
:1022800029440028EED12068186058680028EBD156
:102290006068586098680028E8D1A0689860D8689D
:1022A0000028E5D1E068042AD860E3D130BC70474B
:1022B0007004002010B501F0EBFF094B1B68984734
:1022C000084B1B689847084B1B689847BDE81040AF
:1022D000064A074B127853F822305B68184700BF54
:1022E00014000020800D0020480D0020440F002025
:1022F00098930100F0B50024A3B017AE21463046F4
:102300002C2211ADCDE91144CDE913441594ADF85B
:10231000584016F054FB0BABCDE90333CDE908442C
:10232000CDE90644CDE90056074F05930EA80C945D
:102330000B94CDF833402B463C682A460290294640
:102340000B20A04723B0F0BD0C2600200B4A08B597
:1023500012780B4B53F82230DB689847FFF7CAFF1F
:10236000084B1B699847084B1B699847074B1B692B
:102370009847BDE8084001F027BF00BF440F002088
:102380009893010014000020800D0020480D0020CB
:1023900070B505468AB007F063FF022D24D0032DE7
:1023A00020D0012D044614BF04460024274D2B786D
:1023B000A34215D0684607F0A3FC2B78012B15D05B
:1023C000234E56F82330DB68984756F824302C709B
:1023D0005B68984728780AB0BDE8704007F046BFB0
:1023E0000AB070BD0224E1E70124DFE7002CE7D149
:1023F0009DF822309BB90AF067FED8B100242A78F4
:10240000134B53F82230DB689847124B2C705B68F3
:10241000984722461049642000F054FADAE70AF09F
:1024200017F8044609F0AEFF0AF04EFE0028E5D189
:10243000002CE3D10024FFF789FF2C70FFF73AFF4F
:1024400022460649642000F03DFAC3E7440F00200D
:102450009893010014000020449301007093010040
:102460002DE9F04792B007F02FFC08A807F048FCD0
:10247000584A594B127806A853F82230574C9B689B
:1024800098479DF819909DF81A6003F0D7FF07F060
:10249000F7FE22789DF8263082469A4206D09DF8B3
:1024A000260005F01FFF9DF826302370012400252B
:1024B0004B4BDFF84C81986805F0C0F949484A4F0A
:1024C0002246214643460390CDE9015500946420FD
:1024D00000F0ACF93B6898F80020997891420FD051
:1024E000CDE901552546414A023303920094224624
:1024F0002146642000F09AF93B689B7888F8003008
:102500000DF0C6FE3B688DF81700DB7883421BD1C7
:10251000BAF1000F29D145BB5EB39DF83930002BCD
:102520009DF8383018BF00263BB3002007F09EFE10
:102530004FF00109012E2DD076BB4846FFF728FF4A
:10254000012012B0BDE8F087012200232848CDE920
:10255000013303900DF1170364200092114600F03F
:1025600065F93B68D8780DF07FFE002007F08EFEFD
:1025700002269DF83830002BD7D19DF82F30FBB9BB
:102580009DF82730002BD5D007F06AFE0228CCD06A
:10259000012ED1D10FF018FB164B17491A68632092
:1025A00000F090F9FFF7D2FEFFF784FE134B1249BB
:1025B0001A68632000F086F9012012B0BDE8F087A8
:1025C00007F04EFE0228B0D09DF82730002BB1D086
:1025D000DAE700BF440F002098930100430F00206A
:1025E00028060020109301005C0600201C930100C7
:1025F00038930100A0040020FC920100A4040020F4
:10260000D40400202DE9F0479CB0044602A8884677
:1026100007F076FB0023524E9DF81F20C6E90033D9
:10262000C6E902333382002A54D094F82B0094F880
:102630002AA094F82990504594F828E036D8A0F1C3
:102640001B01A0F10F07821EC9B2FFB2D2B2F14541
:1026500022D84B4612E0A3F10A04022C3DD800EB2D
:10266000431438F91450022436F914C0AC45B8BFED
:1026700026F814500133DBB29E450DD3022AEAD965
:10268000022F33D8A3F10A04022C41D800EB4314E3
:1026900038F914500524E7E70130C0B201310137A1
:1026A00001328245C9B2FFB2D2B2D0D23E2200215D
:1026B0000DF1320016F083F9002340F60115822453
:1026C00000961A460CA91E20ADF830508DF8354002
:1026D00007F044FF1CB0BDE8F0879C1F022C23D8F4
:1026E00000EB431438F914500124BDE70229C1D886
:1026F000A3F10A04022C20D99C1F022C29D99C1E6C
:10270000022CB7D800EB431438F914500624ABE779
:102710009C1F022C17D99C1E022CABD800EB431433
:1027200038F9145003249FE79C1E022CA2D800EB1A
:10273000431438F91450002496E700EB431438F999
:102740001450082490E700EB4315042438F9155081
:102750008AE700EB431438F91450072484E700BFDC
:10276000480F0020F0B5204E83B0054601F120004F
:1027700014461F467160FDF785FD1C4B1C4A996885
:10278000213037604860946060782278E37802FBFB
:1027900000F203F07F0303FB02F3164C22790B6077
:1027A000D3B2012B01D003B0F0BD7721FF221E462A
:1027B000114F397022712379FF2B10D12022294625
:1027C000684616F0CDF8009B032B04EB830206DC71
:1027D000019BD2F8052006FA03F31342EBD105233F
:1027E0003B7003B0F0BD00BF8419002080060020BC
:1027F00064080020FC1B00203007002070B515463F
:1028000000F120042046DF220E4616F097F945B16C
:102810003046FDF737FD2946C0F1DF02204416F0AF
:102820008DF92046BDE87040FDF72CBDF0B5C3B072
:1028300004460E4615460146202202A81F4616F001
:102840008FF8029B032B0EDC01221D48039900EB3D
:102850008303D3F805C002FA01F313EA0C0F02D088
:102860000379934201D043B0F0BD4FF48072002150
:1028700002A816F0A4F800234B99DF220AA8CDE99C
:10288000003316F05BF90AA8FDF7FCFC9DF803C0C5
:10289000489B499A8DF8070063F3060C20464A9C32
:1028A00062F3C71C3B4602A96A468DF800608DF8AA
:1028B00001508DF806408DF803C0FFF753FFD2E7B3
:1028C000FC1B0020F0B5C3B004460D461646014679
:1028D000202202A816F044F8029B032B0DDC0122F3
:1028E0001649039801EB8303D3F8057002FA00F34D
:1028F0003B4202D00B79934201D043B0F0BD002798
:102900004FF48072394602A816F059F8324629462B
:1029100002A8CDE90077FFF771FF3B468DF807006D
:102920006A4602A92046ADF800708DF803708DF854
:1029300004708DF80670FFF715FFDEE7FC1B002022
:10294000F0B585B0654601F043FE01F073FE00214D
:10295000084601F027FBD5E90121044600270120A4
:102960000426CDE90107054823460390009672200E
:10297000FFF75CFF204605B0F0BD00BF5495010095
:102980002DE9F04790F815C082B0BCF1000F2BD0B4
:102990001C4600254FEA4C0606EB8C0603EB061698
:1029A000216294F8247084F8245094F8257084F8F7
:1029B000255094F8267084F8265094F8277084F8EF
:1029C000275094F8287084F8285094F8297084F8D7
:1029D000295094F82A7084F82A5094F82B7084F8BF
:1029E0002B503034A642DBD1BCF1000F2FD09846DB
:1029F0009146824600269AF814301BB300257700D2
:102A0000DAF8003006225C5D68466110013115F08D
:102A1000A7FF9AF8142004F0010406FB0291009B22
:102A20003C449B0004EB440403EB041401984B5D0D
:102A30004444216A00EB8000834001350B43AA42E5
:102A40002362DDDC9AF815300136B342D3DC02B0E4
:102A5000BDE8F0872DE9F04100241962196593F86B
:102A6000241083F8244093F8251083F8254093F828
:102A7000261083F8264093F8271083F8274093F810
:102A8000541083F8544093F8551083F8554093F848
:102A9000561083F8564093F8571083F8574093F830
:102AA000281083F8284093F8291083F8294093F8D8
:102AB0002A1083F82A4093F82B1083F82B4093F8C0
:102AC000581083F8584093F8591083F8594093F8F8
:102AD0005A1083F85A4093F85B1083F85B40017DED
:102AE00082B019B306461D46571E3368062213F8F6
:102AF000048068464FEA6801013115F031FF08F0A3
:102B0000010800994FEA480290448A0002EB08123B
:102B100001992A4417F8013F106A01EB81018B40AB
:102B200003431362337D0134A342DEDC02B0BDE80F
:102B3000F08100BF2DE9F04F95B004AFD1F801301E
:102B400004463863022100203B6101F02BFA00218A
:102B50003862084601F026FA01F06CFBEC46257D50
:102B6000647D804604FB05F2D01DC008ACEBC000BC
:102B70008546EC46960006F10A03DB08ACEBC30C75
:102B800004A8E54600210DF1100CC7F824C0FC6232
:102B9000FE60786115F013FF3246FF21786A15F068
:102BA0000EFF042307F1400202F8043D1146012004
:102BB0007A6001F05FFC3B699A68AB009178FB6139
:102BC000D37812785B1A01339A4240F32F810A239B
:102BD0004FF000092E46BB626300BB60BB6A984998
:102BE0001F2B40F310811A4601FB03F103EB431343
:102BF00002EB431303EBC33301F1404103F14043C4
:102C00002031904A013341F01F018F489362C2E99D
:102C1000081330328242F8D1012204248B4B0192F6
:102C2000CDE902930094BD6A11467B686420FD6380
:102C3000FFF7FCFD3D6AFA680021284615F0BFFE4B
:102C4000FB6A002B00F0D38000234FF0405B7D63D4
:102C5000BB614FF0000A01254FF4FA74BB693A6971
:102C60005344137701F0B4FC01F0E4FC8BF8F3500B
:102C7000D6B1D7E90C3C186806EB000E10F8013B02
:102C800003F0010252450BD15B1008EBC313B3F8FC
:102C900040201988DCF80030521A1344CCF8003078
:102CA00070450CF1040CE9D1013C8BF8F390D9D1BB
:102CB000BAF1000F02D14FF0010ACDE77A6BF96942
:102CC000BB690A447A63BA6802339342BB61C0D1DC
:102CD00004235F4ACDE90034CDE902423D6A324621
:102CE0002B46F96A6420FFF7A1FD7B6AD7F814A090
:102CF000D7F828B0A5F1040CA3F1040E86B17246F2
:102D00006046002350F8041F52F8045FA94238BF00
:102D10000AF803B003F1010338BF11609E42F1D1FC
:102D2000FB6901349C449E44FB6AB244A342E5D152
:102D30000123484ACDE90039CDE90292FD6A7B6959
:102D4000324629466420FFF771FD0423BA6A2946FA
:102D500001321446BA62404ACDE90039CDE9029207
:102D600064207B6A3246FFF761FD3E2C7FF436AF6C
:102D7000FB6A3546B3B100227B6A384E191F5DB13C
:102D80000C46002054F8043F0130A6FB03C38542E3
:102D90004FEA53132360F5D1FB6901321944FB6AF2
:102DA0009342ECD1002400222D496420FFF78AFDD4
:102DB0000122284B642003937B69CDE901440092F2
:102DC000FE6A2A463146FFF731FD22462549642036
:102DD000FFF778FD0420CDE901441F4B2A460393F9
:102DE0007B6A314600906420FFF720FD23E0184BFA
:102DF00032460393F96A0094CDE9011164203B6ADD
:102E0000FFF714FD94E7BB6A1A4601FB03F103EBDD
:102E1000431302EB43130B4A03EBC3330A48936299
:102E2000C2E9081330328242F8D1F5E600220E4999
:102E30006420FFF747FD4437BD46BDE8F08F00BF73
:102E40002084100298000460380604608C9401000D
:102E500098940100AC940100B8940100D34D621025
:102E6000C4940100D8940100E89401002DE9F043D6
:102E7000437D8646007DF3B1002601F1FF3C0F49FA
:102E80004FEA430898B16446DEF80020871812F82C
:102E9000019B14F8015F09F00103334403EB430382
:102EA00001EB031303EB59039742DD73EFD10236B5
:102EB00046458444E6D1BDE8F08300BF9800046035
:102EC00070B5644684B0DCF800000E460125FFF7BB
:102ED000CDFFD4E901210020054CCDE901003346A6
:102EE000009503946420FFF7A1FC04B070BD00BFFF
:102EF00058940100427D02B3F0B40026037DDFF850
:102F00003CC0ABB100247700056806FB03122D5DC1
:102F100005F001033B4403EB43030CEB031303EB0A
:102F20005503DB7B1355037D0134A342ECDC427D6A
:102F30000136B242E5DCF0BC70477047980004608F
:102F40002DE9F04F8146A5B0049160220F460CA8F0
:102F5000002115F034FD4FF4B4620021864815F0CD
:102F60002EFD99F81480B8F1000F21D0002301251F
:102F7000D9F800607C7F9C4217DCBA7F9A4214DB50
:102F8000F25C02F0010E4FEA4E0171441F2A0DF16E
:102F9000900E05FA02FC0EEB011100F3578251F876
:102FA0005C2C42EA0C0241F85C2C01334345E2D12F
:102FB00099F81550002D00F0598200210124D9F80C
:102FC0000420A81812F8013B04FA03F3904241EAE6
:102FD0000301F7D1C1F3130200234FF0405C9DF8C9
:102FE0003E00049E9DF86E707668140C20F00F0071
:102FF00092B22043ADF83C20ADF86C209DF8312012
:1030000027F00F078DF83E0030783C436FF3C30282
:103010008DF86E408DF85F00BDF838408DF88F0058
:103020008DF831209DF83A009DF85E2004F00304ED
:1030300020F03F0022F01F029DF86170ADF838408B
:103040008DF83A00BDF868409DF86A008DF85E2062
:103050009DF88E2063F3C30722F01F0204F00304DF
:1030600020F03F008DF88E200696ADF85C308DF88C
:103070003B30ADF88C308DF86B308DF86170ADF869
:1030800068408DF86A00049E3269CCF84810002D23
:1030900000F0CF814FF0010B4746CDE901329A464F
:1030A000354B039341F480130B932AF003031A4624
:1030B0004FF0000ED9F804C007931CF80A30043210
:1030C0000BFA03F8C8F31308C8F30D039B00099328
:1030D000CDF814804FEA9833039CDDF818800892ED
:1030E0000A9326464FEA4E0524AB754403EB0515BB
:1030F000603D0FCD0FC60FCD0FC695E80F0086E8D7
:103100000F00019A238862F309032380002F00F047
:103110008E8102996FF000420B460F4413F8011B99
:103120008A42A8BF0A469F42F8D1D2B2E27298F80A
:103130000630002B40F05B812368059A62F31F3351
:10314000236094F82E3098F8052023F01F0399F897
:10315000151084F82E304FF00003501EA38506286A
:1031600000F28781DFE810F01C010901E300E100B3
:10317000DF00DD000A0000BF980004600B1F53450C
:1031800040F372810CEB0A031D7994F82E300BFA90
:1031900005F5C5F3044023F01F030343A58584F818
:1031A0002E30C5F31405BAF1030F12DD0CEB0A0340
:1031B00013F8040C94F82E300BFA00F00543C5F315
:1031C000044023F01F030343A58584F82E30C5F384
:1031D0001405CB1E534511DD0CEB0A03D87894F887
:1031E0002E300BFA00F00543C5F3044023F01F0313
:1031F0000343A58584F82E30C5F31405BAF1020FF8
:1032000012DD0CEB0A0313F8030C94F82E300BFAC2
:1032100000F00543C5F3044023F01F030343A585D5
:1032200084F82E30C5F314058B1E534511DD0CEBCD
:103230000A03987894F82E300BFA00F00543C5F392
:10324000044023F01F030343A58584F82E30C5F303
:103250001405BAF1010F08DD0CEB0A0313F8023C68
:103260000BFA03F31D43C5F31405236894F82E00ED
:1032700045EA133545F48015C5F3140320F01F000B
:10328000013940EA13405145A58584F82E000FDD31
:103290000CEB0A035B78C1B20BFA03F32B43C3F3C5
:1032A000140321F01F0141EA1341A38584F82E1075
:1032B000BAF1000F07D0D4441CF8011C0BFA01F13D
:1032C0000B43C3F3140383F4FF130B9883F4FF53EE
:1032D00094F82E1083F01F030340C3F3044021F041
:1032E0001F010143012AA38584F82E100BD0DB4374
:1032F000E268A17BC2F31302134021F00F0242EAFD
:103300001342A381A2733034BEF1000F57D1049B46
:10331000D9F804C0D3F8048099F814704FF0010E66
:10332000DFE6002555E700257EE700259DE701390A
:10333000514540F381800CEB0A035B7894F82E1022
:103340000BFA03F3C3F3044221F01F011143A385D9
:10335000C3F3140284F82E10BAF1000F70D0D444D5
:103360001CF8013C0BFA03F313430B9AC3F3140349
:103370001340C3F31401DB4308E0404A236882EAA8
:1033800013330B9A1340C3F31401DB4394F82E203C
:10339000A18522F01F0242EA114284F82E20A7E7FD
:1033A0004FF0000294F82E30A28523F01F0343F063
:1033B000100384F82E303034BEF1000FA7D0019AEC
:1033C00099F815302032C2F309020192039A0AF1EA
:1033D000010A60320392029A534502F120020292DE
:1033E00027DD049B99F814705B6806935DE6079BE4
:1033F0000CEB0301089B0CEB030511F8013B206863
:103400000BFA03F3226843EA103363F31F328D4251
:103410002260F2D12389099A03F003031343238125
:10342000A37A0A9A23F03F031343A37289E6FF228B
:103430007CE625B0BDE8F08F0022BAF1000F8ED1F6
:103440000B9B1340C3F31401DB439FE711F8580CA7
:10345000203A844605FA02F2C0F30100024362F307
:10346000010C01F858CCA0E500259CE62A46294627
:10347000B2E54FF0FF33002188E700BFFFFF0F00E8
:10348000002900F09F802DE9F04FD1F80120ADF523
:10349000017D0CCA93F8009093F801B01278884629
:1034A00009EB0B0708A9064605929D7893F804A03E
:1034B000DC78FFF71FFD444BF9B2481C83F8290064
:1034C00009F1010C09F1FF3083F8221083F824C0C0
:1034D00083F82500059A002A6FD1A9F10A0983F81B
:1034E00027904FF00009384B4A469E460AF03F0CA1
:1034F00005F01F0004F00F0183F8289002F1140377
:103500000EEB43039C7801326CF305049C705C88DD
:10351000112A60F38A14C4F3072561F3C6055C80A1
:10352000DD70EBD14FF04050002280F8A720347DB1
:10353000BCB14FF0010C3168234D013911F8013F46
:103540001C2BEA5402F1010209DD90F8A7E01D3BB3
:103550000CFA03F343EA0E03DBB280F8A730A24271
:10356000ECD1D8F801103046FFF7EAFC08A9304644
:10357000FFF77CFCD8F8013030465968DA68C97921
:10358000124BFFF7FDF949F640437F00012400206C
:103590000422033793FBF7F70D490290CDE900248D
:1035A000039107AB2246214664200797FFF73EF9B7
:1035B00020460DF5017DBDE8F08F0BF1010B83F87E
:1035C00027B08EE70846704700000460980004604A
:1035D00044950100F0B50C4699B0602200210746E1
:1035E000684615F0ECF930220021544815F0E7F94F
:1035F0004FF4F0709DF80130626843F008038DF8D5
:103600000130BDF80010537960F30901013BADF8BA
:103610000010032B03D8DFE803F07F6D02024FF0A8
:10362000FF344FF0405100209DF82E30ADF82C4073
:1036300043F01F038DF82E30C1F830014FF00133F5
:1036400000216D461278CDF813308DF82F20CDF87B
:103650001730CDF81B308DF81F30CDF80F308DF8B6
:103660000B100CAC0FCD0FC40FCD0FC495E80F009D
:1036700084E80F003D7D3DB33C680126254407E00A
:1036800052F85C3CA54243EA070342F85C3C1BD07D
:1036900014F8013B03F00100420002441F2B18A85C
:1036A00006FA03F700EB0212EADD12F8581C203B81
:1036B000084606FA03F3C1F301010B4363F301006B
:1036C000A54202F8580CE3D16C461C4F0FCC0FC733
:1036D0000FCC0FC794E80F0087E80F00184E0CAD11
:1036E0000FCD0FC60FCD0FC695E80F0086E80F006F
:1036F00019B0F0BD4FF0FF344FF0405100209DF85D
:103700002E30ADF82C4023F01F0343F00F038DF84B
:103710002E30C1F8300191E700204FF040519DF864
:103720002E30ADF82C0023F01F03064843F01003A1
:103730008DF82E30C1F8300180E700BF38060460F4
:1037400068060460FFFF0F00002900F086802DE965
:10375000F84FD1F80160424AD6E900531C7893F83B
:10376000018095F800A004EB0805EDB204F1010911
:1037700093F802C093F804E0DF7805F1010B5FFADB
:1037800089F9631E82F829B082F8225082F8253028
:1037900082F82490BAF1000F5AD10A3C82F82740EF
:1037A00000242F4B224698460EF03F0E0CF01F0CC3
:1037B00007F00F0783F8284002F1140308EB4303D6
:1037C0009C7801326EF305049C705C88112A6CF3BE
:1037D0008A14C4F3072567F3C6055C80DD70EBD15E
:1037E0004FF0405500221F4C1F4B85F8A72084F84E
:1037F0002F9083F82F90077DCFB14FF0010E046812
:10380000DFF85CC0013C14F8013F1C2B0CF80320CE
:1038100002F1010209DD95F8A7801D3B0EFA03F3C2
:1038200043EA0803DBB285F8A730BA42EBD10D4674
:1038300004463146FFF7CEFED5F8013020465968E0
:10384000DA68C979074BFFF705F90120BDE8F88F61
:1038500008F1010882F82780A2E70846704700BFF8
:103860004C0004603806046068060460F0B400256B
:103870004FF040530326D0F8011001248A684D749C
:103880001778042083F82C7157784FF4B47C83F8B0
:103890002D71977983F82A71177A83F82B719778AD
:1038A00083F82E71D27883F82F21D1E9002117787F
:1038B00083F8257183F88E60C9780F27491B18BFDC
:1038C000012183F8841083F8814083F8805083F8C5
:1038D000AE0083F8AF00557893F8891085EA0406A6
:1038E00066F30511022683F8891093F8A11065F399
:1038F000041183F8A11083F88D0083F8B04083F899
:10390000C570A3F8C8C083F8CC60507A517983F8A9
:103910000001907883F80501D07883F80A0183F8D4
:103920000D11117983F81011117A83F8DA10D27918
:1039300083F8A020F0BC00F07FBD00BF012138B5A6
:103940004FF04053D0F80140084693F8415100F041
:1039500029FB637C0649EDB200EBC31001EB054186
:10396000802215F021F8637C0133637438BD00BFF9
:1039700080070160D0F801305B689B7953B3F0B4E5
:103980004FF0C047144EDFF854C084B000246D4699
:1039900069463A46002052F824308032B24241F85B
:1039A000043B1844F7D1394655F8043BA0EB4303D8
:1039B0005B1041F8243080318A42F5D10134202C4B
:1039C000E5D107F50077674506F50076DED104B04E
:1039D000F0BC7047704700BF000200600008006044
:1039E0004FF04053F0B503250021D0F80100012627
:1039F00082680424177883F8E07092F801C00F27DA
:103A000083F8E1C092F802C083F8E2C092F803C0E4
:103A100083F8E3C092F806C083F8E6C0127A83F810
:103A2000E720426883F88E50D278521A18BF0122DC
:103A300083F8842083F8816083F8801083F8AE4097
:103A400083F8AF40026893F8891092F801C08CEABD
:103A5000060E6EF3051183F8891093F8A1106CF32C
:103A6000041183F8A11083F88D4083F8B06083F8C7
:103A7000C57083F88750C17F01EB4101A940A3F8CD
:103A8000C81090F82010B94228BF3946B140C9B2D9
:103A900083F8CC10517A83F80011917883F80511DE
:103AA000D17883F80A11117983F81011117A83F80B
:103AB000DA10D27983F8A020BDE8F04000F0BCBC59
:103AC0004FF04053F0B403264FF0000CD0F8010043
:103AD00001258268017F147801EB410183F8E04001
:103AE000547883F8E14097788C0083F8E270D178BD
:103AF000042783F8E310917983F8E610127A83F8AB
:103B0000E720426883F88E60D278B2EB0C0218BFCF
:103B1000012283F8842083F8815083F880C00268F2
:103B200093F88910507880EA050C6CF305114FF07A
:103B30000F0C83F8891093F8A11060F3041183F837
:103B4000A11083F88D7083F8B05083F8C5C083F856
:103B50008760A3F8C84083F8CC50517A83F80011ED
:103B6000917883F80511D17883F80A11117983F8D7
:103B70001011117A83F8DA10D27983F8A020F0BC02
:103B8000704700BF2DE9F04F93B004AF07F138053F
:103B9000654C664E45F8300D07F1240807F1140A0C
:103BA00094E80F008AE80F0007F160035046414691
:103BB000CAE902567B63FCF763FB94E80F005C4C98
:103BC00088E80F00404607F13401C8E90254FCF7C9
:103BD00057FB012000F09EFC002800F09E80002191
:103BE000E9460A46BB680546D0F801005E7D1C7DAB
:103BF0000368D0F804C004FB06FBC7E903465C7801
:103C00009CF802607C604B4C597002F1140304EB89
:103C100043035988013241F4F861112A5980F4D1E3
:103C20006A460BF10703DB08A2EBC3039D469CF831
:103C3000013004AC01695A4620463B6014F0B4FEE2
:103C40003B68BBF1000F09D0224604EB0B0012F8D1
:103C5000011B0431824202F8011CF8D148F0010234
:103C60004AF00101CDE9002101205A4619462346B8
:103C700002F0FAFDD7E903214FF0000A0123DFF833
:103C8000B8800093CDE901AACDF80C8023466420CA
:103C9000FEF7CCFDD7F810B0D34542DDD646D7E9C4
:103CA000020ABAF1000F0EDD0023027DD5F80110E3
:103CB0000EFB0232496914F802C0C95C0133614449
:103CC0005345A154F1D10EF1010EDE45E9D1214653
:103CD000FFF7CCF8D7E903214FF0000A0120234673
:103CE0000090CDE901AA6420CDF80C80FEF79EFD7E
:103CF0005246104806F01F0602F1140300EB43037E
:103D00005988013266F38A11112A5980F4D1D5F805
:103D100001303A791B685A70CD463C37BD46BDE844
:103D2000F08FB868D3E700BF908B010041290000F5
:103D3000C12E000000000460589401002DE9F04FEE
:103D4000ADF5037D04AF786001200C4600F0E2FB86
:103D50000026D0F80130D4F801201B6854685A7846
:103D6000B8605E700121914607F118004FF4F072BF
:103D700094F801A014F023FEADF5F16D0DF1100BD8
:103D8000584631464FF4F06214F019FEBAF1010FB3
:103D900053DD0124A046384DFE60ABF1040B374ED5
:103DA000304611222146303614F009FEAE42F7D1DA
:103DB00001220426324B07F114000393FB681146DD
:103DC000CDE901830096034664207C61FEF72EFD59
:103DD00000F0FEFB00F02EFCFB682A4ACDE90183CF
:103DE00003924FF0C04320220F2100967220FEF76D
:103DF0001DFD59464FF0C043DFF894C007F118028B
:103E0000186851F8046F04338642BCBF1470086010
:103E1000634502F10102F3D11B4BCDF800800393FF
:103E2000FB680134CDE90133202207F118030F218B
:103E30006420FEF7FBFCA245B1D1786807F11801B8
:103E4000FFF714F801240021BB681048D3F80130B3
:103E50001A6807F1180382F80190CDE90111039067
:103E6000202200940F216420FEF7E0FC07F5FE7786
:103E7000BD46BDE8F08F00BF47060460A7000460A0
:103E80006494010030BB0100589401007494010057
:103E90008007006030B585B000F0CCFB00210846FB
:103EA00000F080F80025044604210120064ACDE9EF
:103EB000010500910392234620220F217220FEF774
:103EC000B5FC204605B030BD30BB0100012170B506
:103ED0000446084600F066F800210546012000F07F
:103EE00061F8D4F801202B1F147C011F05F17C061A
:103EF00053F8042F02FB04F2B3424FEAE21241F8F6
:103F0000042FF5D100F17C0105F1FC0053F8042FDA
:103F100002FB04F298424FEAE21241F8042FF5D175
:103F200070BD00BF704700BF4FF0405393F8412170
:103F3000002082F0010283F8412193F8432182F0AE
:103F4000010283F8432170474FF0405310B593F8B6
:103F50002430CBB172B60E4A14689CB90D490E4B91
:103F600008681160027803EBC2035B68984701237D
:103F70000A4A1375BFF34F8F4FF0405208490C7235
:103F80001370937062B610BD0CF02EFAE2E700BF1A
:103F90005C0F0020840F0020D80400200000105087
:103FA000CC22002001290CD007D3022903D1074BD2
:103FB00053F82000704700207047054B53F820004D
:103FC0007047044B53F82000704700BFAC0F00202F
:103FD000C40F0020DC0F00204FF0C04370B5584CD8
:103FE000584E594D594962682360336029601AB1AF
:103FF0005749201D08F026F873681BB155495648EB
:1040000008F020F86B681BB15449554808F01AF8BD
:104010004F4A4FF48071534807F0A4FF4D4A4FF4C4
:1040200080714D4807F09EFF4C4A4FF480714C4818
:1040300007F098FFA3681BB14B494C4808F002F801
:10404000B3681BB14A494B4807F0FCFFAB681BB192
:1040500049494A4807F0F6FF434A8821434807F098
:1040600081FF434A8821434807F07CFF424A882168
:10407000424807F077FFE3681BB14149414807F028
:10408000E1FFF3681BB14049404807F0DBFFEB68F4
:104090001BB13F493F4807F0D5FF394A5021394805
:1040A00007F060FF384A5021384807F05BFF384A74
:1040B0005021384807F056FF23691BB1364937486D
:1040C00007F0C0FF33691BB13549364807F0BAFF26
:1040D0002B691BB13449354807F0B4FF2E4A8821BB
:1040E0002E4807F03FFF2E4A88212E4807F03AFF5E
:1040F0002D4A88212D4807F035FF63691BB12C49F3
:104100002C4807F09FFF73691BB12B492B4807F020
:1041100099FF6B691BB12A492A4807F093FF244A8B
:104120005021244807F01EFF234A5021234807F05E
:1041300019FFBDE87040224A5021224807F012BF03
:10414000C40F0020DC0F0020AC0F002000008560B1
:10415000A8950100BC950100E00F0020D895010052
:10416000B00F0020C80F0020F4950100CC0F0020F4
:1041700010960100E40F002030960100B40F0020DB
:1041800050960100D00F00206C960100E80F00202F
:104190008C960100B80F0020AC960100D40F0020CF
:1041A000C8960100EC0F0020E8960100BC0F00202B
:1041B00008970100D80F002024970100F00F00207D
:1041C00044970100C00F00202DE9F047114C124E1A
:1041D000124DDFF84CA0DFF84C90DFF84C8004F172
:1041E000140754F8043F1BB15146204607F02AFF3C
:1041F00055F8043F1BB14946284607F023FF56F8FF
:10420000043F1BB14146304607F01CFFBC42E8D1D9
:10421000BDE8F087C40F0020AC0F0020DC0F0020A9
:10422000689501007895010090950100004870475D
:10423000000084600048704700000230F8B5164660
:104240001D4604460F46FFF71BF908B10F4B1F60D0
:1042500031462046FFF778FA08B10C4B5E60069AAB
:104260002946204601F082FC18B1084B069AC3E9A2
:104270000225DDE90712204601F092FC20B1034B34
:10428000089A1A61079A5A610120F8BD640F00204C
:104290002DE9F04F8DB004AF0BF0C6FC02240546AB
:1042A0003861982200215A4814F089FB594B2A7D25
:1042B0002968D3F801000094574B00F0BFFC574B1E
:1042C0006A7D6968D3F80100554B009400F0B6FC94
:1042D0002422FF215348C7F80CD014F070FB0BF0D8
:1042E000A3FC427D067DD31D03F4FC73ADEB030DEF
:1042F00004AB7A617B6041680468B960002A79D0B8
:10430000084613460A4618180DF10F0112F8013B32
:10431000C3F12103824201F8013FF7D100F086FC8E
:10432000814600F087FC8246002E6CD0A3194FF026
:10433000010B98463B4D07F11806C7F800A014F88A
:1043400001AB08224FEA4A01304614F009FB19F983
:104350000A30B96903EBC3032B44FA69585C0BFAC2
:1043600002F20243A0455A54E9D17B69D7F800A074
:1043700013B34FF0010B7B697C6823447B61BB68FE
:1043800003F1FF3814F8011B18F8019F49000822B7
:10439000304614F0E5FA1AF90930B969023303EB33
:1043A000C303FA692B44585C01320BFA02F2024350
:1043B0005A547B699C42E5D1D7F80CD00FF0B2F982
:1043C0000FF0FAF90FF068F9FDF70CFFFDF73EFF6B
:1043D0001249154A154B009138691549CDE901324A
:1043E0000C4B144AFFF72AFFFFF7F6FD2437BD46B2
:1043F000BDE8F08F00F01AFC814600F01BFC8246FD
:10440000002ED9D092E707F11806064DB1E700BF9C
:104410000000046040040020B02E00207004002042
:104420009826002060270020640400201802002045
:104430005C0A0020A80A002008B50BF00FFF054B0E
:104440001B78984204D01846BDE808400BF0E8BE3F
:1044500008BD00BFD404002010B50BF0FFFE0446D9
:104460000BF0F0FE844203D0BDE810400BF0D8BE44
:1044700010BD00BF2DE9F04100248046104B0E46D0
:10448000202221460F481C6014F099FAA04514DD43
:104490002146013E0C4D0B4F06EB080C16F8014F60
:1044A0000A4B53F8042F1078A04204BF47F821208C
:1044B0000131AB42F5D16645F0D1BDE8F08100BFD6
:1044C0005C0F0020840F0020800F0020600F002070
:1044D00070B50E4D2C68B4B1206803780A2B12D841
:1044E0000B4E56F833309847636863B12B682268E7
:1044F000191D29603AB15868037806EBC306736842
:104500009847012070BD0020286070BD5C0F00201E
:10451000D8040020074B10B403F1200453F8042FF3
:104520001178814202D0A342F8D10022104610BC7B
:10453000704700BF600F0020044B11B143F82010FA
:104540007047034A43F82020704700BFA8040020AA
:10455000253F000070B5094C094E04F1200554F8C0
:10456000040F03785A1E092A02D856F823309847B8
:10457000AC42F4D1BDE87040FFF76EBF800F002061
:10458000A804002010B572B60C4A1468A4B90C49EE
:104590000C4B08681160027803EBC2035B68984714
:1045A0000422094B1A75BFF34F8F4FF0405301227D
:1045B00006490C721A709A7062B610BD5C0F00202A
:1045C000840F0020D804002000001050CC220020CE
:1045D000FFF7BABCFFF7D6BF002208B5054B1A7229
:1045E0000CF0AAF9044B054A1A60BDE80840FFF731
:1045F000ABBC00BFCC220020A40F0020493F00002C
:1046000008B50CF0B1F9002303480449044A0360DB
:104610000B60136008BD00BFA40F0020A80F00208E
:10462000F40F0020024B1868003018BF01207047BB
:104630005C0F002008B5084908200BF0F3FCFFF7D9
:1046400089FF0CF091F9002304480549054A0360ED
:104650000B60136008BD00BF293F0000A40F0020BD
:10466000A80F0020F40F002038B572B60CF07CF9CA
:1046700000200E490E4A0F4B08601060186062B6A9
:104680000D4B1C6884B10D4BA3F1200553F8042990
:104690002168914218BF5860AB42F7D1BDE838405D
:1046A000074908200BF0BEBC38BD00BFA40F002096
:1046B000A80F0020F40F00205C0F0020A00F0020A6
:1046C000293F000008B5044908200BF0ABFCBDE809
:1046D0000840FFF73FBF00BF293F000008B504496D
:1046E000082014F051FABDE80840FFF733BF00BFBF
:1046F000293F0000082270B5304C314D23682A60F4
:10470000B3B118680278022A31D05A6882B1FFF733
:10471000DFFE00283FD001232A4A1375BFF34F8FD5
:104720004FF040520020284908721370937012E035
:1047300001260020244A23491672244A087512686B
:104740000AB1904723681868214B027853F8323039
:1047500098470023236010221E4B2A60D3F80021C3
:1047600012071CD44FF0405300225A7070BDD0F88D
:104770000120567C002EC8D1154B1B699847012398
:10478000104A1375BFF34F8F4FF040520E490E720F
:1047900013709370DFE701220B4B1A72DBE70022E4
:1047A00008240D480D49C3F8804102704FF0405372
:1047B000C1F8402100225A7070BD00BF5C0F00207C
:1047C000D408002000001050CC220020EC22002051
:1047D000D804002000E100E0D008002000000250D2
:1047E000F0B5012A83B0164605460C461F462DDC5F
:1047F0000146684614F0B4F836B3009B3F2B1D46C3
:10480000A8BF3F25019A002B134405F03F05B8BF10
:1048100000253F2B1A46A8BF3F22002B4FF0000176
:1048200002F03F03B8BF002304F1100207EB420C73
:1048300009B30A19103207EB4202907965F30500BB
:1048400090710131B142F3DB03B0F0BD104607F0C7
:1048500053FB044106FB04F40F2C294606DD01221C
:10486000684614F07DF80126009BC7E7324668468B
:1048700014F076F8C1E79CF8062063F305028CF883
:104880000620DEE7F0B5012A83B0154604460E4641
:104890001F462DDC0146684614F062F8009B2DB3DC
:1048A0003F2B1C46A8BF3F24019A002B134404F061
:1048B0003F04B8BF00243F2B1A46A8BF3F22002B5D
:1048C0004FF0000102F03F03B8BF002306F11002D1
:1048D00007EB420CF1B18A19103207EB42029079D2
:1048E00064F30500907101318D42F3D103B0F0BD46
:1048F000104607F001FBF30744BF06416E43214613
:104900002A46684654BF06F1FF36013614F028F8EF
:10491000009BC5E79CF8062063F305028CF806208F
:10492000E1E700BF30B5DCF8103085B06446984749
:10493000FFF780FED4E90232002001210425029015
:104940000448CDE9005103907220FDF76FFFA06885
:1049500005B030BD8097010030B5DCF8103085B06F
:1049600064469847FFF766FED4E902320020012131
:10497000042502900448CDE9005103907220FDF710
:1049800055FFA06805B030BD8097010030B5DCF858
:104990000C3085B0644600259847FFF74BFE012197
:1049A0000420064AA36800900392CDE90115142261
:1049B0007220FDF73BFFA06805B030BD8097010075
:1049C00030B5DCF80C3085B0644600259847FFF719
:1049D00031FE01210420064AA36800900392CDE92C
:1049E000011514227220FDF721FFA06805B030BD2B
:1049F000809701002DE9F04F0D46CC1D890087B04E
:104A000024F007040A3121F0070106AFADEB040DD5
:104A10000DF11808ADEB010D9B4606AEBC6A9DB1C9
:104A20000023013800EB050E10F8011F1AB112F82F
:104A300001C008F803C01CB154F8211046F8231037
:104A4000704503F10103EFD1EAB14FF0010A4FF0D5
:104A500000092B4B514603932A464346CDE9019961
:104A6000CDF800A06420FDF7E1FEFB6AFA6AD3F8F6
:104A700001301178D3E9002312780A299B79524436
:104A800014D006292CD06CB14FF0000C0121042465
:104A90001C48334603902A46CDE9011C009464204B
:104AA000FDF7C4FE0437BD46BDE8F08F009340F625
:104AB0004A30CDE9036BCDE9015840F212234FF49F
:104AC000487102F055F804200F4A00900392CDE996
:104AD00001995B4651462A466420FDF7A7FED2E7BE
:104AE000009340F64A30CDE9036BCDE901588223AB
:104AF0004FF4487102F03CF80420044AE5E700BF97
:104B0000FC9701001898010004980100109801001A
:104B10002DE9F04F0D46CC1D890087B024F0070425
:104B20000A3121F0070106AFADEB040D0DF11808B5
:104B3000002DADEB010D9B4606AEBC6A13DD0023D4
:104B4000013800EB050E10F8011F1AB112F801C070
:104B500008F803C01CB154F8211046F82310704522
:104B600003F10103EFD1EAB14FF0010A4FF0000960
:104B70002A4B514603932A464346CDE90199CDF885
:104B800000A06420FDF752FEFB6AFA6AD3F80130F8
:104B90001178D3E90023127809299B79524414D063
:104BA00005292CD06CB14FF0000C012104241C48C5
:104BB000334603902A46CDE9011C00946420FDF79A
:104BC00035FE0437BD46BDE8F08F009340F64A300D
:104BD000CDE9036BCDE9015840F212234FF448713F
:104BE00001F0C6FF04200F4A00900392CDE901991D
:104BF0005B4651462A466420FDF718FED2E7009333
:104C000040F64A30CDE9036BCDE9015882234FF4D9
:104C1000487101F0ADFF0420034AE5E7D497010095
:104C2000F0970100DC970100E89701000048704709
:104C3000B02E002000487047982600202DE9F04F44
:104C400085B0406804AFD7F828904578D01D20F093
:104C5000070009FB05F5ADEB000D0DF1100A0E463E
:104C60005046002190461C4613F0A9FEA94540DBA2
:104C70004FF0000B08F1FF3922224FF0FF312046A0
:104C800013F09DFE33784FFA8BF0B8F1010FE0542A
:104C90002CDD4FF0000E6FEA060C711C11F8012B91
:104CA000A356B3F1FF3F05D1431CAB42ACBF002379
:104CB0005BB2A354984219D092FBF5F005FB10208B
:104CC000012814BF01204FF0FF30204482569A4241
:104CD0000CD00CEB01029145A1EB06027BD0904574
:104CE00001DD1846DAE7BEF1000F40D1BBF1000F3D
:104CF0003AD000223B496420FDF7E4FDB8F1000FF3
:104D00005CDD013EB14606EB080119F8013F93FB5B
:104D1000F5F205FB12324945E254F6D10121002299
:104D2000314BCDE9011203930091234642466420A2
:104D3000FDF77CFD0AF1FF3316F8012FA256B145AD
:104D400003F8012FF8D1012100242848534603908D
:104D500042466420CDE901140091FDF767FD20462D
:104D60000437BD46BDE8F08F4FF0010B84E7012109
:104D700000221D4BCDE901120091039342462346C8
:104D80006420013EFDF752FD06EB08010AF1FF33F6
:104D900016F8012FA256B14203F8012FF8D10124D1
:104DA00000211248CDE90141039053466420424658
:104DB00000942146FDF73AFD2046D1E7012100206D
:104DC000094ACDE90110039223460091424664202E
:104DD000FDF72CFDB7E79045C9DD4FF0010E1846F1
:104DE0005CE700BF9C970100C09701008C97010011
:104DF0002DE9F047D2F8017006467A680D465278E0
:104E00009846012A19D9002815DD00244FF04C09D5
:104E10004D1E01E07B685A78510094FBF1F301FBD1
:104E2000134315F8010F611009FB03830134FFF7E9
:104E3000D7FCA642EED1BDE8F0870028FBDD0024B8
:104E40004FF04C0ADFF8249019F904306110002B60
:104E500006DB7A680AFB03835278285DFFF7C0FC03
:104E60000134A642F0D1BDE8F08700BFB02E00208B
:104E700010B5644684B0DCF80420084BFFF7B8FF97
:104E8000012100202368E268054CCDE90100009172
:104E900003947220FDF7CAFC04B010BD3007046013
:104EA0007497010010B5644684B0DCF80420084B08
:104EB000FFF79EFF012100202368E268054CCDE941
:104EC0000100009103947220FDF7B0FC04B010BD06
:104ED00060080460749701002DE9F047D2F8016082
:104EE0001F4672685278012A1ED900281ADD4D1E0D
:104EF00021244FF04C0805EB000901E073685A7853
:104F0000510094FBF1F301FB134315F8010F04EB7F
:104F1000D47108FB03734910FFF7B4FCA94504F1F1
:104F2000FF34EBD1BDE8F0870028FBDD0D464FF0E4
:104F30004C0A0D4C01EB000904F1220814F9013B65
:104F4000A8EB040101EBD171002B4FEA610106DBF4
:104F500072680AFB037352782878FFF793FC0135D7
:104F60004D45EBD1BDE8F0879826002010B5DCF860
:104F7000042084B0084B6446FFF7AEFF01210022F5
:104F800006482368CDE90122039000911422722083
:104F9000FDF74CFC04B010BD980604607497010046
:104FA00010B5DCF8042084B0084B6446FFF794FF8A
:104FB0000121002206482368CDE9012203900091D7
:104FC00014227220FDF732FC04B010BDC807046043
:104FD00074970100F0B403268C68012527784FF000
:104FE000060C80F8E8706778002B80F8E970A778E5
:104FF000B8BF033380F8EA70E778C3F38F0380F813
:10500000EB70A779D2B280F8EE70247A072780F887
:10501000EF4080F88E60002690F88940096844F0DF
:10502000300480F8894090F8A1406FF3041480F8B0
:10503000A1400C7880F8A94080F8985090F88B40F7
:105040006FF3000480F88B4080F88D7080F8B050CA
:1050500080F8C56080F8815080F8805080F8AEC03C
:1050600080F8AF7080F884604C7A80F89F408C7A2A
:1050700080F89E4080F89C60A0F8CA3080F8CD206F
:105080004B7BF0BC80F800318B7880F80531CB7811
:1050900080F80A310B7980F810310B7B80F8DA3018
:1050A00090F8A330CA7962F3061380F8A33090F821
:1050B000A3300A7A62F3020380F8A330CB7A80F837
:1050C000A0307047D0F8011008B54A684FF4E66385
:1050D00052784FF040505200FFF77CFFBDE8084087
:1050E000FFF7BAB9D0F8011008B54A684FF4066363
:1050F00052784FF040505200FFF76CFFBDE8084077
:10510000FFF7AAB949F6404301441144033149006D
:1051100030B5012293FBF1F10025042487B0074844
:1051200006AB43F8041D0390CDE901251146009418
:105130006420FDF77BFB07B030BD00BF6497010022
:105140002DE9F04F4FF04C09984609FB03F909F19E
:10515000070383B023F0070300AFADEB030D7860C6
:105160003A600C4668464A46002113F028FCB8F124
:10517000000FEA4671DD6B461A200DEB09015A78E3
:10518000187002F0EC0242F002025A704C3399425D
:10519000F5D13A6814F0FF011369566964D053EAF7
:1051A00006020CBF4FF0010E4FF0000E00224FF030
:1051B000010C05E0BEF1000F10D101328A421FD070
:1051C000C2F1200506FA05F523FA02F0A2F1200447
:1051D000284326FA04F42043C007EBD54FF04C0BCC
:1051E0007868234C805C24561F280CFA00F50BFBD2
:1051F00004A425DC6069013205438A426561DFD180
:105200003B68B8F1000F5B6858780FDD00234C2530
:105210005524022807D105FB03A2D17C547421F048
:1052200001019474D17401339845F2D14A46514634
:10523000386B13F0B9FB386B0C37BD46BDE8F08F07
:10524000257E2038AB460CFA00F0C5F30105054376
:1052500065F3010B84F818B0AFE73A6814F0FF016A
:10526000136956699BD1E1E73B685B685878CDE7E5
:10527000B02E00202DE9F04F85B01546D0F8018002
:105280000A7DD8F8044002AF6678086803FB06F68A
:1052900003EBC30A1146334600954246FFF750FF21
:1052A0000AF10703D8F8044023F00703C7F804D035
:1052B000ADEB030D94F805B00DF1080948465246D0
:1052C0000021647813F07BFBBBF1020F00F0C58076
:1052D000BBF1040F00F0B180BBF1010F00F083803F
:1052E00052460021484613F06AFB002E40F3C58069
:1052F0002C464FF0000C4A460023E11812F8010B2F
:105300000133092B0872F8D10CF1010C664509F143
:10531000090904F14C04EEDC4FF0000E2846F1467A
:10532000D8F80480D7F804D098F8064004F01F0499
:1053300004F0030C4FEA8C1CA408002101F11003B7
:1053400000EB430393F806A0DA790AF03F0A22F053
:10535000070201314AEA0C0A2243112983F806A008
:10536000DA71EBD190F84A300EF1010E23F01F03F1
:10537000764580F8489080F8499080F84A3000F1EE
:105380004C00DADC002398F8049098F803A098F811
:1053900002B0504649465A469846012409EB0A0E87
:1053A0000BEB090CAEF10A0E0CF1010C5FFA8EFE4C
:1053B0005FFA8CFC01339E4285F802A02C7185F8BF
:1053C00003C085F8059085F806B085F807E085F8F4
:1053D0001980AC7605F14C05ECDCFFF793FE0C3739
:1053E000BD46BDE8F08F002E47DDCB464FF0000EE6
:1053F000DFF8A0A05946DFF8A0C00023022C03D09C
:10540000012C03D1012B01DC9E4506D003EBC30226
:1054100008781CF8022002430A700133042BEDD1F6
:105420000CF1010CD44501F10101E6D10EF1010EA0
:1054300076450BF1090BDDD15AE7002E1DDD4B46F9
:10544000AA2106EBC600484403F1090203F8011B38
:105450009342FBD18342F7D14AE7002E0DDD4B4644
:10546000AA2106EBC600484403F1090203F8011B18
:105470009342FBD18342F7D13AE7D8F80430D7F80A
:1054800004D0D87819799A78FFF73CFE0C37BD46DE
:10549000BDE8F08F69270020602700202DE9F04744
:1054A00092B0DFF8F4C002AFDFF8F0A007F12C04EF
:1054B00007F11C0907F1080605468846BA619AE813
:1054C0000F0089E80F00214607F16003C9E9026C6B
:1054D0004846FB63FAF7D4FE9AE80F00DFF8C0C035
:1054E00084E80F00C4E9026C204607F13C01FAF79A
:1054F000C7FE0520FFF70EF8034600210220D3F86F
:105500000160FB60FEF74EFDAA7EDFF898C0D31D58
:10551000BCF800C003F4FC73ADEB030D07F14001D0
:1055200021F83CCD02AB386102207A61BB60FEF706
:10553000A1FFBB699847FFF77DF8736844F0010449
:105540005878800106F0D8FCB26849F0010651890C
:10555000BB68CDE900467A6901F042FA79692868AA
:105560008B000A3323F00703ADEB030D02ADD7E93F
:105570000343BA68CDE900342B46FFF7C9FAB8F106
:10558000000F05D07A6929464046920013F00CFAC4
:105590004037BD46BDE8F08725490000A08B0100DB
:1055A000714E0000B08B01002DE9F04792B0DFF89A
:1055B000F0C002AFDFF8ECA007F12C0407F11C09E2
:1055C00007F1080605468846BA619AE80F0089E89F
:1055D0000F00214607F16003C9E9026C4846FB63EE
:1055E000FAF74EFE9AE80F00DFF8BCC084E80F001F
:1055F000C4E9026C204607F13C01FAF741FE09209C
:10560000FEF788FF034600210420D3F80160FB6009
:10561000FEF7C8FC0923AA7E07F1400101F83C3DD2
:10562000D31D03F4FC73ADEB030D02AB3861012015
:105630007A61BB60FEF71EFFBB699847FEF7FAFF71
:10564000736844F001045878800106F055FCB26894
:1056500049F001065189BB68CDE900467A6901F03D
:10566000BFF9796928688B000A3323F00703ADEB93
:10567000030D02ADD7E90343BA68CDE900342B46E8
:10568000FFF746FAB8F1000F05D07A69294640467F
:10569000920013F089F94037BD46BDE8F08700BF9E
:1056A00059490000A08B0100A54E0000F8B59B00F1
:1056B00003F10A0424F0070400AF002AADEB040D47
:1056C000EC460CDDBC69ACF10405013C224414F845
:1056D000016F51F82660944245F8046FF7D11A46DD
:1056E000614613F061F9BD46F8BD00BF70B582B0E8
:1056F0000AF09AFA012104460220FEF753FC002129
:1057000006460220FEF74EFC0546A27E3146920078
:1057100013F04AF92168A37E227D2846009129468C
:10572000FFF7C4FF02B070BD38B50AF07DFA012161
:1057300005460220FEF736FC044600210220FEF753
:1057400031FCAA7E2146BDE83840920013F02CB906
:1057500070B582B00AF068FA012104460420FEF711
:1057600021FC002106460420FEF71CFC0546A27E13
:105770003146920013F018F92168A37E227D284655
:1057800000912946FFF792FF02B070BD38B50AF0CC
:105790004BFA012105460420FEF704FC04460021D3
:1057A0000420FEF7FFFBAA7E2146BDE838409200A8
:1057B00013F0FAB8D0F8011008B54A684FF4D36373
:1057C00052784FF040505200FFF704FCBDE808400B
:1057D000FEF742BED0F8011008B54A684FF4F963ED
:1057E00052784FF040505200FFF7F4FBBDE80840FC
:1057F000FEF732BE2DE9F04F4C261C4606FB03F6A1
:10580000F31D85B023F0070300AFADEB030DF86087
:10581000BA600D4668463246002113F0D0F8002CDD
:10582000E8467BDD6B4600200DEB06015A781870C8
:1058300002F0EC0242F012025A704C339942F5D158
:10584000BB68002DD3F810E0D3F814C06EDD5EEA1B
:105850000C030CBF4FF0010A4FF0000A2346002250
:1058600054464FF001097E609A4603E084B9013244
:10587000954222D0C2F120000CFA00F02EFA02F379
:10588000A2F1200103432CFA01F10B43DB07EDD514
:105890004C26FB6827499B5CC3F12100C9561F2891
:1058A00009FA00FB06FB01812ADC4B69013243EA5D
:1058B0000B0B9542C1F814B0DCD15446BB68002CE8
:1058C0005B687E68587811DD00234FF04C0C6FF058
:1058D0005505022807D10CFB0382D17C557421F0B9
:1058E00001019574D17401339C42F2D13246414694
:1058F000B86B13F059F8B86B1437BD46BDE8F08F9C
:10590000087EC3F10103834609FA03F3C0F30100E3
:10591000184360F3010B81F818B0A8E7BB68002DAD
:10592000D3F810E0D3F814C091DCDFE7BB685B6804
:105930005878C9E7982600202DE9F04F87B01C461B
:1059400094460B46D0F8016002AFFA607268497D58
:105950005578586804FB05F5CDF800C02B46324653
:10596000FFF748FF04EBC402D31D746823F007035C
:10597000C7F808D0ADEB030D94F805900DF10808B9
:1059800040460021647813F01AF8B9F1020F00F0D4
:10599000CD80B9F1040F00F0B980B9F1010F7ED0CC
:1059A000002D40F3D3804FF0000CFC6842460023EA
:1059B000E11812F8010B0133092B0872F8D10CF130
:1059C000010C654508F1090804F14C04EEDC4FF0C8
:1059D000000ED7F80CC0F1466046D6F80480D7F820
:1059E00008D098F8064004F01F0404F00306B6013E
:1059F000A408002101F1100300EB430393F806A073
:105A0000DA790AF03F0A22F0070201314AEA060A6F
:105A10002243112983F806A0DA71EBD190F84A30BD
:105A20000EF1010E23F01F03754580F8489080F8B1
:105A3000499080F84A3000F14C00DADC002398F8F5
:105A4000049098F803A098F802B0504649465A4688
:105A50009846012409EB0A0E0BEB0906AEF10A0E7B
:105A600001365FFA8EFEF6B201339D428CF802A039
:105A70008CF804408CF803608CF805908CF806B024
:105A80008CF807E08CF819808CF81A400CF14C0C5B
:105A9000EADCFFF737FB1437BD46BDE8F08F002D79
:105AA00054DDAB1C7D60C3464FF0020EA4461D467C
:105AB000DFF8B49058462B4CAEF1020A0023BCF13B
:105AC000020F20D0BCF1010F07D1012B05DD022B05
:105AD0000CBF00220122524505D003EBC30201781E
:105AE000A25C0A4302700133042BE8D101344C4517
:105AF00000F10100E2D10EF1010EAE450BF1090BF0
:105B0000D8D17D684FE79E45E7D1ECE7002D1DDD3C
:105B10004346AA2105EBC500404403F1090203F8FE
:105B2000011B9342FBD18342F7D13CE7002D0DDDF1
:105B30004346552105EBC500404403F1090203F833
:105B4000011B9342FBD18342F7D12CE77368D7F84E
:105B500008D0D87819799A78FFF7D4FA1437BD4667
:105B6000BDE8F08F602700206927002089B182B14D
:105B700038B505461446084602232946064AFFF76B
:105B800079FB204629460223044AFFF7D5FE01206F
:105B900038BD0020704700BF3007046098060460DD
:105BA00089B182B138B50546144608460223294614
:105BB000064AFFF75FFB204629460223044AFFF707
:105BC000BBFE012038BD0020704700BF60080460A4
:105BD000C80704602DE9F04F91B0DFF8F8A002AFDC
:105BE000DFF8F4C007F1240407F114053E1D8046D8
:105BF00089463A619AE80F0085E80F00C5E9026C12
:105C00002846214607F160037B63FAF739FB9AE8DF
:105C10000F00DFF8C8C084E80F00C4E9026C20461A
:105C200007F13401FAF72CFB0620FEF773FC03465C
:105C300000210320D3F801B0BB60FEF7B3F998F858
:105C400019A0234A0AF10703128803F4FC73ADEB91
:105C5000030D07F1380121F8382D02ABF86002205E
:105C60007B60FEF707FCDBF8043045F0010558784F
:105C700044F00104800106F03FF9DBF808207B685E
:105C800051894FEA8A06CDE90045524600F0A8FE48
:105C900006F10A0303F4FF63ADEB030D02ACD7E991
:105CA000025398F81510D8F804007A68CDE9003549
:105CB0002346FEF79FFEB9F1000F04D0324621467D
:105CC000484612F071FE3C37BD46BDE8F08F00BF7C
:105CD000B08B0100A08B01008D4900006D4F0000CA
:105CE0002DE9F04F91B0DFF8F0A002AFDFF8ECC083
:105CF00007F1240407F114053E1D804689463A61E8
:105D00009AE80F0085E80F00C5E9026C2846214695
:105D100007F160037B63FAF7B3FA9AE80F00DFF844
:105D2000C0C084E80F00C4E9026C204607F13401CA
:105D3000FAF7A6FA0A20FEF7EDFB0346002105203C
:105D4000D3F801B0BB60FEF72DF90A2398F819A02B
:105D500007F1380101F8383D0AF1070303F4FC7339
:105D6000ADEB030D02ABF86001207B60FEF782FB18
:105D7000DBF8043045F00105587844F00104800157
:105D800006F0BAF8DBF808207B6851894FEA8A06EA
:105D9000CDE90045524600F023FE06F10A0303F464
:105DA000FF63ADEB030D02ACD7E9025398F8151071
:105DB000D8F804007A68CDE900352346FEF71AFECC
:105DC000B9F1000F04D032462146484612F0ECFDEE
:105DD0003C37BD46BDE8F08FA08B0100C1490000F3
:105DE000A14F000070B582B009F01EFF01210446EA
:105DF0000320FEF7D7F8002106460320FEF7D2F86D
:105E00000546627E3146920012F0CEFD6168637EE7
:105E1000627D284600912946FFF748FC02B070BD1C
:105E200038B509F001FF012105460320FEF7BAF855
:105E3000044600210320FEF7B5F86A7E2146BDE83E
:105E40003840920012F0B0BD70B582B009F0ECFE9F
:105E5000012104460520FEF7A5F80021064605208D
:105E6000FEF7A0F80546627E3146920012F09CFDD6
:105E70006168637E627D284600912946FFF716FC23
:105E800002B070BD38B509F0CFFE4FF04053054663
:105E900093F8414101210220FEF784F8E4B2AA7E82
:105EA0000349240421449200BDE8384012F07CBD2F
:105EB0006808016038B509F0B7FE4FF04053054659
:105EC00093F841410121E4B20320FEF76BF821046D
:105ED0006A7E01F1C04101F584319200BDE838408D
:105EE00012F062BD38B509F09FFE4FF040530546F1
:105EF00093F8414101210420FEF754F8E4B2AA7E50
:105F00000349240421449200BDE8384012F04CBDFE
:105F10006808016010B509F087FE4FF0405393F810
:105F200041410121E4B20520FEF73CF8210401F1D2
:105F3000C04101F584315022BDE8104012F034BD5B
:105F400038B509F071FE012105460520FEF72AF853
:105F5000044600210520FEF725F86A7E2146BDE8AB
:105F60003840920012F020BD08B5FEF763FBBDE893
:105F7000084000210220FEF715B800BF08B5FEF763
:105F800059FBBDE8084000210420FEF70BB800BF14
:105F900008B5FEF74FFBBDE8084000210320FEF7DF
:105FA00001B800BF08B5FEF745FBBDE80840002179
:105FB0000520FDF7F7BF00BF704700BFF0B50546ED
:105FC000B3B068B3421E022A01D933B0F0BD03AFAB
:105FD0001C46BC4603F1400E664620686168A26814
:105FE000E368103474450CF1100C0FC6F4D15E2632
:105FF000389B13AC186859689A68DB680FC4389BE3
:10600000186959699A693B4607C4389A1A49908BAE
:106010002A4620800C68009600210120A047D4E782
:106020000E46144603AF0146BC22384612F0C7FCA8
:1060300031683846802212F0B7FC246823AE04F1A0
:10604000300C354620686168A268E3681034644506
:1060500006F110060FC5F4D120686168A268BC245F
:1060600007C60022044800943B46046811460120FC
:10607000A04733B0F0BD00BFE0CA0100F8B500236F
:10608000114C1946236063603C22104812F097FCC3
:1060900000F0EAF94FF480620D4B0E490E4E0F4CA2
:1060A0009B68886030689A606368851C9847A3681D
:1060B0000746984739460246284612F075FC236980
:1060C00034689847E080F8BD60250020A0270020B4
:1060D000800600208419002028060020E0CA010064
:1060E000F0B51E4C85B02678174686421946DDE984
:1060F0000A230546DDF830C018D0A378AB4201D0A2
:1061000005B0F0BDE378002BFAD0CDB94FF4F060C4
:1061100001210A902A460846114B1B680393039CF1
:10612000104BA44605B0BDE8F04060476678002EED
:10613000E3D0CDF800C010321031FFF73FFFDCE7AD
:106140006B1E022BDCD84FF470700121044C0A90B6
:1061500024683B462A4608460394E2E7602500206F
:10616000E0CA0100980004602DE9F04F5A4C85B058
:106170000E9D64790295DDE90F56019614B905B0BC
:10618000BDE8F08F914600240090A0228846534835
:1061900000219A46DFF850B112F011FCA646504A91
:1061A0004E4805F1FF3CCDF80C904FE0002B0CBFA2
:1061B000012302234FF487664370009B047033F978
:1061C0001430029D06FB03F38BFB03761E44DB17A2
:1061D000C3EBE62340F6241655F82450438038F9E3
:1061E0001430C5F3072706FB03F38BFB03961E440D
:1061F000DB17C3EBE6238380039B33F81460EBB219
:10620000FF1AC5F30743C3EB1565AF42C6804FF0D5
:106210004D034BDD03FB07F7BF1107814581019B50
:106220003AF814501B5D85818373009B0EF1010EBB
:1062300033F91430138038F91430538001340A2CA8
:10624000117100F1100002F1060235D01CF8011F97
:1062500013790029AAD1002BF0D04FF48766B2F948
:106260000050B2F9023006FB05F540F6241606FB95
:1062700003F38BFB05678BFB03964FF003091E446A
:10628000DB17C3EBE623019E047080F80190365DB6
:106290002F44ED17C5EBE725C18001814181818144
:1062A0000EF1010E458083808673C7E703FB05F579
:1062B000AB1103814781B2E70A4B03221B6802211D
:1062C0000093009C0120A446044BCDF838E005B0B3
:1062D000BDE8F04F604700BF60250020041000209B
:1062E000A0270020E0CA01008100088010B584B01A
:1062F00003F0C2FF0E4A4379117899420CD04379DA
:106300000C49DBB213700A6803923BB90221009377
:1063100008461A46039CA04704B010BD0023022182
:10632000009308460122039CA04704B010BD00BFA3
:10633000F80F0020E0CA010010B582B003F09CFF06
:10634000437F43B10023054C43771A460093194617
:1063500024680220A04702B010BD00BFE0CA0100BF
:1063600030B583B003F088FF084CC37F22789A428F
:106370000AD00023C07F0649C0B202460D682070D3
:10638000009306210220A84703B030BDFA0F002079
:10639000E0CA010030B583B091B1838B028B1949FB
:1063A0001A44782A0B781FDDB0F924001BB30024AF
:1063B000154A1460013BDBB202200B70106004E050
:1063C0000846114A0F4B11601970104C2378834214
:1063D00008D000230E49024600930D682070072163
:1063E0000220A84703B030BD0020074A1060002BF0
:1063F000E0D11068E9E70123034AA0281360F8DD23
:106400002323D9E700100020FC0F0020F90F002003
:10641000E0CA0100002300B583B0019300F024F826
:106420000378054A8DF80430019BC3F30013137001
:1064300003B05DF804FB00BFFB0F002010B582B075
:10644000FFF77AFFFFF752FFFFF78AFFFFF7E2FF40
:106450000023044900930C681A4604210120A04738
:1064600002B010BDE0CA010000487047A41000202F
:106470004FF48060704700BFF9F704BF12F094BA80
:1064800012F09DBA10B40124034B00221C70034982
:10649000642010BCFCF716BA5D230020A098010010
:1064A00070B505460E46144688B010490022642097
:1064B0000794CDE90556FCF705FA012100200422D6
:1064C0000B4BCDE9011000920393032205AB64202E
:1064D000FCF7ACF9003418BF0124064B03EB45026E
:1064E00003F81560547008B070BD00BF44980100F7
:1064F000789801006025002038B5002204460A493A
:106500006420FCF7DFF9094A40F2F121134623F831
:10651000021B25686468C2F802505C601046BDE842
:1065200038400C2103F0DCBE24980100BC2D002073
:1065300000487047BC9801001EF0040F0CBFEFF339
:106540000880EFF309808169004A1047B502010015
:10655000684620F007018D4601B401BC85467047AE
:1065600072B61EF0040F0CBFEFF30880EFF3098042
:10657000004A1047E966000072B61EF0040F0CBF17
:10658000EFF30880EFF30980004A1047ED66000042
:1065900072B61EF0040F0CBFEFF30880EFF3098012
:1065A000004A1047F166000072B61EF0040F0CBFDF
:1065B000EFF30880EFF30980004A1047F56600000A
:1065C000684620F007018D4601B401BC854670473E
:1065D000684620F007018D4601B401BC854670472E
:1065E000684620F007018D4601B401BC854670471E
:1065F000684620F007018D4601B401BC854670470E
:10660000684620F007018D4619B507232B4CB020B2
:10661000237309F005FE0021294A2A4BA1709A42F2
:106620000CD2111D03335B1A23F0030326480B44DD
:1066300050F8041B42F8041B9A42F9D1234A244B18
:106640009A420CD2111D03335B1A23F00303214835
:106650000B4450F8041B42F8041B9A42F9D11E4A1D
:106660001E4B9A420AD20020111D03335B1A23F0FD
:1066700003030B4442F8040B9342FBD1EFF308826F
:10668000174B9A4205D94FF0CD3143F8041B9A427B
:10669000FBD84FF6FF72094B1A8709F075FC09F019
:1066A0007FFC1049002009F021FC044600F04EF860
:1066B000844200D0FEE70BF065F9FBE700001050C4
:1066C00000560020805600208000000000000020BE
:1066D000400F0020B0CB0100400F002020250020FB
:1066E000F82E0020FCFB0100704700BF704700BF80
:1066F000704700BF704700BF014B93F821007047FF
:10670000C0FB0100014B187E704700BFC0FB0100B9
:10671000014B587E704700BFC0FB0100014B987EC3
:10672000704700BFC0FB0100014BD87E704700BF1F
:10673000C0FB0100014B986A704700BFC0FB01001D
:10674000014BD86A704700BFC0FB0100014B1868BD
:10675000704700BFFCFB01002DE9F04F4FEA820BB0
:1067600083B00BF10A0525F0070500AFADEB050D71
:106770006D463B604B68D1F80080064614468A4659
:106780007B60C0475A462846002112F018F90122C2
:1067900002FA06FB1BF1FF3B17D37B689847814643
:1067A000BBF1000F00D0C047002CF3DDAC46002148
:1067B0005CF8043B59F8042B013113448C424CF82B
:1067C000043CF5D11BF1FF3BE7D2002C09DD294643
:1067D000002251F8043B01323341944241F8043C19
:1067E000F7D1DAF808302946204698473A68DAF8AF
:1067F0000C302946204698470C37BD46BDE8F08F3F
:1068000001322DE9F04191FBF2F404FB121282B047
:10681000DDE90A67DDE90C4512B102B0BDE8F0819F
:106820002022804600921846DDE90812012305F077
:10683000C9FAB8F1000FF0DD04EB48020FFA87FE49
:106840000FFA86FC08E0634655F8041B944203FBEC
:10685000101345F8043CE0D034F9023BB342F2DCBB
:10686000BB42B8BF7346EFE72DE9F04F1446984698
:10687000D31D85B023F0070300AFADEB030D9500EA
:1068800079608346002168463A6012F098F805F175
:106890000A0323F0070341462046EA46ADEB030D09
:1068A000BB6B9847FB6B9847E94601462A4648462A
:1068B00012F07AF8002C40F38880434608EB04017C
:1068C00013F8012B01328B4203F8012CF8D1414619
:1068D0003868BB6B9847FB6B9847043D04384D44C0
:1068E000A9F10403514642464FF0FF0C4FF0010E50
:1068F00008E0AB4281F800E01C6001F1010102F107
:10690000010211D050F8044F53F8046FA642F0DB97
:106910001478AB4204F1FF3481F800C0147001F127
:10692000010102F10102EDD13B685E1E56440AF1FD
:10693000FF334FF0000A1D46C4461C46012209E001
:10694000786888420FDB00228CF80010B4420CF10A
:10695000010C0ED014F9011F0029F7D09CF800009B
:1069600001448B45ECDDB44284F800A00CF1010C2D
:10697000F0D182BBC7E9023241463868BB6B984709
:10698000FB6B9847D7E9023284469E4605E049F8FA
:106990002200AC4202F1010215D015F9011F0029B5
:1069A000F7D05CF8220059F822308342EFDB18F868
:1069B0000200AC42A0EB010108F8021085F800A02B
:1069C00002F10102E9D17346B5E7BB6B4146386875
:1069D0009847FB6B98471437BD46BDE8F08F00BF62
:1069E0002DE9F04F012683B00138B2F100080D46C1
:1069F00000AF9B4606FA00F640F39880013B03EB9C
:106A00000800F1B203F8011F8342FBD1761000F0B9
:106A10009D804FEA880AAAF10409C7F804A07C6B9C
:106A2000D7F830A059464046D047A047B8F1000FEC
:106A300013DD5B465FFA86FC011F00EB090E51F87F
:106A4000040F1A78A842A2EB0C00D6BF624418705B
:106A50001A70714503F10103F1D17610E2D1594664
:106A600040463B6BD7F804A098477B6B98470AF1E8
:106A70000A0323F00703ADEB030DB8F1000F024644
:106A80006C465CDD043C161F20463146AAF1040A20
:106A900002EB0A0C51F8043F5B1B8C4540F8043FA5
:106AA000F8D1D9465B46304602EB0A0E50F804CFC7
:106AB0001978AC4501F1FF3CD6BF013183F800C025
:106AC0001970704503F10103F0D1594640463B6B04
:106AD0007A6098477B6B98477A68924456F8043FEF
:106AE00054F8042F5B1B002A83EAE371A1EBE371E6
:106AF000B8BF52428A420ADA99F80020002B02F10C
:106B0000FF31D6BF013289F8001089F80020B24564
:106B1000236009F10109E1D1594640463B6B984792
:106B20007B6B98470C37BD46BDE8F08F76107FF43D
:106B300070AF3B6B5946404698477B6B98473B6B21
:106B40005946404698477B6B9847E5E7594640468B
:106B50003B6B98477B6B98474FEA880A0AF10A0318
:106B600023F00703ADEB030D02466C468AE700BF36
:106B70002DE9F04F83B00D9EDDE90F9C002E40DD26
:106B8000DFF88480DF021D0388FB073B88FB0538A4
:106B90000E9BFF17ED17013B5200C5EB6815002453
:106BA00000EB01084FF47A7E41F2301AA7EB6B1725
:106BB0001E44411A01921AE008FB00FB59F8240018
:106BC000019A381890FBF2F00EFB00F090FBF5F004
:106BD0000EFB0BFB0AFB00F00C9A9E4202FB10B06E
:106BE00090FBF1F04CF8240004F1010409D013F8F3
:106BF000010F0028E0D19E424CF8240004F101046A
:106C0000F5D103B0BDE8F08F1F85EB512DE9F04FB2
:106C100091460646850099B02A46DDE92448084693
:106C20008A460021139311F0CAFE2A4600214846E5
:106C300011F0C5FE72000021229811F0C0FE32460C
:106C40000021239811F0BBFE2A464046002111F096
:106C5000B6FE002E40F3A480229B221F0693239BA6
:106C6000CDE9079A0B9300230293279B1092C3EB65
:106C7000C3732A445B0012920F93109B53F8041FB6
:106C800010934FEA116BC1F307435B450D9100F27E
:106C90002181002201230392279A29989A400BFB15
:106CA00002020492DDE927200BFB02020992029AFC
:106CB00093400C93CBB20193C1F307230E930E992B
:106CC000019B994232DB099B4FF0010E5E18DC46B6
:106CD00005E0900667D4019B01398B4225DC16F84C
:106CE0000129029B9A42F4D1049B089833F91120A0
:106CF000039C036802FB024401FB02330394079CDC
:106D000003602368069D0CFB02332888236010442F
:106D100028800B9803789342DDDAFF2AA8BFFF2270
:106D2000019B01398B420270D9DDE346049A0F9929
:106D30000D9B0A4404922799099A0BF1FF3BC3F378
:106D40000743521A5B450992B9DD069BB3F900204F
:106D500092B108980399036891FBF2F15B0293FBEF
:106D6000F2F30360079803685B0293FBF2F3029A65
:106D70000360139B23F81210029B109A01330293B5
:106D8000069B02330693089B04330893079B043346
:106D900007930B9B01330B93129B93427FF46DAFD0
:106DA00019B0BDE8F08F00234FF601701C464B4D23
:106DB00018AF95F800B047F8040D494D289816957E
:106DC000059302F00F0500EB010A0A9245FA03F061
:106DD000C20719D516AAD056279A604402FB00A014
:106DE00013F9079010F809900EFA09F0D94540EA16
:106DF000040009D2A04207D0059A044618A81044FE
:106E0000013200F80C9C05920133042BDED10C9B5F
:106E10000A9A23423FF45FAF049B33F911B0D306C3
:106E200016D49DF808307370089A039813680BFB0A
:106E30000B0001FB0B330390079813600368069C5B
:106E40000CFB0B33228803609344A4F800B042E7A4
:106E50004FF00009059B0DF153005A1E914500EBC0
:106E600003070DF1540A1846CDF844B01CDA09F1B5
:106E70000109484514DD54469AF800B00A9214F806
:106E8000013F9B452ABF1D465D465B4658F82520BD
:106E90000EFA03F31343A74248F82530EFD10A9ABC
:106EA00091450AF1010AE2DB059BDDF844B0032BB2
:106EB00009D0042B04D0022BB6D14FEA6B0BB3E7F9
:106EC0004FEAAB0BB0E74AF6AB2303FB0BFB4FEAF1
:106ED0006B4BA9E70023039337E700BFD498010069
:106EE000000001FF0288014B1A807047A4140020A3
:106EF0002DE9F0414FF4614C4EF2B057184C069E0C
:106F000094F8008094F801E006EB410611F1FF319E
:106F100023D336F9024D002CF8D032F9114033F961
:106F2000115068B905F5807504F58074B8F1000F4B
:106F300001D0C5F5F055BEF1000F01D0C4F5804475
:106F40000CFB05F507FB04F42D14241422F8115052
:106F500023F8114011F1FF31DBD2BDE8F08100BF11
:106F6000A41400202DE9F04F40F6FF7CDDE90976FE
:106F700040F6FE7849F64E3944F2507EACEB060BF3
:106F80000344A8EB060AACEB070C10F1FF3020D34A
:106F900013F8014D002CF8D031F9105032F910409F
:106FA00009FB05F50EFB04F42D14BD424FEA244401
:106FB00013DDAC4501DCA8EB0705B4420BDDA345AE
:106FC000D8BF544621F8105022F8104010F1FF307D
:106FD000DED2BDE8F08F3446F4E73D46EDE700BF72
:106FE0000288014B1A807047A8140020002318491A
:106FF000184A70B41848194E194D1A4CC1E900339B
:107000000B81C2E9003318491381184AC6E90033DD
:10701000C6E902333361C5E90033154EC5E90233D1
:107020002B61C4E90033C4E902332361C0E90033B2
:10703000C0E902330361C1E90033C1E902330B61E6
:10704000C2E90033C2E902331361337070BC704788
:10705000F018002040180020741800209C18002010
:10706000C4180020881800204C1800206018002048
:10707000EC1800202DE9F04F8BB09DF854607A4C4D
:10708000CDE9026027786578784C01932478029BDB
:1070900092469C4238BF754A0E468DF824708DF892
:1070A000255038BF1370149D092405F0CBF8039BBD
:1070B0000490DFF8D091DFF8D081DFF8D0B125441B
:1070C000123603F1120739E018F804300AAA0A440C
:1070D00012F804CC0133DBB265489C4508F8043053
:1070E0004FEA440230F914003BF914E0009745D20E
:1070F0000023297808F8043009F804105D4B9852F1
:107100005D4B5B4823F802E0009BB3F900308352EB
:10711000B6F9003059482BF802303AF9143083524E
:10712000019B574833F914308352013C631C05F826
:107130000119A7F10207A6F102063CD006F078F883
:1071400058B13AF91430002B07DDB6F90030B3F529
:10715000007FBCBF01238DF8243019F804102B7870
:107160008B42B1D10023620008F80430404B3BF958
:1071700002E0985E039B13440093BFE7002BBDD051
:107180009DF858302BB92B781BB9384B1B78012B45
:1071900018D038803BF902303380384B01989B5E21
:1071A0002AF81430364B9B5E20F8143018F804305F
:1071B000002BBAD1DAE7029B0BB92C4A13700BB043
:1071C000BDE8F08F049B132BE3DC2A4B9B5E0093FE
:1071D000294B33F902C0009B13B9BCF1000FD8D082
:1071E000009BC31A002B0693B8BF5B420593AEEB1E
:1071F0000C0300930793059B772B2EDD41F6CC0CF7
:10720000A0F1C9039BB26345C3D86FF4C87343F2BE
:107210004A6C73449BB26345BBD841F65C2C069B19
:1072200003EB430303EBD37300EB63030093013BD6
:107230006345AED8079B03EB430C0CEBDC7C0EEBF9
:107240006C0E43F66A1C0EF1FF336345A1D8BDF8FE
:1072500000303B80A6F800E09FE7009B002BB8BF02
:107260005B42772B95DDC9E7A8140020EC180020BD
:107270009C1800204C18002060180020881800205E
:1072800074180020F018002040180020C4180020B6
:10729000F0B40C781A4D14B305EB8406B6F84460CC
:1072A00086421CDD0027661EF6B21F700E702F6C22
:1072B000013FA74206DD05EB8406B6F84C60B042FC
:1072C00017DC0E78B44218BF14701A780132D2B2AB
:1072D0001A7069698A4200DD1970F0BC70472E6C23
:1072E000013EA642F1DD05EB8406B6F84C60B042E3
:1072F000E7DD0020661CF6B218700E70E2E700BFF2
:107300003005002001467422014811F04DBB00BF3A
:107310003005002000224FF480710848084B007DA2
:107320001A61987583F83200DA759A61DA6283F827
:1073300033205A6399821986704700BF30050020B8
:1073400024260020F0B49DF8104024B33B4F3C4D60
:10735000012C18BF00272C78012C21D0002C4BD1F8
:10736000D7F800C0BCF1000F64DDBE88B04247DB37
:1073700023463A4605E016892346864202F1040276
:107380003EDC5C1C6445F6D1DAB20A7007EB83037D
:10739000D888F0BC70472A4D2A4F2C78012CDDD1BB
:1073A000686991F800C0002816784FF0000408DDE5
:1073B00005F1140202EB800052F8041F82420C44D3
:1073C000FAD11878A0B300211F4A02EB800052F8CE
:1073D000043F90421944FAD107EB8603B44507EB0A
:1073E0008C07D888FB881BD91B1A01FB03F191FB82
:1073F000F4F1F0BC084470474FF47A70F0BC704769
:107400000A78A242134608DD4FF0640C6D780CFB3D
:1074100000F006FB05F6B042B7DCE2B22346B4E763
:10742000C31A01FB03F191FBF4F1F0BC401A704761
:107430000146D1E722462346A7E700BF8C0500207E
:107440003005002074050020440500202DE9F04F90
:10745000C600351AAD00904C05F1180787B004EB53
:107460000709002900F0FE8004EB050EDEF810107D
:107470000A2940F3E480D3F800C0CDE90332331A7F
:107480009B00109A04EB03088346E0581168D8F873
:107490000430ACEB0000C91A0028B8BF40420029F4
:1074A000B8BF494204F0A4FC4FF6FF738342A8BF63
:1074B000034698F8172005F1150A29F8123098F8B4
:1074C000173005900133DBB2012B88BF002388F809
:1074D0001730DFF8C881B9F80210E35B98F8002094
:1074E0000B4405F114095B101635012A0293A144DF
:1074F000A244254400F0C88000222B460092494651
:1075000052460298FFF71EFFA6EB0B0304EB830322
:107510001A6998F80C3007469A42C0F287800A220E
:10752000A6EB0B0304EB83031A61012052462B46A2
:10753000009049460298FFF705FFA6EB0B0304EB0A
:1075400083031A6998F80C3082469A4206DAD8F812
:107550001030059A9342C8BFD8F808A0049BA6EB48
:107560000B0203F1010997FBF9F7039B92001B68DB
:10757000A11803FB07FC8868A358C7F57A75034474
:1075800005FB03C3DFF818C14FEAE37E8CFB03035E
:107590000398CEEBA3130360109BC8681B6803FB22
:1075A00007F74B68184405FB00778CFB075E109DBE
:1075B000FF17C7EBAE172F6098F80230029DAB4261
:1075C00010DB0023C1E90233039BA6EB0B061B680B
:1075D000B600A351109B02981B682644736007B045
:1075E000BDE8F08F9AFBF9F98B68A058C9F57A7A53
:1075F000039A03FB0AF31268121A09FB02338CFB8D
:107600000302DB17C3EBA213C8688B60109B00FB5F
:107610000AF01B684A689B1A09FB03098CFB093CAA
:107620004FEAE979C9EBAC13CB60CDE7D8F810305D
:10763000059A93427FF773AFD8F8047075E701316C
:10764000CEF810100129D3F800C07FF416AF4FF028
:107650000008109944F805C00968CEF80C80CEE9FE
:10766000011808E74FF480700C4A05F110035269C5
:107670000291E1502344988002982544E975AA7547
:10768000E15107B0BDE8F08F2B46524649460298BB
:10769000FFF7FEFD30E700BF242600203005002064
:1076A000D34D6210F8B505461A4C0146B02220466B
:1076B00011F07AF92E1D04F15C0C0FCEACE80F002E
:1076C0000FCEACE80F0096E8030005F1300704F197
:1076D00088068CE803000FCF0FC60FCF0FC697E8C0
:1076E000030086E8030005F18807261D0FCF0FC6AB
:1076F0000FCF0FC697E803005C35303486E80300EF
:107700000FCD0FC40FCD0FC495E8030084E803002C
:10771000F8BD00BFAC1400202DE9F84F9DF828708B
:10772000012F34D004460E469246DFF80CB103EB2D
:1077300040050BF130090BF1040814F1FF3426D396
:1077400035F9023D002BF8D056F82430DBF85820EC
:1077500093423ADA022F5DD17F209B1A00FB03F39C
:1077600002EBA31246F824205AF82410DBF800306C
:1077700099420EDA022F44D17F20C91A00FB01F191
:1077800003EBA1134AF8243014F1FF34D8D2BDE83A
:10779000F88FDBF82C30C1F5E0519942CDDA022F99
:1077A00043D008B2494604F079FB5AF82410DBF8BC
:1077B0002C30C1F5E051C91A00FB01F103EBA11314
:1077C000C3F5E0534AF82430B7E7DBF88420C3F56B
:1077D00078539342C8DA022F25D018B2144904F026
:1077E0005DFB56F82430DBF88420C3F578539B1AF0
:1077F00000FB03F302EBA312C2F5785246F82420F3
:10780000B2E708B2414604F049FBDBF800305AF811
:107810002410B2E718B2074904F040FBDBF8582007
:1078200056F8243099E77F20E1E77F20C3E700BFC7
:107830003415002008150020AC140020F0B4847A20
:10784000494B0278012C1A7022D142884749C2EB79
:1078500002329208A1FB02120226120A5A80818883
:10786000434DC1EB0131A5FB0121890A9980C188F3
:107870008672C1EB0131A5FB0121890AD9800289F9
:107880003C49C2EB0232A5FB0252920A1A810C70EB
:10789000027C012A52D012B90121364A1170827C31
:1078A000324C9A74B0F81320D0F81B50C2EB02325D
:1078B0009208A4FB0212C2F30F22A3F81320B0F81F
:1078C00015202D49C2EB02329208A4FB0262C2F3DA
:1078D0000F22A3F81520B0F81720C2EB023292084D
:1078E000A4FB0262C2F30F22A3F81720B0F81920FC
:1078F000C3F81B50987FC2EB0232060900F00F0755
:107900003D053005A0EB0620A5EB07258008920871
:10791000AD08A4FB0262A4FB0565A4FB0004587F2C
:107920001E7F00EB1424154806EB1525C2F30F2229
:107930000D800480A3F81920F0BC704700250226B2
:107940001A7481890A4CC1EB0131A4FB0121890A17
:107950009981C2890674C2EB0232A4FB0212054966
:10796000920ADA810D709AE75C15002071000770A9
:1079700049D6B9F2E02D00205C2600200428002022
:10798000002370B4124D134A13482B606B60AB6038
:10799000EB602B61114D124C124E136053609360DB
:1079A000D3601361036043608360C36003612B6035
:1079B0006B602B8123606360A360E36023613360AD
:1079C00073603381194670BC2822074810F0F7BF56
:1079D000842E002078260020F0270020BC260020DE
:1079E0009C2E00206026002020250020C0F5FF638B
:1079F0000733002B2A4BB8BFC0F57F621B78B4BF9A
:107A00000E320246D3B110B4264B1C8994422BDDB2
:107A1000002C39D0244A12888A4235D8234A128849
:107A20008A4231D3DB7E012B33D0022B2CD140F2A2
:107A3000FE71884294BF0220012026E0194BD889AC
:107A4000904201DD022070479A7C02B3B3F8172000
:107A50008A42F7D8B3F81900C0F57F600F30814231
:107A6000CCBF0220012070479A7C52B1B3F8172096
:107A70008A42CDD8B3F81920C2F57F620F328A420C
:107A8000C6DB012010BC7047022010BC70470120EB
:107A9000704740F2FE7188428CBF02200120F4E75B
:107AA000E02D00205C1500205C260020042800202A
:107AB0002DE9F04F91B0834606A8CDE901238A460F
:107AC0001A9E02F01DF99DF82130022B00F0B780BC
:107AD000644B1B780593002B00F0B1800024A14675
:107AE000DFF89C81604AABF1020BAAF1020A3178FF
:107AF0003BF9027F3AF9025F18F8013B002941D0B7
:107B0000A9B2B8B2CDE90332FFF770FF019B01289B
:107B100033F914E0029B33F914C0DDE9033200F0BD
:107B20008A80022824D1115D19BB4FF00101115543
:107B30005BBB4E494E4851F8241020F81470481C85
:107B400001214C4F27F814504B4D25F814E04B4DB4
:107B500025F814C03370454B43F8240001340A2C37
:107B600008F8011C06F10106C1D111B0BDE8F08F83
:107B7000115D0129DCD0012B07D03C4B115D43F88E
:107B80002490EBE7012B1155F7D1394B4FEA840CC8
:107B900033F9141063007F1A002FB8BF7F423349B6
:107BA000972F51F8240017DC324931F914106D1A5F
:107BB000002DB8BF6D42462D0EDC2F28115D02DC72
:107BC00011F0FD0542D001293ED1284B013086F845
:107BD000009043F80C00C1E74FF0020111550599E0
:107BE0002F28C8BF002108460221204D45F80C90DF
:107BF0000028B3D01E4D1F4FE85E019DABF800007A
:107C0000F85EAAF800001C48185E25F814001B480E
:107C1000029D185E25F814004FF0010516483570D6
:107C200023F80090124D154825F8039027F803908B
:107C300023F8009092E74FF0020111559BE711B035
:107C4000BDE8F04FFFF79CBE0020CEE7012903D02E
:107C5000064840F80C50CDE7044D013045F80C00C3
:107C6000C8E700BF5C150020BC26002020250020AE
:107C7000842E00209C2E002078260020F027002053
:107C800060260020C0F5FF630733002B3C4B70B427
:107C90001D78BABFC0F57F640E34044645BB9A7C9C
:107CA000002A51D0B3F81320364E8A42367806D8CF
:107CB000B3F81520C2F57F620F32914257DD002ED6
:107CC00045D02522304D2D888D4240D82F4D2D880E
:107CD0008D423CD3A2423ADADB7E012B49D0022B03
:107CE00035D140F2FE71884294BF022001202CE081
:107CF000244A1278A2B164295A882BD8914232D8EA
:107D00009A7C52B1B3F813208A42DAD8B3F815201E
:107D1000C2F57F620F329142D3DC70BC0120704704
:107D20009A89A24213DC9A7C002AF6D0B3F8132079
:107D30008A420CD8B3F81500C0F57F600F30884236
:107D4000B4BF0220012000E0104670BC7047022042
:107D500070BC7047914206D89A88A242D0DD252A8D
:107D600028BF2522AEE7DA88A242F8DCC8E7284619
:107D7000EBE740F2FE7188428CBF02200120E4E76D
:107D80005C150020E02D00205C2600200428002047
:107D90002DE9F04F8BB0064668460F4601F0B0FF64
:107DA0009DF80930022B38D0204B1B7873B3002488
:107DB0004FF00209A0464FF0010A149BDFF870B0A3
:107DC0005D1E15F8013FDBB137F8141036F81400CA
:107DD000FFF758FF012816D0022805D11BF8043000
:107DE00023B90BF804A003E01BF80430012B01D1E8
:107DF00085F8008001340A2CE3D10BB0BDE8F08F88
:107E00000BF80430F6E70BF80490F3E7084A136028
:107E1000536013810BB0BDE8F08F0022044B1A6051
:107E20005A601A810BB0BDE8F08F00BF5C150020CE
:107E30006C2600202DE9F04105460E46174698466F
:107E400082B0089C0094FFF7A3FF43463A463146B0
:107E50002846089402B0BDE8F041FFF729BE00BFF4
:107E600001465422014810F09FBD00BFA405002028
:107E70000021044B03F1780299600C339342FBD14B
:107E8000704700BF0C2E00202DE9F04F3F4F85B00A
:107E90003C68DDF83880012C08BF002200295AD048
:107EA0004FEA400A0AEB0001394D89006E18B468A8
:107EB0000A2C59DDD3F800C00AEB000105EB810163
:107EC00049680AEB00094FEA8909044655F8090098
:107ED0001E46D8F80030ACEB0000591A0028B8BF95
:107EE00040420029B8BF4942039203F081FF039A40
:107EF000834607EB0217D7E9022379683F690097A9
:107F000003F060FF05EB090700283BD0326855F805
:107F1000093002FB0BF203FB00230BEB00025110B4
:107F20000B4493FBF2F33360D8F800307F6803FB17
:107F30000BFB07FB00B0084490FBF2F0C8F8000010
:107F400033685444A4002B51D8F800302C446360AB
:107F500005B0BDE8F08F0E4B00EB400003EB800056
:107F6000816005B0BDE8F08F0134B460012CD3F816
:107F700000C0A1D145F801C0D8F800107160D3F855
:107F800000C09EE7D8F80000D8E700BFA405002095
:107F90000C2E002030B40546064C6968AA68EB68D0
:107FA00000680FC428696969AA69EB690FC430BC0D
:107FB000704700BF7C1500202DE9F04F524EC7B02E
:107FC000726800219200824610F0F9FC73683269F1
:107FD000581EA0EB630090477369984773685A1E58
:107FE0000592002B7DD0D6F800900AEB830AA3F10E
:107FF000020845AC80224FF0FF3106A810F0DFFCEC
:108000008022002126A810F0DAFC19F1FF39DDF8F2
:1080100014B030D3B36998470746BBF1000F6BD05B
:1080200070683369A8EB600098471BEB090F01D01B
:108030007369984706A925AA7C3757F87C3C0D68D8
:10804000AB4203D20B601D4657F87C3C52F8040F3C
:10805000043198423CBF1846136057F8043FAB42C6
:1080600038BF41F8043C834288BF13609442E4D196
:1080700019F1FF39CED2002725AA05A952F8040F1D
:1080800051F8043F07449442A7EB0307F6D11F4B76
:108090004FF001094FF0040B039300234946CDE94B
:1080A0000193202226AB7220CDF800B0FAF7BEFB78
:1080B000174BCDE900B903930023494602932022D0
:1080C00006AB7220FAF7B2FBD6F80090059B97FB3F
:1080D000F9F7013B0593013308F1FF384AF8047DB5
:1080E00088D17368326903EBD3705B10C3EB600017
:1080F000904747B0BDE8F08F73683269581EA0EB17
:108100006300904791E700BF7C150020E0980100D4
:10811000F49801000E4BF0B45F68022F15DD00EB00
:1081200087070C3F0438024600230A4900F10C0679
:1081300052F8045F11F9014B964205FB0433F7D165
:108140001B1140F8043F8742EDD1F0BC704700BFDF
:108150007C15002088150020DFF868C0F0B4DCF83A
:1081600004600024002E0ADD01EB8606043E0B1F8E
:1081700053F8045FAC42B8BF2C469E42F8D1DCF8FD
:1081800008304610A34214DA002818DD00236FF0EF
:108190000045043951F8044FAC42B8BF1F4603F103
:1081A0000103B8BF25469842F4D1B81B1560F0BC56
:1081B000704751F826300020F0BC136070476FF014
:1081C0000045F2E77C150020F0B40446074E00F1AC
:1081D0003007354620686168A268E3681034BC4205
:1081E00006F110060FC5F4D1F0BC70479C150020B5
:1081F0002DE9F047DFF8E89002EB400599F82C30C4
:1082000099F82D2082B0441E0F468DF804208DF879
:1082100005304E464FF0000A4FF0640800E0013C84
:10822000631C17D035F9023D002BF8D0314637F9E1
:10823000140003F033FEB5F9003098423EDBD9F864
:10824000282008FB03F302FB00F29342C8BF4FF063
:10825000020AE4E71F4B1878BAF1000F13D11E4A47
:10826000C2F800A060B91D4999F82E400A68013291
:10827000A2420A6004DD01221046C1F800A01A7073
:1082800002B0BDE8F0870546AAF10200B0FA80F01E
:108290004009854217D0104C02A92268014411F808
:1082A000041C01328A42226011DD00221870226013
:1082B00000220A4B1A6002B0BDE8F0870020054B8F
:1082C0001D788542E7D10022034B1A60F0E728466B
:1082D000EEE700BF08190020FC1800200419002058
:1082E0009C150020014B1870704700BF0819002032
:1082F000034B1B781BB9034A1368013313607047A3
:1083000008190020041900200278014B1A707047E8
:10831000F80500200022034B83F8F02083F8E421C5
:10832000704700BF142800202DE9F04F614D97B031
:108330002C78002C69D000296BD0F42404FB00F4C5
:10834000DFF874811E4608EB040C9CF8F0301746E9
:10835000FF2B68D00133DBB28CF8F030D2F800E0AC
:10836000D6F8009004F1D00B012BCDE904E9C34409
:1083700061D00DF1100900234FF4807A5A460EA8FF
:1083800008EB040B4946CDE90633039300F096F859
:108390000EAA06A9584600F037F9039B59461A461B
:1083A000CDF800A00123484600F084FA012304F12F
:1083B00034011A460A904144CDF800A0484600F026
:1083C00079FA04F168010B9041444FF4C87302221A
:1083D000CDF800A0484600F06DFA04F19C010C9025
:1083E000414449F640430122CDF800A0484600F040
:1083F00061FA06AA0D900AAB594608A800F018FACF
:10840000DDE908232C783A603360204617B0BDE8D8
:10841000F08FF422284B02FB0033204683F8F01043
:1084200017B0BDE8F08F1268336804F1D00BCDE9C6
:108430000423C3449DE74FF0000A61465246534669
:108440008CF8F1A08CF8F2A00132042AC1F800E007
:10845000C1F80C904B600B618B60C1E90533C1E939
:108460000733C1E90933CB6201F13401ECD1F421C6
:108470004FF4C863FA2201FB00800DF1100902637A
:108480004266C0F89820C0F8CC208361C36483653D
:10849000C0F88030C0F88C30C0F89430C0F8B430E8
:1084A000C0F8C030C0F8C8304946584600F098F8C7
:1084B00061E700BFF805002014280020F0B4D1E9DE
:1084C0000057D2E900134E1BDB1B002EB8BF7642CB
:1084D000002BB8BF5B421E44C82E84B004DC4EF6AD
:1084E000602113898B4266D90124C2E900571346E3
:1084F000002123F8084F02F11C0533F8024FA14276
:10850000B8BF21469D42F8D1937FB142B8BF3146F2
:10851000082B02EB43048CBF00230133052966813D
:10852000937722DD27294BDC294B4A1F03FB02F2FC
:10853000284BD41783FB02531344C4EB631303F299
:10854000CA341429009413DD31293EDC6FF0D102C6
:10855000143902FB01F1204ACB1782FB01520A4475
:10856000C3EB221303F28E3304E040F2CA340094CA
:1085700040F28E3301934FF42F730146CDE902335D
:10858000164F00F1280601ADC4F57A7287FB02C3CD
:10859000A3EBE2739BB200F1080220F8023B824297
:1085A000FBD121F80A4B8E4202D055F8044BEBE781
:1085B00004B0F0BC704701339CB296FBF4F696E72A
:1085C0004FF42F7431290094C0DD4FF42F73D1E79D
:1085D000F2FEFFFFEBA00EEA8988888856555555B4
:1085E00070B4D1E90062034600256424C0E900624A
:1085F00000F11C0223F8085F23F8024F9342FBD1DD
:1086000070BC0023837770472DE9F04F0C469246EB
:10861000CFB003900146D0221AA8A4F1020B10F0AB
:10862000C3F95D46D6465046A046804F0AF108067B
:10863000002213461AA930F833C00C6B0133042B07
:1086400004FB0C2201F13401F5D1B2F5FA6F34BF0D
:108650000122A7FB023200F1020028BFC2F38F12F1
:10866000864225F8022FE3D144460023A11D8C4603
:10867000CDE90633CDE908330AF1200A0DF12409CA
:108680000DF1680806AA15464F465C467646D8F8AE
:108690003010029236F8022B34F8020F01FB02F27E
:1086A000B2FBF0F2A445134445F8043B47F8042F0D
:1086B00001D02B68EEE70EF1080EF24508F1340800
:1086C00009F11009069BDDD1002108460C461AADC0
:1086D00005F1D00C2A6B2F68EE683435AC45114497
:1086E00007FB024406FB0200F4D194FBF1F490FB7B
:1086F000F1F1039A10461460D1609346042290462B
:10870000CDE9040300218C460F460E460C46084670
:108710000AAB019303EB080E1AAA00915EF8103B16
:108720001168D2F8089001FB0300D168D2F814A0B8
:1087300001FB0344516809FB03CC01FB036611698B
:10874000343201FB0377009995420AFB031300932F
:10875000E4D1194606AB53F8083008F1040890FB41
:10876000F3F094FBF3F496FBF3F697FBF3F79CFB23
:10877000F3FC91FBF3F1B8F1100FCBF83400CBF818
:108780004040CBF83860CBF84470CBF83CC0CBF815
:1087900048100BF1340BB5D1DDE904430399D03116
:1087A00003910025A846AE46AC462F462E46DDF87E
:1087B00004901AA9009359F8100B8B69D1F82CB0CA
:1087C00003FB0066CB690BFB005503FB00770B6ACC
:1087D00003FB00CCD1E9093A34318A4203FB00EEB5
:1087E0000AFB0088E7D1009B96FBF3F697FBF3F7B3
:1087F0009EFBF3F09CFBF3FC98FBF3F195FBF3F588
:10880000019BC4E9066704330193039BC4E908C0D4
:10881000C4E90A153434A34204D0029951F8043F44
:108820000291BEE74FB0BDE8F08F00BFD34D62109C
:108830002DE9F0438C460C460026DFF87480971E25
:10884000043B063237F802EF53F8045FBA4205FBE7
:108850000EF5A8FB059ECCF8305006EB9E160CF1E9
:10886000340CEFD101250A46D031136B3432B3FBFF
:10887000F6F3002B08BF2B4642F8043C9142F4D19A
:1088800000210D460E46236BD4F800C0E76834344F
:10889000A24219440CFB036607FB0355F3D196FB78
:1088A000F1F695FBF1F1C0E90061BDE8F08300BF8E
:1088B000D34D62102DE9F04FD2B28BB0012A019254
:1088C000044600F05881C0F02881022A00F09D8003
:1088D00000234FF480629C461F461D469E469B46E1
:1088E0001E46984699469A46CDE90733059203936A
:1088F0000293069304930093039AD4E90004A4EB33
:10890000090406FB04290BFB0433A0EB0A0043F324
:10891000951308FB00EE06FB00550BFB007708FBE8
:1089200004CC49F39519C1E90493029B4FEAAE2E9A
:108930008B61019B45F3951547F395174FEAAC2CD6
:10894000C1E900E5C1E9027C002B00F0E080009A5B
:10895000059B764203FB02F3069A002B4FEA822A1C
:10896000009AB8BF03F2FF3306FB02AABAF1000F68
:108970004FEAA323B8BF0AF2FF3ACB614FEAAA231A
:108980004B62019B022B00F037810023C1E90A33BF
:108990000B6204FB04F400FB0040A94B984200F377
:1089A000AE80642404FB00F0149BA64A90FBF3F411
:1089B0006310934200F3A38042F21071A24AE417BD
:1089C00082FB0302C4EB223201FB12309F4D561C86
:1089D00080EAE07401FB1633A4EBE07435F816006E
:1089E000002B00FB04F035F81220B8BF5B4202FBFD
:1089F0000300974FA7FB0030400B01FB00F0149BD6
:108A000090FBF3F00BB0BDE8F08FD1F82090D1E9E6
:108A100006073D1809EBD970D1E90ACED1F824A098
:108A200005EB60050EEBDE7809EB0C064FEA6808F3
:108A30000CEBDC7B3D4406EB08024FEA6B0B574422
:108A4000554404925F445D4402EBD27B8A684F44F4
:108A500003924A69674409920A687344914605EB98
:108A60006B05079307EB080300932B4648680AEB56
:108A70004C0A0290029AF24409EB2219039ACDF8AB
:108A800018A009EB621A099AD1E9036006EB2016D7
:108A900006EB6219002D149AB8BF05F10F0302EB23
:108AA00023134FEA851898FBF3F8009A1493960164
:108AB000049AC8F580634FEA821B149A059396FBCB
:108AC000F2F69BFBF2FB029A03FB05F31546099FA6
:108AD000002B3844F444039AB8BF03F2FF338001FB
:108AE000CDF820C003909812099B1544AD01029067
:108AF00097019B014FEA8A2E4FEA892CFCE642F24D
:108B00001070149B90FBF3F00BB0BDE8F08FC1E93F
:108B10000733C1E90933CB623BE78869149A034400
:108B20001846002BB8BF03F10F0002EB20124FEAEA
:108B3000831898FBF2F81492C8F5806202FB03F0E8
:108B400000230028D1F800A0D1F80C90B8BF00F2A3
:108B5000FF3005928212CDE902231F461D469B4637
:108B60001E46CDE907330693049300934FEA8A2EFD
:108B70004FEA892CC0E6486AD1E9065605EB460E55
:108B8000864403440693734632184D6800920A687F
:108B90000F6902EB251ACA68BEF1000F02EB271914
:108BA000149AB8BF0EF10F0302EB23134FEA8E188D
:108BB00098FBF3F81493C8F5806303FB0EFE05934E
:108BC000009BBEF1000F4FEA8316149BB8BF0EF254
:108BD000FF3E96FBF3F600234FEAAE220292BA0163
:108BE000AD0103921F469B46CDE9073304934FEA3C
:108BF0008A2E4FEA892C7FE6DDE9042303FB02F38A
:108C0000089A002BB8BF03F2FF334FEA822C9B1265
:108C1000049A0B62079B06FB02C6049A9B020BFB9D
:108C2000123B002EB8BF06F2FF36BBF1000FB8BFF3
:108C30000BF2FF3BB6124FEAAB238E62CB62A8E683
:108C400014AE47016F110100AD8BDB68089901007C
:108C50005917B7D10268014B1A607047CC15002034
:108C60000146B82201480FF09FBE00BFD01500207A
:108C700070B4D0E900250A4B8468017B867B1A60BA
:108C80005D60427BC57B9C60047C19735A739E7344
:108C9000D0E90512DD731C74C3E9051270BC70477E
:108CA000D01500202DE9F0430746032200204FF0A5
:108CB000010803FB07F6079D104C29448E5D94F8CC
:108CC0000090DFF83CE0DFF83CC006F00F0646FA03
:108CD00002F4E4070CD512F90E4012F90C503C4492
:108CE00003FB0414645D4C453CBF08FA04F42043C4
:108CF00012F1FF32EBD2BDE8F08300BFD89801003B
:108D000018990100209901002DE9F04F8DB0199FAD
:108D10000546059097F802B0F87888468345CDE976
:108D20000832DDF874A04DDC0123B8461F9C0BFA15
:108D300003F20AFB024204921E9A97F801900BFB81
:108D40000A2603FA05F28B40134303934FEA4A03C2
:108D50000693EBB2CDE90A13079298F800404C4510
:108D60000CDD23E0FA0606D4079B834200F09780CF
:108D7000002800F0B1800134A14515DB375DB9064C
:108D8000F9D51E9B1C9A0093214653465846FFF77F
:108D900089FF039B8342E5D19DF81430335598F841
:108DA00001900134A145E9DA98F80300049B069A82
:108DB0000BF1010B1344584556440493CDDA474652
:108DC000DDF828801A993B680846059A40F8223059
:108DD00050F828309400C3F30741B1EB136F4FEA0A
:108DE00088003B6019DC94461E9B97F801900AFBB3
:108DF00001353B7899450BD32B4413F8016B46455D
:108E000004BF03F801CC97F801905A1B9145F4DA9E
:108E1000FB7801318B425544EBDA1B9B08F10101D1
:108E20001844099B8B420FDD01279C461B9A059D28
:108E3000161952F82550026807FA01F31340013160
:108E40001D438C453560F6D100231B9A984542F8A6
:108E5000283040F383800122059F1B9802FA08F115
:108E60000444BC4602FA07F0CD4316461B9F06E0B9
:108E700002432A4047F82320013398456ED057F823
:108E800023200A42F8D09C45F2DCF2DA226806FA86
:108E900003FE42EA0E02226057F82320E9E79DF81C
:108EA000143008983355049B98F8019033F9142036
:108EB000036804FB02F103EB412303600BFB02F1A7
:108EC000169B1B6803EB412316990B60189B1B68CC
:108ED0001344189A13604EE707F00F03CDF864802F
:108EE0000325984648FA05F3DB072FD51D4B1C9A3E
:108EF000EF561D4B5F4415F903901E9BA144009350
:108F0000384653464946FFF7CDFE039B83421DD1A9
:108F10001E9B0B9A0AFB0737049B07F80920325562
:108F200033F91420089804FB02F1036803EB412392
:108F300003600BFB02F1169B1B6803EB41231699A0
:108F40000B60189B1B681344189A136015F1FF35CA
:108F5000C8D2DDF8648098F801900CE70DB0BDE848
:108F6000F08F00BF18990100209901002DE9F04F02
:108F7000814293B005460C460B9298461C9F01DB3C
:108F800004460D461E9B58F824A033F914201D9B5F
:108F900057F8249033F814C002FB0AFE09FB02F6CE
:108FA00002FB0CFC1D991E9B31F815B033F91530EE
:108FB00058F8250057F8251003FB00EE03FB0BCCF7
:108FC00001FB0366AAEB00001344A9EB0101CDE904
:108FD0000FC3CDF834E00E9602F00AFF209B8346C3
:108FE00053F8242053F825309446D9B2D0B28842A1
:108FF00088BF61F3070CC2F30720C3F3072188423F
:1090000038BF61F30F2CC2F30740C3F30741884216
:109010004FEA136388BF61F3174CB3EB126F88BF3D
:1090200063F31F6C269B239A0993259B0692229A31
:109030000893249B0592209A0DF1440E10A80FA9C5
:1090400007930EABCDE900310492CDE9020E0B9AE5
:109050000DAB29462046CDF844C0FFF755FE0DA8BC
:109060000FC891FBF3F190FBF3F092FBF3F24FEAA0
:10907000840948F8090047F809101D9966008A53C9
:109080001E9A4FEA450A9353219B33B19B5F9B4540
:10909000B8BF9B46219B23F806B01F9A1F9B115D0A
:1090A0005B5D00228B4238BF0B461F990B551E9B00
:1090B00023F80A2013B0BDE8F08F00BF2DE9F04F70
:1090C000DFF8D0B08FB09BF80C40189F002C5ED01A
:1090D00000285CDD00250D9337F9153005F1010AF4
:1090E000002B91468846064654464EDD564503DC25
:1090F0004DE00134A64240D037F91430002BF8DDA2
:1091000059F8243059F8250058F82510C01A4EF2A5
:10911000B05358F82420891A0029B8BF494203FBEC
:1091200001F14FF461430028B8BF404203FB00F057
:109130000914001402F05CFEDBF814308342D8DD21
:10914000209B21460A931F9B324609931E9B28466B
:1091500008931D9B013407931C9B06931B9B05934F
:109160001A9B0493199BCDE902730D9BCDE90093E3
:109170004346FFF7FBFEA642BED1554637F91530F0
:1091800005F1010A002B5446B0DC5645F5DC0FB062
:10919000BDE8F08FD01500202DE9F04F654C95B05B
:1091A000247C1E9F34B3002824DD90468A468146E5
:1091B0004FF0000B0D9337F91B30BBB158F82B2043
:1091C000249902F58072521201FB02F65AF82B30F4
:1091D000259903F5807331445B12C95C56485945A3
:1091E000057825D0A94209D3880671D40BF1010B6B
:1091F000D945E0D115B0BDE8F08F7746269B4A46A9
:109200000A93259B58460993249B0893239B079315
:10921000229B0693219B0593209B04931F9BCDE9E2
:1092200002730D9BCDE900835346FFF79FFEDDE7F8
:109230004FF0FF306FF0FE1C864603243D49CDF809
:109240004CC089680DF1480C11913C490E95129162
:1092500026991E9701EB4601109159000F9113AE0C
:109260001EEB020E18442BD4002829DB23997145EC
:1092700026DD2499814223DD01FB0EF725990E9D01
:109280003944095CA9421BD20F9D8B4505EB47076A
:1092900016D0269D35F907E06425109F05FB0EFECC
:1092A00037F91370119D05FB07F7BE4508DD109DCA
:1092B00035F91000AE46642505FB00F0B84237DCF6
:1092C00024B1013C14F90CE0A057C9E71E9F8DE7BB
:1092D000209850F82B00C0F307249C4224D0C0B241
:1092E00098420BBF032401244FF0020C4FF0000CF6
:1092F000BE4601F00F0025990B4440FA04F1C9075E
:109300000DD50F49249F61560E4E114407FB0131C4
:10931000A657895DA94202D259457FF46EAF013C40
:109320006445EADA774661E703244FF0020CDFE791
:109330001E9F63E7D0150020D89801000101FFFFB0
:1093400018990100209901002DE9F04F83B0DDE963
:109350000D4704FB02FE07EB0E04E65C864245D097
:109360008E4243D016F0200549D000250324AA469A
:109370004FF0010BDFF8A4C006F00F069CF8009038
:10938000019307EB030C46FA04F7FB0715D5214FB1
:10939000214BE75714F903800D9B174403FB07C7C4
:1093A00017F808800BFA08F7C84547EA050704D202
:1093B000AF421CBF3D460AF1010A14F1FF34E2D26C
:1093C000012202FA00F002FA01F10843A842019BCF
:1093D00019D0284010D05B0003EB4E0E0F9B33F9E1
:1093E0000E0090FBFAF003B0BDE8F08F5B0003EBDA
:1093F0004E0E0F9B33F90E0003B0BDE8F08F2846E8
:1094000003B0BDE8F08F934003EB4E0E0F9B33F992
:109410000E00F1E71899010020990100D898010089
:109420002DE9F04FB74CADB0E47B1D94002C00F05B
:109430000E81002800F0038121930023CDE91B1247
:109440001293431E16902093129B209A934280F20F
:10945000FE803A9B129A194651F82230511CCB409B
:109460004FEA82021E911792119300F05981169BC8
:1094700019461E9B994240F3538110930023129A80
:109480001F93369B03EB42031A930BE0109B119A38
:10949000013352081093119200F03E81169A9A42BD
:1094A00000F03A81119BDB07F0D51B9B17991C46F6
:1094B00058581C9B109A1D4654F82240595855F88C
:1094C0002230051B0E940F93CC1A85EAE573A3EBAB
:1094D000E573189384EAE473A3EBE4731993369E5F
:1094E0001A9B36F91220B3F90030002C40F0FF80AF
:1094F000002D40F018814FF4007BDDF874800E9E43
:109500000F9F34463D4604FB03F402FB004405FB79
:1095100003F5134494FBF3F402FB015595FBF3F5BB
:10952000389B179A9C469A5824941446CDE9256195
:109530000026109B23905CF82330D0B2D9B2814230
:1095400038BF61F30704C2F30720C3F30721884241
:1095500038BF61F30F24C2F30740C3F307418842C9
:109560004FEA136388BF61F31744B3EB126F88BFF0
:1095700063F31F642795230EC4F307459D42289784
:10958000CDE929662B9600F3D48001331393E3B21F
:109590001493C4F30723159329AF149C159A94428E
:1095A0005CDC9DF848306E020D9333464646984683
:1095B0009DF840A002F101093E9B2A4603933D9B82
:1095C000514602933C9B0D9801933B9B009323468D
:1095D000FFF7BAFE00283DDDDDE90E324FEA442CEC
:1095E0000221ACEB030E0EB30BFB0EF3A2EB6323D5
:1095F000A3EB0803002BB8BF5B42B3F5007F09DA89
:10960000C3F5007300FB03F357F8212002EB63233B
:1096100047F82130F1B1013923AB53F8213026AAA4
:1096200052F82120ACEB030E002EDDD1A8EB020294
:109630000BFB02F2A3EB6223A3EB0C03DAE76FF060
:109640000043314C3149324A23600B6010602DB029
:10965000BDE8F08F01344C45AED1B046139B0135C7
:109660009D429AD1DDE92A42DDE91801299B642552
:109670009A42A8BF1A4605FB04F4154602F0F0FB17
:109680002D2801DDC0F15A001E4A0CCA03FB00F36D
:10969000C0F12D0002FB00321E4B83FB0231D317B9
:1096A0000A44C3EB621305FB03F3A342BFF6EEAE1D
:1096B0003E9B169A0A933D9B109909933C9B1298E6
:1096C00008933B9B07933A9B0693399B0593389BE2
:1096D0000493379B0393369B0293219B01931C9B1E
:1096E00000931B9BFFF742FC1D9B1F93CEE6DDE919
:1096F0001867BE4217DA6D0295FBF4FBDDF8748043
:10970000FDE600BFD01500201C060020200600202A
:1097100024190020B7600BB61F9B002B7FF494AE7A
:109720001E9B129390E6640294FBF5FB4FF0000839
:10973000E5E6DDE9180102F093FB2D287FF7A6AEE0
:1097400000252C469EE700BF2DE9F04FA54CAFB099
:10975000A47B002C00F03581002800F03281914676
:109760001793389B4FF0000B023B189303EB400319
:1097700010934B4689469A460D901E2200211EA842
:109780000FF01DF900211E2226A80FF018F9964BA4
:109790004FEA4B0133F91B301391002B40F3368114
:1097A000924B33F91B30C3EBC3139B1214930D9BE5
:1097B000002B40F32B8100238D4A1F468A180F92FD
:1097C0008C4A1293189B8A180E921D46CDF858B0F9
:1097D00003E0109B01379D4272D035F9022F002A19
:1097E000F7DD0E9B0F98B3F9004059F827205AF87F
:1097F0002710B0F90000611A801A02F0F9FA662405
:109800003A9E7D4904FB00F4F05D51F8046C02F0CF
:1098100045FBA4128046794920B202F03FFB0E9A24
:1098200015900F98B2F900C05AF82710B0F900202F
:1098300059F82700ACEB01016A4B101A00299A6F06
:10984000B8BF49420028B8BF4042D3F87CB011925B
:1098500002F006FB2D28C8BFC0F15A0000FB0BFB2D
:10986000119AC0F12D0002FB00B2654B654983FBE4
:10987000023C139B9444595ED2170E44C2EB6C1207
:1098800008FB04F806FB02F6B04580F29D806420D8
:10989000544BD3F8802000FB02F2424540F3948001
:1098A000159B8B42129B03F1010280F28D800121F6
:1098B000D3B212931EABD955109B01379D428CD168
:1098C000129BDDF858B0012B40F2A0809DF8782063
:1098D000002A40F092811EA913460D9C04E011F865
:1098E000010F002840F07C8101339C42F7D1199B85
:1098F0009F004FEA430809EB07030F930AEB0703A6
:1099000011933B9B1F44389B43441293399B9844CB
:109910000026CDF84CB0CDF83880DDF834B0DDF855
:1099200064801DAC1CAD002A3DD0B0453BD026ABB9
:109930009B5D419A002B3C9B18BF00230A92409AE2
:10994000059309923F9A4B4608923E9A31460792F8
:109950003D9A404606923B9A04923A9A0392389A6C
:109960000292179ACDE900A25A46FFF7FFFA38682B
:10997000129B119A0F99B3F900301268096802908E
:109980004198CDE900540690409805903F98049086
:109990003E980390404601F05FF9DDE91C0102F0BA
:1099A00027FA0E9B18800136B3452DD01EAB9A5D69
:1099B000B9E7109B0BF1010B023310930D9B5B4534
:1099C00037D12FB0BDE8F08F149BA3427FF701AFD2
:1099D000012212991144CBB2129326ABDA551EAB79
:1099E000DA55F6E6D01500204C2700206825002027
:1099F000CC2D002010260020F81500202016002075
:109A0000B7600BB6F82D0020DDF84CB00BF1010B60
:109A1000BBF10A0F7FF4B1AE5346CA4699460D9B7F
:109A2000002BCEDD4FF0000B399B4C46DDF8E0906B
:109A3000109339F91B3009EB4B02002B1892B8DD5B
:109A40004FEA8B030AEB03021B93E3184FF0000865
:109A50001A92199340E02E4659464546419B0D9A6D
:109A60000A93409B284609933F9B08933E9B07938C
:109A70003D9B06933C9B05933B9B04933A9BCDE90E
:109A80000293179BCDE900435346FFF76FFA3B98CB
:109A90000E9F0F9BC059159A1699B3F900301268A2
:109AA0000968029041980690409805903F9804906C
:109AB0003E98039026A801901EA80090284601F029
:109AC000CBF826991E9802F093F930800D9B08F18F
:109AD000010843453FF46DAF39F918304FEA4805A6
:109AE00009EB0502002B0F92F0DDC345EED054F8D0
:109AF00028205AF8283054F82B105AF82B00891ACD
:109B0000C01A02F075F95AF82B3011905AF8280053
:109B100054F828101B1A54F82B2083EAE376A6EB9E
:109B2000E3763A9B521A82EAE277394913F80B003E
:109B3000A7EBE27702F0B2F93A9B1290344913F89E
:109B4000080002F0ABF9334A3946D2F8B03013902E
:109B500030461493D2F8B46002F082F942F2107CDD
:109B60004FEA88032D280E935344C8BFC0F15A0012
:109B700016930E9B00FB06F6E3181593149BC0F199
:109B80002D0003FB0063234A109E2348D2F8847003
:109B9000B6F9001080FB0320129A184402FB017EE4
:109BA0003999139A31F91810DB1702FB01E2C3EB64
:109BB0006010119B02FB00F20CFB03FC399B9445E7
:109BC0001D4483DAC345FFF646AF189B41460F9309
:109BD000199B5D4615931A9B16931B9B0E933DE7AD
:109BE0009F0009EB07010F910AEB070111913B99C7
:109BF0004FEA43080F44199385E6389BDDF8E4806B
:109C0000CDE911A300233B9FCDF83C9019937FE64B
:109C100058160020D0150020B7600BB684B038B5B8
:109C2000174D04AC84E80F00272240F21461154858
:109C300004AC00F0C1F80FCC28606960AA6003CCC6
:109C400018222861696128464FF4B871EB6000F072
:109C5000B3F80D494FF4606000F0FCF80B494FF485
:109C6000905000F0F7F8642000F0DAFC632000F078
:109C7000D7FCBDE83840602004B000F0D1BC00BF84
:109C8000482500202C1900206006002070060020C6
:109C900084B030B402AC84E80F000A4B9DF8082071
:109CA0009DF80A109DF812509DF813401A70997093
:109CB0009D72DC7230BC184618224FF4B87104B0A3
:109CC00000F0A4B848250020F8B500F0D5FA044605
:109CD0000A4E00F12007354620686168A268E368F3
:109CE0001034BC4206F110060FC5F4D12068306074
:109CF000A288A379B280B371F8BD00BF2C190020EF
:109D0000F0B4074604460C4E06F1200C35460FCD44
:109D1000654520606160A260E36006F1100604F111
:109D20001004F3D130682060B288B3793846A2803D
:109D3000A371F0BC704700BF2C19002070B404461A
:109D4000174D00686168A268E368164E0FC5206968
:109D50006169154A03C57368A569207F51692B4362
:109D600073600870A37F657FCB71E17F93680F48B4
:109D70000570197094F820000D49587094F821501E
:109D80000C489D7094F82250DD70D368A28DD4E900
:109D900009651A811E605D60086070BC704700BF75
:109DA00088270020B0080020380800209C190020D7
:109DB0000C2600201DA30000F8B5134B0C0A53F825
:109DC00024606EB1F468CFB2013C05E073681B5D9E
:109DD000FB1A002B05DA2C46631C04F1FF35F5D184
:109DE000F8BD1546B368326833F81430014652F8AE
:109DF00024002A4618440EF0D7FDB36833F8142027
:109E00002A4423F81420F8BD90060020104BF0B42B
:109E10000C0A53F824706FB1FB68CEB2013B05E029
:109E20007C68E45C341B002C06DA2B46591C03F1D9
:109E3000FF35F5D1F0BC7047BC68396834F8134081
:109E400051F82350A41A01462819F0BC0EF0ACBDFD
:109E500090060020044B000A53F820201AB9142859
:109E600098BF43F8201070479006002000232DE98A
:109E7000F043036069B3CE68D2B206F1804C06F1BC
:109E800000470CF1FF3C013F06F1FF3EB342A7EB58
:109E90000308AEEB0305ACEB030915D04C680133A6
:109EA000645D141BF2D40D6855F82990B9F1000FC8
:109EB00007D08D6835F818502D1B002DE6DD0560A4
:109EC000A1444846BDE8F0834FF000094846BDE88C
:109ED000F0838946F5E700BF0023B1F5704F70B4F9
:109EE000C1F30724036028DA132C1FD9144D06464A
:109EF0006A68E86889B2431E02EB400204E032F867
:109F0000020D081A07D52346581C03F1FF34F6D179
:109F1000002070BC7047AA68296852F8232051F8C5
:109F20002330121A3260184470BC7047054B8AB255
:109F300053F8241070BCFFF799BF1846E9E700BF3B
:109F4000800600209006002000B583B0014601A8DD
:109F5000FFF7C2FF044B186008B1019B1844034B84
:109F6000186003B05DF804FB9019002094190020DC
:109F700070B50E4E024635681DB10D4B1C68A542EA
:109F800006D31446084600210EF019FD204670BD88
:109F9000641B8442A8BF044608462246294625443D
:109FA0000EF002FD3560204670BD00BF9019002004
:109FB0009419002070B50B4E35681DB10A4B1C6812
:109FC000A54202D30024204670BD641B8442A8BF72
:109FD00004462846224625440EF0E6FC356020461D
:109FE00070BD00BF9019002094190020B0F5C06F1B
:109FF00010B521D0224A1378DC0908D1B0F5047FCE
:10A000002BDC204B5B69EBB1BDE81040184792F99F
:10A010000030002BF5DAB0F5047FF2DD137803F0A1
:10A020007F0303F504739842EBDC44189C42E8DD9F
:10A0300000F04EF8012010BD002905DB124B1A7804
:10A04000A02A18D0002010BD0D4A1378DB09D8D003
:10A0500092F90030002BD4DAE0E703F07F0303F538
:10A0600004738342CDDB4418A342E1DB92F9002064
:10A07000002AC6DADAE7052201201A7010BD00BFF7
:10A08000A41B00208827002030070020024B1B69FA
:10A0900003B118471846704788270020084B094A23
:10A0A0005B78DBB2012B137006D0022B03D10122A7
:10A0B000054B5A7070477047044B1B68184700BF28
:10A0C00044070020DC1900203007002088270020EA
:10A0D00008B50A4B1B78012B0CD0022B02D10022B1
:10A0E000074B5A70074A137803F080036FF3C713C6
:10A0F000137008BD044B5B689847F3E7DC19002038
:10A1000030070020A41B0020882700202DE9F843F9
:10A11000254EDFF8A8903378244DDFF89C80244F3B
:10A12000012B06D0022B1BD06A78934238D1BDE8B0
:10A13000F883D8F8083098470446B9F1000F28D1C1
:10A14000D8F804309847D8F800309847DFF8709076
:10A150006B783278DBB2934209D1002CE0D1E6E78C
:10A160001A467C786B78E4B2DBB29342F5D0012AD0
:10A1700012D0022A02D100220D4B5A700D4A697882
:10A180001378317003F080036FF3C7131370BDE8C9
:10A19000F88309F1FF39DBE7074B5B689847EDE788
:10A1A0001A46012AE5D1F7E7DC1900204407002010
:10A1B00030070020A41B002088270020FF2C01006E
:10A1C000FE2C010038B5194C2378012B17D0022B37
:10A1D0000CD0174A5278934206D0164A137803F0EF
:10A1E00080036FF3C7131370002038BD124B104A61
:10A1F00059785278022AF7D000225A70EDE70F4DB5
:10A20000AB68984718B16B6898472B6898470A4B1A
:10A2100007492278587849789142E5D0012A02D13D
:10A220006B689847D9E7022AE6D0D6E7DC19002008
:10A2300044070020A41B00203007002088270020AE
:10A24000A023034A13701378A02BFCD0704700BFE3
:10A2500030070020014B1878704700BF44070020EA
:10A26000014BD878704700BF44070020014BD870DD
:10A27000704700BF4407002000487047480700208F
:10A28000014B9878704700BF44070020014B98703D
:10A29000704700BF4407002008B5FFF793FF08B9D7
:10A2A000014B186008BD00BFA01B00200A46F8B58E
:10A2B000094F0A4C3B6826689B79B51803EB83016C
:10A2C00003EB41039D4200D9FFDE0146B8683044EC
:10A2D0000EF06AFB2560F8BD84070020A01B00205B
:10A2E00070B50D460646FFF711FF094A094C137871
:10A2F000094963F07F0365F306038D80A568137039
:10A30000A660FFF7CBFEFFF701FFA56070BD00BFA1
:10A31000A41B002084070020900700202DE9F04FA7
:10A3200087B09DF8584006460F4690469B469DF8DC
:10A3300064903CB1FFF7B0FF002800F0D98007B06F
:10A34000BDE8F08F6F4B1D460193FFF7DFFE2C60D9
:10A350000024A642CDE90344059440F3B6804B4661
:10A36000DDF84CA0684DD1469A466BE037F914E011
:10A3700038F9140021B1B5F90020724500F0BB8016
:10A3800001239DF80E104FEA2E2C9DF80C206CF343
:10A39000030104F1010C6CF303029DF80DC063F39B
:10A3A00007124CEA030C149B8DF80FE08DF8100097
:10A3B00013F804E00012109B60F307118DF80E10E3
:10A3C00033F914108DF80C20FE29C8BFFF223BF88A
:10A3D0001400119BADF8110053F824006EF3410CEA
:10A3E000D4BF8DF813108DF813208DF80DC0C1B2B5
:10A3F000C0F3072CC0F30742ACEB0101C2EB1062C3
:10A4000091428DF815A04FF04D0354DD03FB01F18F
:10A4100089118DF816108DF817200C210DEB010015
:10A42000FFF744FF37F9142099F800102A8038F913
:10A4300014206A800134A642297109F1010905F14D
:10A44000060542D099F800202979002A8ED10029EA
:10A45000F0D0B5F900109DF80DC09DF80E009DF8E4
:10A460000CE062F3000C0A1262F30300621C62F358
:10A47000030E7246012363F30712149B8DF80F102D
:10A48000195DB5F902E061F3410C0C218DF810E083
:10A490004FEA2E2E6EF307108DF80E000DEB010023
:10A4A0008DF815A08DF80DC08DF80C20FFF7FEFE7D
:10A4B00099F80010BEE703FB02F2ACEB000092112A
:10A4C0008DF816208DF81700A7E7019B1B68002B5D
:10A4D0003FF435AF0D490E480A78838002F07F02C1
:10A4E00063F306020A70FFF7D9FD07B0BDE8F08FED
:10A4F000044B01932CE7B5F9022082427FF440AF70
:10A5000098E700BFA01B0020A81B0020A41B002070
:10A510009007002030B5094D83B02B780446834264
:10A5200008D00B23022101A88DF805408DF80430D6
:10A53000FFF7D6FE2C7003B030BD00BFEA1B002031
:10A5400000B583B08DF804008DF8051001A8022134
:10A55000FFF7C6FE03B05DF804FB00BFF0B4224C69
:10A5600082B025788DF80720854202D002B0F0BC79
:10A570007047FF261D4802AD076B15F8012DBF6817
:10A580001B4892000361C0E902151A4B3A81069AF2
:10A5900026701A608A7822B30B7908784E7902FB0C
:10A5A000003006F07F06144B06FB00F09F68386011
:10A5B0008B795BB10022013B01EB83056D89013B87
:10A5C0002A445D1CF8D102FB06023A60A0230B4A24
:10A5D00013702378FF2BFCD00523137002B0F0BC5E
:10A5E00070474A78D8E700BFEC1B00209006002097
:10A5F000B0070020841900208006002030070020CA
:10A60000014BDB685881704738080020034B1879EC
:10A61000A0F10100B0FA80F040097047FC1B002057
:10A6200000B583B00146202268460EF099F9012357
:10A630000099064A019802EB8102D2F80510834086
:10A640000B43C2F8053003B05DF804FBFC1B00208F
:10A65000014B1878704700BFAC08002070B4184A4E
:10A66000184B90601960827802B9427803790178BA
:10A67000457902FB013105F07F05134B05FB01F124
:10A680009E68316083795BB10022013B00EB83045B
:10A690006489013B22445C1CF8D102FB0512326044
:10A6A000A024FF2309480A4A04700A49137002E0F3
:10A6B0000B78022B02D11378FF2BF9D070BC7047B6
:10A6C000A008002084190020800600203007002008
:10A6D000AC080020440700200246024B0068516885
:10A6E00003C370478816002000230B490B4A0C480F
:10A6F00010B4C1E90033C1E90233C2E90033C2E951
:10A700000233C0E90033074C0B6113610381C4E9D4
:10A710000033238110BC7047B0180020D8180020E7
:10A7200018190020141C002009232DE9F04F324C89
:10A7300085B0656824688646039530480294304F9A
:10A74000DFF8C090DFF8C0A01A44009137E0067827
:10A750004FEA430C3EF91350002E36D039F913B0AE
:10A76000FC5CA5EB0B010191029988460399002C32
:10A7700018BF884644460199E4B20029B8BF49424F
:10A780008C422ADD009931F913803AF91310A8EBB5
:10A790000108B8F1000FB8BFC8F1000844451CDD3E
:10A7A00034462EF813B03AF90C50009921F81350A2
:10A7B000013B591C00F8014902F1FF3219D014780D
:10A7C000002CC4D1DC551478F2E7009929F8135015
:10A7D00031F913502AF81350EAE7009929F80C5080
:10A7E00031F913404FF00101F9542AF80C40147864
:10A7F000DEE705B0BDE8F08F8816002021190020A3
:10A80000141C0020B0180020D818002030B40546D1
:10A81000044C00686968AA68EB680FC42869206066
:10A8200030BC704790160020014B1878704700BF6D
:10A830001E1C00204FF0000C2DE9F04FE0464FF0B9
:10A840006409334F85B002923A69D7E901EA01926F
:10A85000FA68039210F1FF3044D33A78002AF9D015
:10A8600033F91040744544DD0E9D35F910505545BF
:10A870003FDD4FF0010694460F9D2E547A78002A52
:10A88000E8D0109A52F82060C6F307255FFA86FBDD
:10A89000C6F30742A5EB0B05C2EB16620135013288
:10A8A0009542B5BF09FB05F509FB02F295FBF2F2F3
:10A8B00092FBF5F2019DAC42CCDD51F82040029DA7
:10A8C000A4F50074A4B2B4F5705F55F8205014D903
:10A8D000039C9442BEDD4FF001040F9A145410F112
:10A8E000FF30BAD260460B4B83F800C005B0BDE81C
:10A8F000F08F0F9A02F80080C0E7A5F50075ADB2A1
:10A90000B5F5D05FA6D9039C9442E4DCA2E700BF72
:10A91000901600201E1C00202DE9F04FC3F30746BF
:10A920001C0E8BB0A642DDF85090DDE917E856DC2E
:10A9300006FB09FC12B2A2EB46220292621CDDB2B7
:10A9400009920AB2079505926544159AC3F3072741
:10A950006B1ED3180193169B089703EB4C0C4FEA20
:10A96000490301370693079B08998B422ADC029A18
:10A97000019D002AB8BF5242039204E08A0631D4F6
:10A980000133BB421ED015F8011F8142F6D13CF9BC
:10A990001340002CF4DD059AA2EB432181EAE17219
:10A9A000A2EBE172DEF80010013304FB0211CEF8D5
:10A9B0000010D8F800200399BB4201FB0422C8F81C
:10A9C0000020E0D1069B01369C44019B4B4401933F
:10A9D000029BA3F500730293099B9E42C3D10BB067
:10A9E000BDE8F08F0022159C01F00F0104EB030B72
:10A9F000049341FA02F4E3070BD5094C094B1457B1
:10AA000012F903A0344409FB04B414F80A40A0422C
:10AA100004D00132042AECD1049BB1E7049BB6E7D1
:10AA20001C99010024990100F0B404460F46124E0F
:10AA300000F1300C354620686168A268E368103484
:10AA4000644506F110060FC5F4D13D4620686168E3
:10AA50000A4F03C605F130063C4628686968AA68B3
:10AA6000EB681035B54207F110070FC4F4D1286820
:10AA7000696803C7F0BC7047201C0020581C0020E8
:10AA80002DE9F04F824693B01F46BDF98C3084000B
:10AA900007939DF8903088469146002122461C98E5
:10AAA00006930DF08CFF22461D9800210DF087FFC4
:10AAB000BAF1000F72DD0024DFF898B102E0013432
:10AAC000A2456BD037F91430002BF8DD0025229E0B
:10AAD0001E9B12A853F8243059F8242058F824104B
:10AAE00040F8245D0296219E04900196209E08A8BD
:10AAF0000390009620460895FFF70EFFDDE9083227
:10AB000037F9141093FBF1F392FBF1F11C9A42F820
:10AB100024301D9B43F82410069B012B41D058F88C
:10AB200024005946C0F30800B0F5807FC8BFC0F5C7
:10AB3000007001F0B3F9064659F824004349C0F308
:10AB40000800B0F5807FC8BFC0F5007001F0A6F91D
:10AB50001D9B054653F824101C9B53F8240001F05C
:10AB600047F9DBF82C3083424BDC4020064637F9AE
:10AB700014C0DDE9082302FB06F603FB00F34FEAED
:10AB80008C1C96FBFCF693FBFCF31C9A42F82460A9
:10AB90001D9A42F824300134A24593D113B0BDE888
:10ABA000F08F1C9B58F8242053F8240059F82430C7
:10ABB000C2F30802C3F30803B2F5807FC8BFC2F531
:10ABC0000072B3F5807FC8BFC3F50073CDE90B01F8
:10ABD0000D920E930A9401F00BF900220121042337
:10ABE0000F901B4837F91450079ECDE90220CDE99C
:10ABF000003108220AAB6420CDE91065F7F716FE94
:10AC00005DE7DBF82830079A37F914C09A4202DC76
:10AC100040200646ADE7C6F14003DBE90C12604672
:10AC20000093002301F0CEF8084B37F914C0D3E9A4
:10AC30000C12C5F14003009306440023604601F066
:10AC4000C1F837F914C0284493E700BF581C00200E
:10AC500028990100201C00202DE9F047002688B02B
:10AC60001C1EDDE91087C8F800603E604FDD8A4693
:10AC7000169D08AB43F8046D0295159D0DF1180C57
:10AC80000195149DCDE903C30095129B914606964C
:10AC9000FFF742FE1F4ECAF30800B0F5807FC8BF21
:10ACA000C0F50070314601F0F9F8DFF86CA0C0F192
:10ACB0004003316BDAF83420054600932046002328
:10ACC00001F080F8C9F30809B9F5807FC8BFC9F55C
:10ACD000007905441049484601F0E0F8DAE90C1221
:10ACE000C0F14003064600932046002301F06AF8B5
:10ACF000DDE90623304403FB00F302FB05F0A40169
:10AD000093FBF4F390FBF4F4C8F800403B6008B008
:10AD1000BDE8F087201C0020581C0020F0B4044639
:10AD2000094E00F13007354620686168A268E36883
:10AD30001034BC4206F110060FC5F4D120686168DA
:10AD4000A26807C6F0BC7047A41600202DE9F84F92
:10AD5000061E33DD994690460F4600244FF0640BE3
:10AD6000174DDFF860A002E00134A64226D015F8A6
:10AD7000011B0029F8D0134938F9140001F08EF8AE
:10AD8000DAF8303037F9141003FB00F00BFB01F157
:10AD900039F814E08142DAF828100BFB0EFE01FBB3
:10ADA00003F1B4BF002001208E45B8BF00220A9BEA
:10ADB0001855B8BF1A550134A642D8D1BDE8F88F4E
:10ADC0008C260020A41600202DE9F84F071E2FDD49
:10ADD000DFF860B09D1E0A9B941E4FF06408D946B0
:10ADE00004EB47078E1E03F1FF3A0BE001FB00F076
:10ADF00008FB03F38342B4BF00200120BC420AF8E1
:10AE0000010F15D0494634F9020F01F047F8DBE98C
:10AE10000A3135F802CF03FB01F208FB0CFC944524
:10AE200036F9023FE2DA0020BC420AF8010FE9D10C
:10AE3000BDE8F88FA416002000283BDD2DE9F04383
:10AE4000002637468C1E04EB4008951E34F902EFAD
:10AE500035F902CF7745B8BF77466645B8BF664635
:10AE60004445F3D100254FF06408A946124CD4E9BB
:10AE70000DC404FB06F60CFB07F7079C013C04EB32
:10AE8000000E14F8010F78B131F915C008FB0CFC65
:10AE9000BC4505DB32F9150008FB00F0B04203DACF
:10AEA00084F8009003F80590A64505F10105E8D166
:10AEB000BDE8F083704700BFA4160020034610B41D
:10AEC000034C59689A680068DB680FC410BC70476F
:10AED000E01600200023F0B4344A354D354C364896
:10AEE000364F3749C2E90033364EC2E902331361A7
:10AEF000C5E90033344AC5E902332B61C4E90033A4
:10AF0000324DC4E902332361314CC0E90033C0E95A
:10AF1000023303613B602F487B603B81C1E9003312
:10AF2000C1E902330B61C2E900332B49C2E90233A4
:10AF3000C6E9003313613381284A294EC5E900333D
:10AF4000C5E902332B612360264D6360A360E36093
:10AF50002361254C036043608360C36003610B6021
:10AF600022484B608B60CB600B61136020495360BB
:10AF70009360D360136133601E4A736033812B602A
:10AF8000C4E900336B602B81036043608360C3605E
:10AF900003610B604B608B60CB600B61238113609E
:10AFA00053609360D3601361F0BC7047E41C0020D1
:10AFB000F81C0020201D0020D01C00208C26002022
:10AFC0000C1D0020A41C0020BC1C0020901C002094
:10AFD000F82D0020DC270020E42D00204C27002045
:10AFE0008025002008280020B01C0020CC2D002047
:10AFF00010260020682500202DE9F04F440004F1C0
:10B0000008058BB0824625F00705073020F00700C1
:10B0100000AFADEB050D6E46ADEB000D6846FD6F64
:10B02000F961E91D21F00701ADEB010DBA610021C5
:10B0300052467B61BE60D7E920B378607B620DF039
:10B04000BEFC2A464FF0FF3168460DF0B8FC2246A0
:10B05000796F3046C7F810D00DF0A6FCBAF1000F9A
:10B060007B6A67DDBA6E002602F1FF3909EB0A023E
:10B070007A6203E07A6A013691455BD019F8011FC4
:10B080000029F7D07A6F002D32F916A0604A516876
:10B0900001EB4A0AEEDD4FF0FF323A62D7F88C201E
:10B0A000C7F80C900024A2F10208994602E001348E
:10B0B000A54220D038F9022F002AF8D03B6F59F86A
:10B0C000241033F916C0FB6E5BF8242033F9160008
:10B0D000A1EB0C01101A00F08BFE4FF4614303FB4F
:10B0E00000F000145045B8BF3C6204F10104B8BF41
:10B0F0008246A542DED13A6A4B46511CD7F80C90E5
:10B10000B8D0396989564A1C78D0BA6832F911002A
:10B110008245AFDA00244FF0010C22F816A0386AFD
:10B120003A6916547A68545402F806C07A6A0136AD
:10B130009145A3D1002D5DDDD7E9246CD7E926E840
:10B14000002210463969013D0D444C1E7D6214F900
:10B15000011F4D1C4AD05BF8225053F82290AA469A
:10B16000FD6925F811A0BD6925F81190D7F8885020
:10B170001CF8029035F812A07D6925F811A0D7F8C7
:10B180008C5035F912A03D6D25F811A036F912A0AA
:10B190007D6D25F811A0BD6D05F801901EF8029097
:10B1A000FD6D05F80190BD6F6A54D7F8A05035F9D0
:10B1B00012903D6EAA4658F822504AF821507D6EF2
:10B1C00025F811904BF82200D7F8881043F8220098
:10B1D00021F81200D7F88C1021F8120026F812007E
:10B1E0000CF802000EF8020048F82200796A0132D9
:10B1F000A142ACD12C37BD46BDE8F08F0121BA6821
:10B20000386A22F816A03A6916547A68915531E7DF
:10B21000E01600202DE9F04F04469FB00AAFD7F8A2
:10B2200090B0F9620BF1070121F00701ADEB010DC0
:10B230000AA9F960BA6208465A464FF0FF317B60AE
:10B240000DF0BDFBE31D23F00703ADEB030D0DF186
:10B25000280A2246504600210DF0B1FB00229345FA
:10B260007A6452DDBE6FC7F834A004E07A6C013214
:10B270005A457A6447DAD7F8A03033F91230002BF8
:10B28000F4DD0023D7F8D0209C42C7E912237A6C62
:10B2900040F3E0814FF0FF3804E0FB6C0133A34240
:10B2A000FB6424DA36F913100029F6DDF86AB96A6E
:10B2B00031F9131030F91330D7F8980050F82250B4
:10B2C000D7F89400691A50F82200C01A00F090FDD7
:10B2D0004FF4614303FB00F3BA6C1B149A4200F372
:10B2E0008081FB6C7A6C0133A342FB64DADB4FFA9A
:10B2F00088F30121F868835401327B6B5A4503F8C7
:10B3000008107A64B7DBD7F834A0002C40F39E8194
:10B31000D7F87C90013C0AEB04034FF000083B6136
:10B320000AF1FF3AC7F8309008E03B6B08F10108DA
:10B3300002333B633B699A4500F088811AF8013F6C
:10B34000002BF2D0BB6FBBF1000F33F91890FB6AF2
:10B35000C7F8449033F91820BB6A09FB02FE33F9A1
:10B3600018C07B6809FB0CFC33F81810D7F8843040
:10B3700009FB01F113F808303B62D7F8803013F86D
:10B3800008307B62D7F8CC3013F80830FB61D7F86F
:10B39000883053F8285040F361810024724660469B
:10B3A000FB68C7F808A05E1ED7F894A007F14C030D
:10B3B000BB617E637E6B16F9013F43457E6340F0BF
:10B3C000AE80D7F89860D7F8A03056F8246033F9EB
:10B3D00014307E615AF82460994406FB03227E698A
:10B3E000C7F8449006FB0300C7E90E202A46D7F8A9
:10B3F0009C6036F814C003FB0C11D7F8B0305FFA2C
:10B4000085FC53F8243039645FFA83FEC3F30720C8
:10B41000F445C5F3072188BF6EF30702C5F3074C57
:10B420008142C3F3074138BF60F30F221B0E8C45E6
:10B4300088BF61F31742B3EB156F88BF63F31F62D8
:10B4400094465FFA82F9F14588BF6EF3070CC2F3A8
:10B45000072E864538BF60F30F2CC2F307408842A1
:10B4600088BF61F3174C1546B3EB126FD7F8C820AD
:10B4700088BF63F31F6C0992D7F8C42007F13C031F
:10B480000892D7F8C02021460792D7F8BC20069230
:10B49000D7F8B8200592D7F8B0200492BA69039281
:10B4A00007F14402029207F14002CDE90032F86947
:10B4B00007F138035A46C7F84CC0FDF725FCD7F80A
:10B4C0008430396A1A5D00239142B8BF1146D7F81B
:10B4D000A8207E6A3962115D4AF824300E437E62EC
:10B4E000D7F89860BA6B46F82430D7F89C60D7F844
:10B4F000449026F81430D7F8A060F86B26F8143082
:10B50000D7F8A460396C26F81430D7F8A860335502
:10B51000D7F8AC603355D7F8B06046F82430013422
:10B52000A3457FF447AF96468446D7F808A09EFB14
:10B53000F9F69CFBF9FC91FBF9F4D7F8C8300FFA47
:10B5400089F90693D7F8C43007F148010593D7F875
:10B55000C03062460493D7F8BC30F869CDE9025395
:10B56000BB690091019331464B46C7E90E6C3C64C0
:10B57000FFF772FBD7E9120100F03AFC66230122C3
:10B580004FF0000E4FF0020C00B203FB00F3354900
:10B59000386B9B120391038011460346CDE9012EBF
:10B5A000CDF800C07420F7F741F9BB6F23F818906D
:10B5B000FB6A23F81860BB6A23F81840D7F880307C
:10B5C0001A4697F8243002F80830D7F884301A4623
:10B5D00097F8203002F80830D7F8883043F8285020
:10B5E000A3E64FF0000A01254FF0040952461E4918
:10B5F0006D20BB64D7F84C80F7F764F91B4B2A46E3
:10B60000CDE902A3294607F144030195CDF8009046
:10B610006420F7F70BF9164B2A460393294607F1E6
:10B620004C03CDE9015ACDF800906420F7F7FEF8FD
:10B63000104BCDE9015A0393CDF800902A462946D4
:10B6400007F148036420F7F7F1F84AE65437BD469E
:10B65000BDE8F08F4FF0FF3398464AE607F14C0300
:10B66000BB6164E7549901003499010040990100DD
:10B6700044990100489901002DE9F04FB0F1000A0A
:10B6800091B0DDF868B06BDD16460D4600245F46CC
:10B690000D9337F91430002B5FDD4FF0FF3B4FF077
:10B6A0000009DDF89C804C4513D037F91930002B88
:10B6B0000FDD56F8241056F8292055F8240055F8C7
:10B6C0002930891AC01A00F093FB4045BCBF804660
:10B6D000CB4609F10109CA45E5D1BBF1FF3F3CD09A
:10B6E000259B52460A93249B59460993239B204647
:10B6F0000893229B0793219B0693209B05931E9BF7
:10B7000004931D9BCDE902730D9BCDE900632B468D
:10B71000FDF72CFCA34526DD259B1E9837F914C0A8
:10B7200056F8242055F8241050F824000693249B42
:10B7300002900593239B0EA80493229B00900393F1
:10B740000FAB019320466346FFF786FADDE90E0151
:10B7500000F04EFB1B9B23F814000134A24598D146
:10B7600011B0BDE8F08F259B1E9837F91BC056F825
:10B770002B2055F82B1050F82B000693249B029099
:10B780000593239B0EA80493229B009003930FAB79
:10B79000019358466346FFF75FFADDE90E0100F0BA
:10B7A00027FB1B9B23F81B00D7E700BF2DE9F04FB9
:10B7B000B0F1000B83B0DDE913C9DDF86CA0DDF852
:10B7C000748050DD00264FF0FF34DFF8A0E00193D5
:10B7D00002E00136B34546D01EF806000028F8D135
:10B7E000013408EB0400019B02E00134A4453ADD7A
:10B7F000077805460130002FF7D06445019332DA0F
:10B80000159859F8247050F8240021F8167022F881
:10B810001600169830F814701998005D23F8167009
:10B82000179F0C9B37F9147023F81670189B33F987
:10B8300014700D9B23F816700E9B98551A9B185D7B
:10B840000F9B98551C9B28785AF8247033F9145094
:10B85000109B43F82670119B23F81650129B9855A5
:10B860000136B345B8D103B0BDE8F08F8C26002077
:10B870002DE9F04F99464FF01F3304469DB018AFA5
:10B88000C7E90133BB81BB6BCDE90B410E46391DC6
:10B89000D7F840A00F930A91FB6B396FCDE9103AAE
:10B8A00005917B6CF96E12930491BB6CB96E139386
:10B8B0000391FB6C796EDFF8A0E1DFF8A0C114936F
:10B8C0000D92BB6D9046CDF838907A6D0291396E2D
:10B8D0005F480191CDE908CEF96DDFF884C1009190
:10B8E000CDE906C0396D0A20FFF786FB594AD7F823
:10B8F0008C00D2E9023200210092642200F062FA48
:10B90000002860D0BB6F002B5DD0D7F88430002BAF
:10B9100059D083463D1D3B6F1595D7F88850059348
:10B920001495FB6ED7F8845004931395BB6ED7F82B
:10B930008050039312957B6EFD6F029311953B6EC1
:10B94000BD6F01931095FB6DFD6C0093396DD7E9C8
:10B950001523CDE907680694CDF858B00F95BD6C56
:10B960000A200E957D6CCDE90CA5FD6B0B95BD6B8A
:10B97000CDE90995FFF74EFCD7F88C301BB30023B7
:10B980003A1D0C92D7F8882006930B92D7F88420A2
:10B990004B460A92D7F8802031460992FA6F20462A
:10B9A0000892BA6FCDF834B00792FA6C0592BA6C6F
:10B9B00004927A6CCDE902A2FA6B0192BA6B009202
:10B9C0004246FFF759FEE31D23F00703ADEB030DDD
:10B9D000002C0DF1600C11DDBB6B0DF15F011D46FC
:10B9E0009A1E02EB440032F9023F002BD4BF002321
:10B9F0000123824201F8013FF5D1BD63FB6B07943F
:10BA00000C93BB6BFC6CCDE90A937B6F109406938F
:10BA10003B6FBC6C0593FB6E0F940493BB6E7C6C08
:10BA200003937B6E396D02933B6E0A200193FB6D8D
:10BA3000CDF844C00093D7E91523CDF834A0CDE963
:10BA400008680E94FFF7B2FE1437BD46BDE8F08FCC
:10BA50000C1D0020E0160020901C0020201D00205E
:10BA60008C2600202DE9F04F4FF0000883B082466D
:10BA70008946019344460F9D574E584ADFF878B1E6
:10BA80002BE000232354002963D13AF91430544F9A
:10BA900022F8143039F91400524927F814003AF901
:10BAA0001400514B2BF8140039F91400371921F800
:10BAB00014000199287831F9141023F814100E9B02
:10BAC00033F91410494B387023F8141008F10108A9
:10BAD00001340A2C05F1010537D02B78311900917A
:10BAE0004348315D002BCCD14148DFF8F8C0DFF886
:10BAF0000CE10029ECD0215C3BF81470013149B213
:10BB0000DEF800E0215422F814703CF81400344FA1
:10BB1000714527F81400DBDD31192CF81430354855
:10BB2000DFF8C4C00B70314922F8143027F8143004
:10BB30002BF8143020F814302CF8143021F814307D
:10BB400001340A2C05F10105C7D1404603B0BDE818
:10BB5000F08F234F32F9143039F914C037F914102B
:10BB60003AF91400ACEB0101C01A009200F040F960
:10BB7000204B3BF914C023F814003AF91430009A12
:10BB8000A3EB0C0C174903EB6C0322F8143039F9C2
:10BB9000143031F914C01448A3EB0C0C03EB6C0304
:10BBA00027F814303AF9143095F800C02BF8143007
:10BBB00039F9143021F81430019B311933F914305C
:10BBC00081F800C020F814300E9B33F91410074B95
:10BBD00023F814107AE700BF8C2600200C1D0020EB
:10BBE000201D0020F81C0020D01C0020BC1C0020C0
:10BBF000A41C0020901C0020E41C0020E016002063
:10BC00002DE9F04F4FF0000983B0CDE900129846BE
:10BC10005F4D604B824695E8070003C34C460E9E7D
:10BC2000DFF89CB11A803BE000215A4F9E42DFF8BA
:10BC300080E1DFF884C15848584A395565DB3AF944
:10BC40001430574FA15CEB53009B564F33F914301F
:10BC5000EB533AF91430544F25F80B30009B33F96D
:10BC6000143025F80E30019B33F914E04F4B25F8C2
:10BC70000CE038F914C027F805C00C9F17F804C071
:10BC800004F800C0385D814238BF0146A1540D9AC6
:10BC900032F91420EA5209F1010901340A2C30D09A
:10BCA00038F91420404BB2424FEA440533F91430BE
:10BCB000BADC9E423E4A3F49EFDA364F35F80B0078
:10BCC0003B5D096801335BB23B55354F35F802C027
:10BCD000E85334488B4225F800C0DEDD00233649A6
:10BCE000AB526B522C4A2D492B52A3542E482F4A4B
:10BCF000635401340A2C25F80B30EB534353AB52F9
:10BD0000CED1484603B0BDE8F08F264B009FEA5ED7
:10BD1000234B37F91410EB5E3AF91400891AC01A54
:10BD200000F066F8254B35F90B1058533AF91430EA
:10BD30001F4A591A03EB61031949A85E6B5237F980
:10BD400014301D49181A03EB600316482B523AF9B8
:10BD50001430114825F80B3037F91430124FAB521C
:10BD6000019B0E4A33F914306B5238F91410A35C5E
:10BD700079530C99095D21540C99085D0B49834254
:10BD800038BF0346A3540D9B33F914306B5282E73E
:10BD9000A41C0020B01C00200828002080250020C2
:10BDA000CC2D0020102600204C27002068250020E4
:10BDB000E42D0020E0160020F82D0020901C00202B
:10BDC000DC270020884210DB904210B40ADA441AC3
:10BDD0000198521AC01A04FB00F494FBF2F210BC52
:10BDE000D0187047019810BC70471846704700BFC4
:10BDF00081EAE173A3EBE17318B30028B8BF4042B6
:10BE0000F1B198421FDA820192FBF3F2402AA8BFF7
:10BE1000402211498A5CC2F15A028AB10F4910B41A
:10BE2000C2F15A0431F8122031F8141003FB02F366
:10BE300000FB01F01B1403EB2043184610BC7047B5
:10BE40000346184670479A0192FBF0F2402AA8BFB9
:10BE5000402201498A5CE0E7389A01007C9A01009F
:10BE600088420ADB40B1890191FBF0F04028A8BF6D
:10BE70004020094B185C7047704751B1800190FB1E
:10BE8000F1F14029A8BF4021034B595CC1F15A0090
:10BE900070470846704700BF389A010070B40E68BA
:10BEA0000C89022E25DDA04223DB0B460125013E35
:10BEB00002E0844206DC15466A1C96429C8903F126
:10BEC0000403F6D101EB8505AE88ED88A6420DD0BE
:10BED00001EB8201CB88001B5D1B00FB05F0A41B5E
:10BEE00090FBF4F41C4420B270BC704728B270BCC4
:10BEF000704700250122E5E77F280CDC402824DA82
:10BF00000F2824DC082827DA022829DB0428B4BFFC
:10BF1000012002207047B0F5806F08DAB0F5007F8D
:10BF20001CDAB0F5807FB4BF072008207047B0F559
:10BF3000805F05DAB0F5006FACBF0B200A207047B8
:10BF4000B0F5005F0CDA0C207047062070472028FF
:10BF5000B4BF0420052070470320704709207047B4
:10BF6000002070472DE9F04F056887B0144665B191
:10BF70002C4E2D4D314600226020F6F7A3FC2246C0
:10BF800029466420F6F79EFCF4E7284A0746136822
:10BF900008460133884613600CF0F6FC386020B187
:10BFA000234B00EB08029A422CD90025DFF888B019
:10BFB000DFF888A0DFF88890494600226420F6F771
:10BFC00081FC042601223868114600EB080C04AB02
:10BFD0000490CDE9025B019500966420CDF814C071
:10BFE000F6F724FC012200961146CDE9025A01958C
:10BFF00005AB6420F6F71AFC002221466420F6F710
:10C0000061FCD9E70B4A2B46114602E00133322B83
:10C0100005D051F8044B002CF8D142F8230007B0AA
:10C02000BDE8F08FE8990100EC990100FC1D0020AB
:10C03000F83A0020341D0020209A01002C9A0100BB
:10C040000C9A01002DE9F04D0746006886B088463D
:10C05000B8B1244D00232A4602E00133322B18D018
:10C0600052F8041B8142F8D1002445F823400CF01B
:10C0700093FC1D4A3C601368013B136006B0BDE8A9
:10C08000F08D0A4664201949F6F71CFC06B0BDE89D
:10C09000F08D0024DFF85CB0DFF85CA0144E314670
:10C0A00000226420F6F70EFC042501223B681146AD
:10C0B0000593CDE9024B05ABCDE900546420F6F7BA
:10C0C000B5FB414600226420F6F7FCFB0A220095EE
:10C0D000CDE9024A01941146024B0020F6F7A6FB77
:10C0E000DDE700BF341D0020FC1D00208C990100FD
:10C0F000AC990100309A0100D49901000D4B1B68E6
:10C10000002B15DD70B500260B4D0C4C84B021467C
:10C1100000226420F6F7D6FB01220423CDE9026554
:10C12000009301921146034B6420F6F77FFBEEE784
:10C13000704700BFFC1D0020509B0100349B010094
:10C1400010B50446FCF78CFD04F1F00104F1B800D1
:10C15000FEF76AFC04F59470FBF7A4FA04F5EC70A2
:10C16000FAF7C0FE04F5EE70FEF750FB04F5F87028
:10C17000FCF72AF804F51770FEF7D0FD04F52670D9
:10C18000FEF79CFE04F52A70FCF764FD04F2813092
:10C1900002F0A2F804F2AE20FCF7B6F894F8AE3242
:10C1A0000BB9FCF7B7F804F52C70FBF759FE04F552
:10C1B0004170FBF7A7F804F55E70FEF78DFA04F501
:10C1C000617001F02DF80023044C194623604FF4F0
:10C1D0007072BDE8104002480CF0F1BB001900205D
:10C1E000FC29002038B9064A136801338B4205DD6B
:10C1F00010600120704700231846014A1360704701
:10C200000019002008B5FAF7F1FEFEF76DFAFEF707
:10C2100061FEFCF77FF8FBF72BFEFBF77BF8BDE830
:10C22000084002F051B800BF0022014B1A6070476D
:10C23000001E0020024A136801331360704700BFDC
:10C24000001E0020014B1868704700BF001E002030
:10C250002DE9F04F0024DDE90A57A246A046A14689
:10C2600040F6FD7EDDF830C0013D15F8016FBEB12E
:10C2700031F814B0ABF5007BBBF5406F10D232F84B
:10C2800014B00BF1FF3B1FFA8BFBF34508D833F9D1
:10C290001490C14556DDC846B146099E36F914A032
:10C2A00001340A2CE1D100263546A7F1020E07F22F
:10C2B000BE377146002205E0262B00D90135013238
:10C2C000202A0AD031F8023F062A03F113039BB259
:10C2D000F2DC262BF3D90136F0E70EF1400E77455C
:10C2E000E7D10027ACF102030CF10A0C33F9022F5D
:10C2F0009C451744FAD100220D9B0D99023301F1A0
:10C30000180C33F9021F9C450A44FAD143F2B0637A
:10C310000E994968994211D89F2D0FDC452E0DDCEE
:10C32000C0B1B9F1000F0FD0B8EBEA0F0CDD104A25
:10C330001368032B03DC0133136000E00B24204659
:10C34000BDE8F08FB146ABE70022094B20461A60EA
:10C35000BDE8F08F952F02DD962AA8BF0B24044B71
:10C360001A68002AEBD0002220461A60BDE8F08F40
:10C37000181E0020024B0A201978FEF7E1B800BF12
:10C38000C8080020002001220249034B08601A70EF
:10C39000704700BF0C1E0020041E0020014B1878BF
:10C3A000704700BF041E002019B10E4B1860FFF744
:10C3B000E1BF0C4B30B41C680B4D84422A680DD091
:10C3C0000A2C14BF28210021914203DD01322A608A
:10C3D00030BC704730BC1860FFF7CCBF02B1296099
:10C3E00030BC7047C8080020081E002070B586B019
:10C3F0000C9CDDE90A56029401960F9C0E9E009556
:10C400000D9DCDE9046403950E4D2C68FFF720FFC8
:10C4100001210D4AE31782FB0462C3EBA20303EB85
:10C4200083030A4AA4EB430301FA03F311680A28C1
:10C4300014BF0B4321EA0303013413602C6006B0E0
:10C4400070BD00BF0C1E002067666666141E0020CB
:10C45000034B18680028D4BF00200120704700BF9C
:10C46000141E00202DE9F04FDFF84CA187B09AF898
:10C470000040169E002C35D0B42404FB06F4484D31
:10C48000DFF8388185FB045BE417D8F80050C4EB73
:10C49000AB14AC4249DA434C074624688C460A2C5C
:10C4A0009646994621D14FEA460B0BEB0604A5426E
:10C4B0001BDB06EB8606B5EB860F3B4E02DA3468D3
:10C4C000A3454ADC0021394B39481A6801238A42C6
:10C4D000D4BF00220122013502708AF80010C8F88A
:10C4E0000050336007B0BDE8F08F159B614605939F
:10C4F000149B72460493139B38460393129B2A4E57
:10C500000293119B0193109B00934B46FFF7A0FEF3
:10C510000021FFF749FF0123D8F800500135C8F882
:10C520000050336007B0BDE8F08F159E0596149E4D
:10C530000496139E0396129E0296119E0196109EDB
:10C540000096FFF785FE1B4AAC42136840EA0300E1
:10C5500010601ED00123144EE0E7159C0594149C36
:10C560000494139C0394129C0294119C0194109CBB
:10C570000094FFF76DFE0B2808BF00234FF0000169
:10C5800008BF3360FFF710FF3368D8F8005001335D
:10C59000C4E7044B1860FFF7EDFED8F80050D9E768
:10C5A000D34D6210C8080020101E0020141E002069
:10C5B000051E0020CC080020041E00200C1E0020B8
:10C5C000014B1878704700BF051E002038B50D4C90
:10C5D00030B123680A2B03D00A232360FFF7CAFE79
:10C5E00000230A220849094D0B60094809492B60BC
:10C5F00003600B60084D094809492B7003702260E5
:10C600000A6038BDC8080020081E0020141E002043
:10C61000101E00200C1E0020051E0020041E0020FD
:10C62000CC0800206E20704738B500240B4B0C4D11
:10C6300021464FF42072C3E90044C3E90244C3E930
:10C64000044408482C600CF0BAF92146BDE8384093
:10C650004FF4967204480CF0B2B900BFF0210020EC
:10C66000241E0020281E0020A82000202DE9F04FC5
:10C6700000261F460C4693B00DF128080DF118094D
:10C68000824615463146202240460696C9E9016693
:10C69000C9F80B600CF093F9BB104A4A142BB8BFD1
:10C6A0001423B442C2E90066C2E9026616616CDD79
:10C6B0004F46CAEBCA714900CDE901664FEA4A0C00
:10C6C0000091611E0596049605EB0C0209EB040E21
:10C6D0000391BAF1000F16DD00210098A7EB090BBA
:10C6E000101830F9024B9C4207DD3E7811F80850D3
:10C6F000013601353E7001F808501F2937DD9042A0
:10C7000001F10101EDD1013777456244E1D1019B8F
:10C71000002B52D1059A9DF828609DF81830002A08
:10C7200047D1002528462F4629460DF119020DF163
:10C7300027040BB1012528448B42C4BF19460127A9
:10C74000944202D012F8013BF3E77FBB5DBB0021AE
:10C750000B460DF12D020EB101210B44904502D084
:10C7600018F8016FF7E7D9B913B0BDE8F08F029D53
:10C77000BBF1000F2544029504DD039D5D4501DDFD
:10C78000052904DD01240194B9E73346C9E7049E75
:10C790000125A642B8BF2646059504960195AEE749
:10C7A000084A9360E0E7074B1860D0E7054B5960F3
:10C7B000CCE7044A04991161B3E7024B029ADA60AC
:10C7C000A8E700BFD42100202DE9F04F95B000AFBD
:10C7D0007B61D7F894300028BB60D7F89830C7E960
:10C7E0000621D7E91ECED7E92C51D7F8B8407B6097
:10C7F0007862386240F37D81C54EC64B30689946F9
:10C8000003EB8013786A023A4000F860023B02EBC7
:10C81000000832F9020F904523F8020FF9D123687E
:10C820003B61FB69002B19DD7B693268A3F10208CB
:10C830004346B948C2EB021200EB4202F869023AE1
:10C8400008EB400633F9020FB34222F8020FF9D188
:10C850003B6A002B40F36E81AE4B99460022C7F82D
:10C86000B84047F6FF764C46C7F8B410DFF8C082F0
:10C87000B9697A6200234FEA420B786A04EB0B092C
:10C88000C34439F940ABCB455344FAD18246786270
:10C89000A24880FB0309DB17C3EBA9031BB2002BE3
:10C8A00021F81230994602DD5046184478629E42C3
:10C8B000A8BF1E469C450CDAB5F808902B6809F114
:10C8C0000109A5F8089031F91290A9EB0C0A53441C
:10C8D0002B60CE450CDDB5F80A906B6809F10109B3
:10C8E000A5F80A9031F91290A9EB0E094B446B6040
:10C8F000022A40F32E813B6A01329342BADCD7E927
:10C900002D143A69AE811546854B786A83FB055331
:10C91000A3EBE2732360E3683A6A3B61FB6990FB37
:10C92000F2F0002B40F3EF807B69A3F102086FF077
:10C9300001054FF0000E47F6FF7CFB69464603EB0E
:10C940000508C7F82480744AD7F80490D7F80880FF
:10C9500078611046002302F5967B30F91EAB8345C3
:10C960005344FAD16D4880FB03A0DB17C3EBA0034F
:10C970001BB29E45B8BF9E469C45A8BF9C464345FA
:10C9800026F8023F09DD0B89086801330B81B6F9EF
:10C990000030A3EB080A50440860994509DD4B8933
:10C9A000486801334B81B6F90030A3EB090A5044C3
:10C9B00048600A2D23EAE37000F291803B6901355B
:10C9C00003443B61E3607B6A0232AB42C1D17869C8
:10C9D0000FFA8EFE0FFA8CFCFD68A1F80EC02B46F4
:10C9E000083323F00703ADEB030DFB69A1F80CE05E
:10C9F000A3F1040C3B6A6946002B38DDBB690026B5
:10CA00009A1E154440F24458A946A1F1020E32F98B
:10CA100002AF256AAAEB000323EAE3731BB2AAF173
:10CA2000970AAB421FFA8AFAC8BFC4E90763C24536
:10CA30002EF8023F06F1010602D8A3690133A36173
:10CA40009145E4D1B1F90030002B10DDA36A3A6AB8
:10CA50001A441046013304E031F9022F002A40F352
:10CA60009B8098421D4603F10103F5D1A06247F671
:10CA7000FF703B690326984293FBFCF1B8BF184650
:10CA80000023284AC7E90E33C7E91033C7E9123338
:10CA9000254D264BA16000B207F12801C7E90C2300
:10CAA000C7E90A65FFF7FAF9E2686369012A1146E6
:10CAB000B8BF01219B0193FBF1F323EAE373984292
:10CAC00009DAE369B34206DD41F287339A4202DCB8
:10CAD000012384F824305437BD46BDE8F08F6369E4
:10CAE0000135034463617B6A0232AB427FF431AFAC
:10CAF0006DE723683B61FB69002B3BDD3B6A044E1D
:10CB00005B00FB6090E647F6FF7C4FF0000E63E7AA
:10CB1000241E0020281E0020A820002067666666CC
:10CB200056555555E8034000F4013200D007400047
:10CB3000A820002047F6FF72AA813A69174B1046D9
:10CB400083FB0003A3EBE2732360E36800203B61F7
:10CB5000EDE631F912903869D7F8B830B9F1000F25
:10CB6000A8BF48445B6838619944D7F8B830C3E936
:10CB70000009C0E647F6FF70FA69084BA2F1040C01
:10CB80003A69A88183FB0263E068A3EBE273044A7D
:10CB900023603861CA606AE7A56268E75655555553
:10CBA0000000FF7F0020A2F1040C2DE9F047E046D1
:10CBB000064647F6FF77DFF858E1DFF858918D1EFB
:10CBC000106050609060D0601061043135F9023F10
:10CBD000002B3ADD98B2441E092C39D81C461E445D
:10CBE0009E45B8BF9E469F42A8BF1F468D4248F84B
:10CBF000044FEBD14348BEF57A7FC1791CDA012F8F
:10CC00003B46B8BF01231BB29EFBF3F3052B13DD9C
:10CC100091B93D4D0E4602F108015CF8043F312BFD
:10CC200006DD85FB0374DB17C3EBA403CCF80030EF
:10CC300061451E44F1D1C179344B116183FB061368
:10CC4000A3EBE673D360BDE8F08700242346C7E773
:10CC5000A0F10B04092C11D9A0F1150ABAF1090FA2
:10CC60001C4612D803EB43035B00A9FB0303DB085C
:10CC700003339BB21C461BB22644B1E75B1005335D
:10CC800098B2044603B20644AAE7A0F11F0ABAF11B
:10CC9000090F0ED9A0F1290ABAF1090F11D8DB004A
:10CCA000A9FB0303DB08043B9BB21C461BB22644D2
:10CCB00096E7C3EBC303A9FB0334E408264423B27D
:10CCC0008EE7A0F1330ABAF1090F04D93D382728BD
:10CCD0000CD91E4484E703EBC303A9FB0303DB0861
:10CCE000093B9BB21C461BB2264479E7C3EBC30346
:10CCF0005B00A9FB0303DB08263B9BB21C461BB26F
:10CD000026446DE7F0210020676666665655555546
:10CD10000080FFFFCDCCCCCC84B02DE9F0470024BF
:10CD2000814609A880E80E003D4D9DF848603D4FC2
:10CD3000DFF81481DFF814A115F8013BABB90F9BA4
:10CD4000122B02DCB9F1000F28D00EB300223649B5
:10CD50004920F5F7B7FD002305F8053C0134042C04
:10CD6000EAD1BDE8F04704B0704707EB4403099AE5
:10CD70001B899A424FF0000202DD0B9B1E2B29DC1F
:10CD800041464920F5F79EFD002305F8053CE5E7FF
:10CD9000324626494920F5F795FDDFE74A46244902
:10CDA0004920F5F78FFD109B062BD7DD7EBB0E9B30
:10CDB000B3F57A7F25DD139B052B22DC119BB3F5A0
:10CDC000FA7F1EDA32461B494920F5F77BFD05F84C
:10CDD000056CC3E751464920F5F774FD012305F8BA
:10CDE000053C46B1002214494920F5F76BFD0023AC
:10CDF00005F8053CB2E7324610494920F5F762FDD7
:10CE0000ACE700220E494920F5F75CFDA6E74A464B
:10CE10000C494920F5F756FD05F8059C9EE700BF33
:10CE2000F4210020609B0100349C0100709C0100F3
:10CE3000889B0100D89B0100C09C0100F09C010070
:10CE4000FC9B0100B09B0100009D0100A49C01001F
:10CE500082B010B401A981E80C00DDE90234012B95
:10CE600018D0A0B1511001EB4201994202DCD11E51
:10CE7000032907D9023B032B09D8012C07DD023A0D
:10CE8000042A04D80022074B5A709A70DA7010BC3A
:10CE900002B07047042AE4DC0022024B5A709A70F8
:10CEA000DA70F4E7F021002030B400250124104BA3
:10CEB000181D1A7919786AB979B1597A0131C9B24C
:10CEC0000A29597201D91C715A7201338342F0D177
:10CED00030BC704719B15D73F7E75972F5E75A7BBB
:10CEE0000132D2B20A2A5A7384BF19715973ECE71E
:10CEF000F021002084B030B49DF8484002AD85E8B0
:10CF00000F00002C2FD0109BB3F5FA5F14DD2A49D7
:10CF10000B680133052B34DD052301220B60002350
:10CF20000120264D264C27492B602360264B087094
:10CF300030BC1A7204B07047119B642BE7DC214BA4
:10CF40001B780BB3204B1E490A6801320B2A2EDCDA
:10CF50000A6002220021184C18482160016030BC90
:10CF60001A7204B07047154A154B146002221C60F7
:10CF700014481149144B04700C601A7230BC04B090
:10CF800070470B600222CAE70F4B9979DA790A439E
:10CF9000D9D00A4908480A680132052AC8BF0522C3
:10CFA0000A600022064902600A600222C0E70B20E4
:10CFB00000220860CEE700BFE82100200822002000
:10CFC0001C1E0020EC210020F021002000212DE972
:10CFD000F0473B4F92463A46994601250B468EB0A4
:10CFE0009DF8A080189E1A9C364842F8041B12F83F
:10CFF000011B31B930F813108E4202DD1E2CC8BF60
:10D00000FD540133042BF2D16C461BAD0FCD0FC480
:10D0100095E80F0084E80F0018AD95E80E0048462B
:10D02000FFF77AFE25AB93E807008DE8070023ACF5
:10D0300094E80C0049465046FFF70AFF00234FF0E2
:10D04000010C42F2107026994BB3032B32D05A1CBC
:10D05000042A01D00133F7E740F2DC539E4206DC9C
:10D0600043F698239942CCBF01230023BB706E4640
:10D0700007AFFFF719FF0FCCCDF830800FC723683B
:10D080001CAC3B600FCC0FC694E8070086E8070095
:10D0900095E80F00FFF72EFF0EB0BDE8F08797F878
:10D0A00000E00122BEF1000FD4D18142C8BF07F8D1
:10D0B00003C0CDE7FA78002ACED10422F5E700BFFD
:10D0C000F0210020609B0100034B187AA0F10100C1
:10D0D000B0FA80F040097047F021002020B90C4BD5
:10D0E0009A7952B10320704701280FD1084B1B7A5F
:10D0F000002B14BF0420052070475A790AB1022082
:10D1000070471879003018BF012070470020704721
:10D11000F02100202DE9F04FA3B00025DDE93C8788
:10D120006E4681468B4617AC149220462C22002175
:10D130009DF800A115930BF042FCCDE90F74CDF8DA
:10D1400038800DF1D40C0DF11C0EBCE80F00AEE8D8
:10D150000F009CE807008EE807000DF1B80CBCE852
:10D160000F00C8F80050C8F80450C8F80850C8F8B4
:10D170000C50C8F810503D607D60BD60FD603D61A1
:10D180000FC69CE807002D9B86E8070059462C9A9D
:10D190004846194EFFF718FB0DAFCDF848A00FCE4B
:10D1A0000FC736680FCC3E6002AE0FC60FCC0FC65D
:10D1B00094E80700159B86E807002D990F4C019114
:10D1C0002C99149A009148465946FFF7FFFE2368B0
:10D1D0002C9901330A2B18BF1D4648463E9A2560FC
:10D1E000FFF7E0FC3E9B3F9ADB6850469382FFF7D7
:10D1F00075FF23B0BDE8F08FD4210020241E00204D
:10D2000030B9064B187810B10138C0B218707047A9
:10D210001423024A18461370704700BF201E0020D6
:10D2200001464FF4A67201480BF0BEBBF016002079
:10D23000014B1878704700BF312200202DE9F04FD4
:10D240000026B7B0CDE90A23884B894C1E70894D62
:10D25000894B8A4A8A4926608246499C0CA81E60EE
:10D260002E6016600E60FCF74BFD3146802216A83A
:10D270000BF0A5FB04F10E0009902F68B346304671
:10D280001F257D4B7D4A7A4C1268D3F800807D4B78
:10D290007B49059293F902302268CDE90666D1F800
:10D2A00000E00896049202930DF1D409764B4FEA00
:10D2B000450C03EB0C02A3F570739C44CDF804C03D
:10D2C000099C84461DE04FF0010B9E44D844CDF8E4
:10D2D00018B0052DA2F140020FD00298591D8342CB
:10D2E0000BDA20780CF1010C0390D9F8000001440E
:10D2F0000398C9F800101F2817D0019B013C9A42DF
:10D300001DD0B2F98033534504BF2F4601260B2BA5
:10D31000D9DC13F10B0FDCDA0120079005980130FE
:10D320000590049818440490D3E748980028E4DD59
:10D330000898013C1844019B08909A42E1D1013DB4
:10D340006B1C6046A9F10409B0D1079B002B78D172
:10D35000069B13B1484BC3F80080BBF1000F02D00D
:10D36000474BC3F800E00EB1424B1F60454B2022F3
:10D370009988B3F90660B3F90840409F1F2314E071
:10D3800007EB4202B2F854205AB18A4209D236AAB7
:10D3900002EB830252F8802CB24202DA089AA242CF
:10D3A00012DC5D1E8BB11A462B46052BE8D1B7F86F
:10D3B0005E30002B4CD08B424AD21A9B9E4247DDF6
:10D3C000089A0423A242ECDD01230A9AB2F57A6F8F
:10D3D0004AD9409A118B5A2994BF0021012140F269
:10D3E000EE22409C248E94423CD9409CB4F84A40A2
:10D3F000944294BF00220122012B2CD1409C248B0B
:10D40000142C28D91E2826DD0B98052823DD11BBF6
:10D410000ABB9DF8361001F0FF00E1B919491B4C19
:10D420000D784A9E216835448D42D8BF18460F4E6C
:10D43000C8BF01313370CCBF2160226037B0BDE876
:10D44000F08F0E4B059A1A60094B049A1A607FE719
:10D4500004230325A7E7002318460C4A136037B0BE
:10D46000BDE8F08F0022C7E70021B8E718220020AE
:10D47000202200202C220020242200201C22002018
:10D4800028220020F0160020FC2900200C22002079
:10D49000F0B58DB0BDF954509DF890609DF8947032
:10D4A000C0B9B9B93D4C2178C9B1132A55DC139ADA
:10D4B000632A52DC133350DB129B092B4DD8384BB7
:10D4C000384AD9691368994260DD01210B44136021
:10D4D000217024E00022314B1A700DB0F0BD239969
:10D4E000104609912199CDE90A6708912099079181
:10D4F0001F9906911D9905911C99CDE903511B991E
:10D5000002911A9901911E9900911946DDE91223A1
:10D51000FFF794FE207010B12348F9F7E3FCFCF705
:10D52000ABFE2478054624B3204C214E2388327864
:10D5300001331BB22380002ACFD1632BCDDD1D4BDD
:10D540001B78002BC9D002210920FCF7F9FF012329
:10D550006422AB7733702280BFE7114B1399B3F984
:10D5600018209142ACDC002201210E4B21701A6080
:10D57000D5E70F4E0D4A33781480002BADD0032130
:10D580000920FCF7DDFFAC773470A6E700230A48DA
:10D5900013602370F9F7A6FCC1E700BF3122002019
:10D5A000F01600201422002004C7010032220020BF
:10D5B000302200201822002008C50100054A92F8F8
:10D5C0004E30834204DA8B42B4BF00200120704702
:10D5D00001207047F01600203228CCBF0020012027
:10D5E000704700BF2DE9F04F95B00393BDF980302F
:10D5F00005460193BDF984300C460693FCF730FED6
:10D60000012801D0002D48D000231F259E469A46B0
:10D610009946184619461F4698469C46C24ADFF866
:10D620002CB31360C14AC24E1360C24ACBF800301B
:10D630001360C14A136006F5707207E04FF00108ED
:10D640000CF1010C1F44403A964211D0B2F98033DC
:10D65000A34204BF294601200B2BEFDC13F10B0F73
:10D66000F1DA4FF0010A403A9642D1449E44EDD19E
:10D67000013D6B1CA6F10206DDD1B8F1000F40F0B0
:10D68000D881002840F0DA81BAF1000F05D0A74B0D
:10D69000C3F80090A84BC3F800E0039890F8292045
:10D6A00090F8281090F82B30891A02EB610B5A463B
:10D6B000032AA8BF0322049190F82A1052B2C91A73
:10D6C00003EB6109B9F11E0F059100F3AB80BBF1CB
:10D6D0000C0F00F3B380B9F1020F4FF0030300F316
:10D6E0000C8101211F465A450BF1FF300BF1010659
:10D6F00040F3B080002302933C2C06DD019B292BD4
:10D7000003DC069B292B40F323810023019300298E
:10D710000CBF04230323B042069300F3028109EBFC
:10D720004B18C24603200025DFF81CC209F1FF3E5A
:10D7300009F10107BE450EDC0322804BA8EB401126
:10D740003CF91A6003EB410131F9023B013AA3EBCA
:10D7500006031D44F8D10138ECD16F423FB202F00C
:10D76000B9FB072809DD039AB2F924301146772B5B
:10D7700003DC136A142B00F22681002624220021E8
:10D780000BA80BF01CF9642240F2B6334FF4617120
:10D790004FF4C87E4FF4167C3846ADF82E20ADF815
:10D7A0003020ADF83E304FF4AF72ADF842304FF05C
:10D7B000C80A40F2592340F28A280627ADF83A10E9
:10D7C0000AA9ADF840300A97ADF832A0ADF8342080
:10D7D000ADF83680ADF838E0ADF83CC0FEF75EFB42
:10D7E000574BB3F90A30A3420BDAD12C09DC1E9B4C
:10D7F00033F91930312B00F3DB80059A062A40F209
:10D80000F680019B13B9002E00F085804D4A2299C5
:10D8100013688B4278DB012600233046136015B075
:10D82000BDE8F08FC9F11F07BBF10C0F7FB25FDCC1
:10D83000032F00F0F6800323012154E7CBF10E0300
:10D84000B9F1020F5BB258DC032701210BF1FF3065
:10D850000BF10106C3F10F055D457FF74BAFB9F141
:10D86000030FCC46A8BF4FF0030CCC453FF742AFA7
:10D87000C7F120054D457FF73DAFABEB02025B449E
:10D880009A423FF737AF002502952F4D4F440133A1
:10D890000897A9EB0C08079307F1010C05EB82151B
:10D8A00009F1FF3709F1010A089B434519DB43469B
:10D8B00009910CE09A450CDB35F913E01EF1090FD4
:10D8C00002DA0299013102910133634508D0BB426B
:10D8D000F0DA8242F8DBB242EEDD01336345F6D185
:10D8E0000999079B01329A4205F14005DCD103E713
:10D8F000CBF10E03032F5BB2A7D1BBF1020F00F3F4
:10D900008A8003270121EEE60026304601331360AA
:10D9100015B0BDE8F08F30460A4B1E6015B0BDE86B
:10D92000F08F00273D461AE72C2200201C22002001
:10D930007A26002028220020202200207A2A002097
:10D94000BC0D002010220020FC29002024220020F1
:10D950003C4B1E9A1B6832F91330012BB8BF0123D0
:10D9600094FBF3F3022B7FF7D0AE374B374D1B6898
:10D97000C3EB431203EB820385FB0325344ADB1719
:10D98000C3EB6513126802339342FFF6BEAE314B10
:10D99000314D1B682D68002BB8BF5B42B5EB430FC0
:10D9A000BFF6B3AE092AD4BF002301230193AEE62C
:10D9B0001F9A32F91B20272A3FF723AF059A062A20
:10D9C0003FF61FAF13E0536992686433B3EB520F15
:10D9D0007FF6D3AECB8B502B7FF6CFAE40F6B7336E
:10D9E0001D4A16689E42CCBF00260126C6E6049A50
:10D9F000062A3FF606AF029A06998A42FFF601AF61
:10DA0000643504DA039A52688242FFF4FFAE002BB9
:10DA10003FF7F7AEFAE60322991A18BF012117461D
:10DA200061E6BBF1020FCABF002101213A463B4625
:10DA300059E6094BCBF800C01F6022E6014B196084
:10DA400022E600BF2C2200201C2200201F85EB5163
:10DA50002422002020220020282200202DE9F04F3F
:10DA6000013883B0002801916CDD012872D04FF09D
:10DA700000094FF0010C09EB000303EBD3735B10BB
:10DA800032F9131032F910404500A14204DD22F8AA
:10DA900013400C4622F8101032F919104FEA490BC6
:10DAA000A14202EB0B0A04DD22F81940515332F96E
:10DAB000191032F913408C4205DD22F8131022F8B8
:10DAC0000B4032F9134006460BF10201555E02EBA2
:10DAD0004C0E22F81350545232F90B503EF9028F7B
:10DAE0000CF1010CA845F9DB711E02EB410301E0CA
:10DAF0000E4601391F4633F90249AC42F8DC8C4529
:10DB000007DCAEF80040A7F800800E46BAF90050D6
:10DB1000E4E7019B22F80B408B423D8018DBE14695
:10DB200016DD48450EDD09F1010C8445A3D102EB59
:10DB300049094000B9F90030115E8B42C4BFA9F811
:10DB400000101352019B32F9130003B0BDE8F08FAF
:10DB5000B01EE6E791460220ECE700BF2DE9F04F4A
:10DB6000013800EBD07383B05B10002801936CDDAB
:10DB7000012872D04FF000094FF0010C09EB0003AF
:10DB800003EBD3735B1031F9132031F910404500DA
:10DB9000A24204DD21F81340144621F8102031F987
:10DBA00019204FEA490BA24201EB0B0A04DD21F8D0
:10DBB00019404A5331F9192031F91340944205DDD7
:10DBC00021F8132021F80B4031F9134006460BF1E0
:10DBD00002028D5E01EB4C0E21F813508C5231F98C
:10DBE0000B503EF9028F0CF1010CA845F9DB721EB7
:10DBF00001EB420301E01646013A1F4633F90249A0
:10DC0000AC42F8DC944507DCAEF80040A7F8008091
:10DC10001646BAF90050E4E7019B21F80B40934205
:10DC20003D8018DBE14616DD48450EDD09F1010CAB
:10DC30008445A3D101EB49094000B9F900300A5EDF
:10DC40009342C4BFA9F800200B52019B31F9130085
:10DC500003B0BDE8F08FB01EE6E789460220ECE78E
:10DC6000831A042B10B413DDDC1EB1F90430002A32
:10DC70000B804B8031F9143008DD4000A0EB4202EC
:10DC80000A44014421F8023D8A42FBD110BC70478E
:10DC90005C1E032C08BF9C1EE7E700BFF0B40446DF
:10DCA000049E0846DDE90551A642DDF81CC019DDD9
:10DCB00004F10044AF1E013C07EB460705EB4405A9
:10DCC0008E1C06E09C42B8BF1C46BD4226F8024F9F
:10DCD00008D035F9024F9442F4DD1446BD4226F8CF
:10DCE000024FF6D1F0BC6246FFF7BABFF0B400288D
:10DCF0000F46DDE90561DDF81CC014DB013006EBE1
:10DD000040048D1C06E09842B8BF1846B44225F87E
:10DD1000020F08D034F9020D9042F4DD1046B442EF
:10DD200025F8020FF6D13846F0BC6246FFF798BFDF
:10DD30002DE9F043B1F9009002284FEA4918DDE9D6
:10DD40000767C2E90088DDE909CE21DD8C1E5B0191
:10DD500076017F01043204EB4000023103E0A84663
:10DD600031F9029C0432B1F90050B1F9024006FBCE
:10DD700005F503FB0454156802310CFB054407FB51
:10DD8000094408FB0E4481424FEAA4245460E6D1C2
:10DD9000BDE8F0832DE9F041884684B04C0008349A
:10DDA00004AFBD6B24F00704ADEB040DBE69039511
:10DDB000FD6904AC0195009602947D6BFFF76EFF40
:10DDC0003B6B21460293FB6A03950193BB6A404675
:10DDD0000093D7E90823FFF7ABFFBD46BDE8F0810C
:10DDE0002DE9F041884684B04C00083404AFBD6B87
:10DDF00024F00704ADEB040DBE690395FD6904AC86
:10DE00000195009602947D6BFFF770FF3B6B2146F6
:10DE10000293FB6A03950193BB6A40460093D7E9DE
:10DE20000823FFF785FFBD46BDE8F0812DE9F04FDF
:10DE30008FB00AAF7D6D9A461B1A023300F10308BA
:10DE40008B465919FB6B18EB050804461646FB6018
:10DE500000F0AA804FEA8809002934D109F10A09A3
:10DE600029F00709C7F808D0ADEB090D08953E6DFC
:10DE70000DF128090796FE6C13460696BE6C5A46AD
:10DE800005967E6C414604963E6C0396BE6BCDF8BB
:10DE90000890CDE900A6FFF7A3FF002C0DDBFE687C
:10DEA0000235013409EB850906EB440459F8043BBB
:10DEB0005B1124F8023DA642F8D1D7F808D01437F8
:10DEC000BD46BDE8F08F8B000A3323F00703C7F887
:10DED00004D0ADEB030D08953A6D0AAB0792FA6CCE
:10DEE00009F10A090692BA6C29F0070905927A6CC1
:10DEF00004923A6C0392BA6BCDE900A2BB605A4619
:10DF000002933346FFF746FFADEB090D0895396DD7
:10DF10000DF128090791F96C33460691B96C5A4600
:10DF20000591796C20460491396C0391B96BCDF859
:10DF30000890CDE900A14146FFF752FF631C9A45C6
:10DF400011DDFE68BA68E91CB31E02EB810103EB28
:10DF50004A0A06EB440251F8043B5B1122F8023FE7
:10DF60005245F8D1FE60002C0DDDFE68E91C09EB7E
:10DF7000810106EB440251F8043B5B1122F8023D9B
:10DF80009642F8D1FE60BB68023559F8252053F857
:10DF900025301344FA689B1122F81430D7F804D0C6
:10DFA0001437BD46BDE8F08F8B000A3323F007031A
:10DFB000E946ADEB030D08953E6D0DF12808079677
:10DFC000FE6C13460696BE6C5A4605967E6C049609
:10DFD0003E6C0396BE6BCDF80880CDE900A6FFF736
:10DFE000D9FE544512DAFA6804F10044013C0335C5
:10DFF000931E02EB440608EB850803EB4A0A58F827
:10E00000043B5B1126F8023FB245F8D1CD461437E8
:10E01000BD46BDE8F08F00BF2DE9F04788B09946B6
:10E020004FEA430808F1080424F0070408AFADEBF9
:10E03000040DD7E90D563C6BCDE90656BD6AFE6A64
:10E04000059403953C6A7D6A049608AECDE90165A6
:10E050000094FD6BFFF7EAFEB9F1000F10DD023C02
:10E06000A044A6F1020A34F9023F3AF9022F9B1AA2
:10E07000AB42CCBF5B1B03EAE37344452380F2D180
:10E08000BD46BDE8F08700BFF0B50D4685B0074638
:10E090001B49642014460022F4F714FC00260122D8
:10E0A000042118482B460091039011466420CDE9C5
:10E0B0000166F4F7BBFB0120134AE91B49090090F4
:10E0C0000392CDE901663B4620226420F4F7AEFBC3
:10E0D000294651F8043BA342FBD000220124C5F19C
:10E0E0001F030A481944CDE90122039049092B4630
:10E0F000009420226420F4F799FB05B0F0BD00BF26
:10E100002C9D0100409D01004C9D0100649D01007B
:10E110000B68934209D070B50D4614460646224658
:10E1200029463046FFF7B0FFF9E770472DE9F04187
:10E1300000258CB00790081A2E46049309952B46AB
:10E14000CDE905218410129D06E00133B4EB830F65
:10E150004FF00106C0F28A8051F80429AA42F4D097
:10E16000002E40F09E8000274FF0040801224E4B05
:10E17000861B1146CDE901770393642007ABCDF8E8
:10E1800000800A96F4F752FB01221446474B484E92
:10E190001146CDE901770393642006ABCDF80080EA
:10E1A000F4F744FB224621460297CDE9008409ABEF
:10E1B00064200396F4F73AFB3E4BCDE90147224633
:10E1C00021460393CDF800800AAB6420F4F72EFBC0
:10E1D000049C3946A446059C0997A4EB0C07BF1084
:10E1E000ACF104020B4605E00133B7EB830F4FF0AF
:10E1F000010147DB52F8040FA842F5D000294DD1A8
:10E200000025042701222C4BA4EB0C04C1EBA40431
:10E210000393114605ABCDE90155009764200B949B
:10E22000F4F704FB01221446244B11460393CDE975
:10E23000015504AB00976420F4F7F8FA09AB2246C5
:10E24000214602950097039601946420F4F7EEFAB4
:10E250001B4BCDE9014503930097224621460BABAA
:10E260006420F4F7E3FA0CB0BDE8F08164200022EA
:10E2700014490993F4F726FBDDE90640099B201AAF
:10E280009E0070E70F49002264200993F4F71AFBFF
:10E290000999059C8900DDF810C0B1E70993990040
:10E2A000AEE709939E005EE7849D0100909D01000A
:10E2B000409901009C9D0100B09D0100BC9D0100A2
:10E2C000C89D0100789D01000022024BC3E9002295
:10E2D0001A817047AC2200200278014B1A707047F7
:10E2E0003C180020314B1B78002B5AD02DE9F04F01
:10E2F00016462F4A87B08946804600242D4F136862
:10E30000DFF8B4B0DFF8B4A0013E14E03D5D38F9A9
:10E310001410022D2BF8101005F1010E39F914100C
:10E320009CBF5FFA8EF53D55032D2AF8101017D0CB
:10E3300001340A2C0CD04FEA440C0CEB0401C81831
:10E3400016F8011F0029E1D1395501340A2CF2D108
:10E350000133022BC8BF0023136007B0BDE8F08F64
:10E360000CEB04035B000BEB0301086853440290C1
:10E370001868B1F804C09B88049002A9284601924D
:10E38000ADF81430ADF80CC0FFF7E8FB04A928F88D
:10E3900014002846FFF7E2FB019A29F814001368DD
:10E3A000C6E7044AC2E90033138170473C180020D5
:10E3B000B8220020AC22002034220020702200204D
:10E3C000F0B483000A3323F00703002800AFADEB5D
:10E3D000030D30DD6B4600260439B20002F18042A5
:10E3E00092F880C292F8815292F8824292F8832287
:10E3F0005FFA8CFCEDB2E4B2D2B2013683F800C011
:10E400005D709C70DA70BCF1000F03D00CF1FF3C22
:10E4100083F800C01E2D9CBF01355D700CB1013C1E
:10E420009C700D2A9CBF0132DA7053F8042BB04265
:10E4300041F8042FD1D1BD46F0BC704792F822308C
:10E44000002B39D1F0B5002889B00E460546144698
:10E450000FDD936942189A420FDB00231A4684F8B5
:10E460002130237D93429CBF012384F8203009B0E2
:10E47000F0BDF2D1D3698B42EFDD94F82130002258
:10E48000013384F821300D496420F4F71BFA002091
:10E490000121042202900A4B94F821706420CDE9F6
:10E4A00000210393032205AB069607950597F4F721
:10E4B000BDF994F82120D4E7704700BFE89D010022
:10E4C000109E01002DE9F04F98468BB0DDE9145302
:10E4D000012DA946B8BF4FF00109012B9C464FF012
:10E4E0000004B8BF4FF0010C169E07923788B6F8AB
:10E4F00004E01268D8F8006005FB072503FB0E66F0
:10E50000002895FBF9F596FBFCF6CDE908442ADDD9
:10E51000A446A146A246023901EB40000694CEF182
:10E52000000B059031F9023F5A1B22EAE272334494
:10E5300003EAE37397420EEB030403DC0120D21BD2
:10E54000069092445B4505DC4FF0010C002CB8BFEF
:10E550006442A144059B9942E4D1069B002B3AD129
:10E56000BCF1000F3AD1012400260425079F1D4B62
:10E57000224621460393CDE901463B46009564209F
:10E58000F4F754F9184B224621460393CDE901468E
:10E59000434600956420F4F749F9144B224621467E
:10E5A0000393CDE9014608AB00956420F4F73EF9EA
:10E5B0000F4B22460393CDE9014609AB0095214656
:10E5C0006420F4F733F9DDE908233A60C8F8003035
:10E5D0000BB0BDE8F08FCDF820A0C1E7CDF82490B6
:10E5E000C1E700BF209E0100309E0100409E010057
:10E5F000549E010070B19A4215DC0F4A1368C72B74
:10E6000001DC013313600D4B187808B181F0010073
:10E6100019707047084B1A68C72AF4DD1860074B59
:10E620000120197070470022034B1A60034B1878C1
:10E630000028EDD0EAE700BFC0220020C62200205B
:10E6400098B130B441F69C046FF4E170A1F1E1059A
:10E65000A5420144187809D941F2D864A1420FD9E2
:10E6600008B901221A7030BC70477047E42A18DCE0
:10E6700041F2D8629142F3D80028F4D1014608E073
:10E6800043F2D451A2F5E6728A428CBF00210121E7
:10E6900008B901221A700029E5D030BC00221A7096
:10E6A000704741F2D864A14206D90028DBD143F675
:10E6B00087018A42D7DDD4E743F2D454A2F5E6714C
:10E6C000A1428CBF002101210028E4D143F687003C
:10E6D0008242C8DDDDE700BF10B401299DF8044087
:10E6E00008D900B924B11378022B01D80133137073
:10E6F00010BC7047002BF4D10028F3D013781CB164
:10E70000022BF3D910BC7047002BF1D0013B1370E2
:10E71000EEE700BF2DE9F04FC14DADF2245DCDE92C
:10E720001623DDF868452B7834A81893231C18BFEE
:10E7300001238B461B930DF59079FBF7E1FA1E221E
:10E74000002124A80AF03BF93C22002148460AF0A7
:10E7500036F978220021EEA80AF031F91E220021B4
:10E760002CA80AF02CF93C22002157A80AF027F91E
:10E7700066A83C2200210AF022F90023DDF8680592
:10E78000CDE91F33CDE921332393002840F0D48312
:10E790004FF020080F27DDF86035B2AA0793DDF8A7
:10E7A000643594A90693EEAB02932CABCDE90093AC
:10E7B000D0AB0393CDE9047857ABF8F727FA0123E0
:10E7C00000240093974B4246394603936C20DDF8B2
:10E7D0006435CDE90144F4F729F8D0AB0493DDF8B2
:10E7E0006035DDF868050893DDF86435B2AA079353
:10E7F00066AB0393EEAB02932CABCDE9009394A9E7
:10E8000057ABCDE90578FAF7C7FCD0AB0493DDF838
:10E810006035DDF868050893DDF86435B2AA079322
:10E8200066AB0393EEAB02932CABCDE9009394A9B6
:10E8300057ABCDE90578FAF7F3FDD0AB0493DDF8DB
:10E840006035DDF868050893DDF86435B2AA0793F2
:10E8500066AB0393EEAB02932CABCDE9009394A986
:10E8600057AB0DF58666CDE90578FAF727FC0DF56F
:10E8700095652146782230460AF0A1F82146782293
:10E8800028460AF09CF8684BDDF868051A68DDF840
:10E890008C355278B3F924300892DDF8602507935F
:10E8A0000692DDF864254B460592EEAA0292CDF859
:10E8B00010800397CDE90065B2AA94A9FCF7E0F8AF
:10E8C000DDF868350DF5EA7AA3420DDD574655F8B7
:10E8D000041B56F8040BFDF78BFADDF8683501349C
:10E8E000A34227F8020BF2DC0F242025DDF88C254B
:10E8F000DDF86015B2F924201846CDE90912DDF8DB
:10E900006425CDE906450892D0AA059266AA04922C
:10E91000EEAA03922CAACDE901A257ABB2AA94A900
:10E92000CDF80090FAF710FF0023012021463D4C5E
:10E93000CDE900032A46CDE902346C20DDF86435C8
:10E94000F3F774FF9DF8D930DDF868050093B2AA9B
:10E950004B4694A9F8F7E0FEDDF8680500280CDDC9
:10E96000524666240AEB4001B2F9003004FB03F37F
:10E970009B1222F8023B8A42F6D1EEAB029324AB03
:10E98000CDE900A3B2AA4B4694A9FBF753FFFEF7CB
:10E990004FFC002840F040829DF8D630002B40F01C
:10E9A0002482189B012B04D19DF8EF30002B40F0FE
:10E9B000D1820026DDF8943584AC03F51770FCF79E
:10E9C000ADF9DDF868352660B34200F32D820126EB
:10E9D00000250420154B32463146009003936D20EC
:10E9E0000DF5AD63CDE90165F3F720FFDDF8A875FE
:10E9F0004FF020081597DDF86075169A1497DDF82A
:10EA00006475CDE906B21397D0AF1097DDF8507555
:10EA100066AA0F971FAF0E97DDF85875059207E0AD
:10EA2000440F0020689E01005C060020A09E0100AB
:10EA30000D97DDF85C75EEAA0C97DDF8547504921D
:10EA40000B97DDF84C752CAA0A97DDF84875179BD3
:10EA500009970F27039224AACDE901A257AADDF84E
:10EA60006805089394A91346CDF80090B2AACDF892
:10EA700048801197FCF7FCFE0E48CDE90155039044
:10EA800000966C2042463946DDF86435F3F7CEFE39
:10EA9000DDF86805A84230DDDDF84C25179BA2F1B2
:10EAA0000208DDF84825B146DFF80CA0971E9E1E2F
:10EAB00006E000BF689E0100AC9E0100A8421CDD7C
:10EAC00038F9021F37F9023F36F8022F2560C4E9F2
:10EAD00001130135E260002BF0D004220023412015
:10EAE000CDE90193CDF80CA0009223460121F3F764
:10EAF0009DFEDDF86805A842E2DC14231FAA169DDE
:10EB00000192DDF85C25294600920293DDF84C2540
:10EB1000DDF848355846FDF773F8179EDDF8503597
:10EB2000DDF84C250093DDF8481533460A20FCF744
:10EB30004BF9DDF85035DDF84C250093DDF848152C
:10EB400033460A20FCF702F9DDF85035DDF8482598
:10EB50000093DDF84C15DDF854350A20FCF76CF90C
:10EB6000DDF85035324603931FAB0293DDF85C3578
:10EB700029460193DDF84C3558460093DDF84835B9
:10EB8000FCF770FFDDF84835814600935A462B4666
:10EB90000A210020F8F7ACF92946DDF8502558463F
:10EBA000FFF7A0FBFEF744FB189B0026022B08BFD3
:10EBB00040F001005FFA89F31993C3B2CDE917362B
:10EBC000DDF85075DFF860A3DFF860833EAD169B7B
:10EBD0003BF9160033F916C0CC4B014633441D9067
:10EBE000286062463878CDF878C0C4F800C0FFF7D6
:10EBF00027FD1AF806301A97002B40F06581DDF8E2
:10EC000094153A7891F8AE3222B1C04A925D002A4A
:10EC100040F04381002B00F0448118F80630022BAD
:10EC200000F2628123462A4639783046F9F77CFBA8
:10EC3000002800F087811EAB39780022009330460F
:10EC40001DABF9F721F918F806201D9B296803FB75
:10EC500002F3C2F1030201FB0233AD4880FB031251
:10EC6000A2EBE3732BF8163018F806201E9B2168E0
:10EC700003FB02F3C2F1030201FB023380FB031228
:10EC8000A2EBE373169A22F81630A248F8F72AF995
:10EC9000189BB3F5C87F00F31C819C4B9B5D179AB2
:10ECA00038781999009208EB0602FFF715FD17F85E
:10ECB000013B0AF80630B9F1000F03D108F80690BD
:10ECC0000AF80690002E00F0E6800226169B0BEB59
:10ECD00006089F19DDF8503503F1010A38F9020FD3
:10ECE00037F902CF1AF8011F2B4600940022286042
:10ECF000C4F800C03046F9F7C7F801362A6823681F
:10ED00000A2EA8F800203B80E8D1B9F1000F40F3AB
:10ED1000118128220021284609F051FEDDF86805FE
:10ED2000002840F344810026DDF850350138DDF835
:10ED300058251844013B13F8011F19B1116845F813
:10ED400026100136834202F10402F4D1F6B23E22CB
:10ED500000210DF2122009F032FE822742F20F004C
:10ED60004FF0200CDDF860352146009332462080BC
:10ED70002B46032084F802C06771FBF7EFFB169C5B
:10ED80009DF8D530DDF8502502930092DDF84C3522
:10ED9000DDF84825214658460196F8F76BF9DDF86D
:10EDA000502521465846FBF7BFFC00229DF8D9307C
:10EDB0005946022B0CBF13460D230A20CDE9002330
:10EDC000DDF850352246F8F7CDF8DDF850355846D5
:10EDD0000093DDF84825DDF84C352146F9F72AF88F
:10EDE0001B980DF2245DBDE8F08F9DF8D730002B05
:10EDF0007FF4D7AD4A465146DDF86805F9F7F8F9D2
:10EE0000DDF8AC35187000283FF4D3ADDDF894354B
:10EE100003F50870FBF782FF84AC0026DDF8683547
:10EE20002660B3427FF7D3ADDFF80481002241466C
:10EE300070200125F3F746FD04230227364A2946B0
:10EE4000CDE9026200932A46234670200195F3F72C
:10EE5000EDFC2368314A2946CDE902620AEB4303FF
:10EE60002A46702001950097F3F7E0FC23682C4AAE
:10EE700009EB4303CDE90262CDE900752A46294634
:10EE80007020F3F7D3FC2368DDF868252B44934208
:10EE90002360CBDB9BE5012699E6032208F80620D8
:10EEA00013BB179BD3B918F8062039782B4600946A
:10EEB0003046F8F7CBFA2A6823682BF81620169A02
:10EEC000189022F81630E0E6DDF8943593F8AE326B
:10EED000A0E61448F8F706F80023E0E64FF0000338
:10EEE000002208F80630E0E723462A460021304693
:10EEF000F9F71AFA00287FF49EAE02460146009404
:10EF00002B463046F8F7A2FA95E600BFBC22002057
:10EF10005655555508C5010040990100889E0100CD
:10EF2000949E010004C70100C4220020C8220020D2
:10EF3000709E0100002622E7EEA9FFF741FADDF8F6
:10EF4000680525E43978024600942B463046F8F7E8
:10EF50007DFA70E62422002185A809F030FD1125F4
:10EF60001E2084ACFA214FF416724FF496774FF0BE
:10EF7000320C4FF03C0E2581A081642546200526E9
:10EF80004FF028080223C4E90B50E781A4F810C011
:10EF9000A4F814E02046E18061816282E28226606A
:10EFA000C4F82880C4E90D33FBF7B8FE35E7002626
:10EFB000CDE600BF2DE9F04FC7B2C0F3072883B0FC
:10EFC000474501900C992BDC9DF806A052000AF1F0
:10EFD00000499DF807B009F1FF390AFB023301EB44
:10EFE000490901EB4B0C0D9908F1010801EB470EA3
:10EFF000DA4518D849461C460C4D34F9170031F94A
:10F00000026F8542B8BF05468642B8BF08808C456E
:10F010001444F2D12DB2013747452EF8025BE7D1F7
:10F0200003B0BDE8F08F014DF5E700BF0080FFFFA2
:10F030002DE9F04F05468FB04FEA410A08AF184658
:10F040003A608846524600216C007B60D7F84490B5
:10F0500009F0B5FC2246386C002109F0B0FC002D07
:10F0600067DD0AF108033E6C23F0070B4FEAA803A3
:10F07000FB603B683119B9609C1EC7F814D0ADEB3A
:10F080000B0D08ABA51C18462946524609F08CFC0E
:10F09000F96802464046FEF7E1FCB8F1000F014670
:10F0A00053DD00202246034632F902CF8C4508BFCB
:10F0B000184601339845F7D10522ADEB0B0D15230A
:10F0C0004FF0290E07926FF4247240F23E6CCDE9A6
:10F0D00003E3069208AA02930095CDF814C03A61A2
:10F0E0000192BD6CFA6C43468A1A2944FEF79EFED3
:10F0F0003B697A689D1E0AEB040134F9023F35F939
:10F10000020F1B1AA3EB0903002B238006DD1088D6
:10F110009BB2184410803088034433808C4202F143
:10F120000202EAD1BB6802369E42D7F814D00C46E0
:10F13000A3D100233A68C8EBC8084FEA48081C3737
:10F1400022F80830BD46BDE8F08F6FF424724FF00E
:10F15000050E152340F23E6C2920ADEB0B0DCDE9D9
:10F16000062E08AA049302930095CDF814C00390CC
:10F170000192B86CFA6C43468A1A01440020FEF7EB
:10F1800055FE04EB0A01CDE72DE9F04F9FB08A0050
:10F1900008AF7A61083222F00702ADEB020DB861C8
:10F1A0004E0008A800297963B860FE6119DD4FF4AC
:10F1B000004E47F6FF7C0025B11ED7F8842001449D
:10F1C000D7F88C00023A96190DF11E04023822F885
:10F1D000025FB24221F802EF20F8025F24F802CF6A
:10F1E000F5D1B969786B4A0000FB02F2083222F0CF
:10F1F0000702ADEB020D08AA00297A6040F3E38014
:10F200007A6400223A6300EBD07222F00102043BE0
:10F210000A32D7F88010BB6322F007033B617B6999
:10F220000439CB18F9603B653B69C7F82CD0ADEBCE
:10F23000030D08AAADEB030D08ABBB647B6BFA644E
:10F24000002B40F33981D7F890200023013A14466F
:10F2500047F6FF797A629046D7F88C209A46951E39
:10F260007A6CC7E90F33CB46FE68D7F838E0A2F1D5
:10F27000020C3C620BE0FC6C4A4524F8130002DAF5
:10F2800001468146FB633A6D0133964221D056F820
:10F29000040F5EF8042F35F8021FC2EBA0121144D0
:10F2A000298018F8014F10B2E4072CF8020F4946E4
:10F2B000C7F854B0DFD4BC6C5A4524F81A0003DAFE
:10F2C00083467865C7F840A03A6D0AF1010A964274
:10F2D000DDD1C7F828A015254FF0000B05266FF4E7
:10F2E000247840F23E694FF0290AFA6C3C6A009299
:10F2F000F86B6431CDE9066B0395CDE9015A4FF007
:10F300000042CDE90498FEF787FECDE902A5CDE9DC
:10F31000066BCDE904980195BE6C4FF00042009653
:10F32000796DBB6A6431386CFEF776FE796B7B6A67
:10F33000FD6C0B44594618467B6C14F8012F0233C0
:10F34000D2074BBF35F81B2036F811200BF1010B0B
:10F350000131844223F8022CEFD17A6CF9693B6BBE
:10F360000A447A647969BA6B01330A44BA63BA69A8
:10F370003B639A42D7F82CD07FF456AFD7E90C897B
:10F380007A68FB69A2F1020CBA6800269E46924692
:10F390009D1E1544B9F1000F11DD29466046AAF102
:10F3A000020230F9023F31F9024F9C42B8BF0B8094
:10F3B00032F9024F9C42C8BF1380AA42F1D10136F4
:10F3C0004645F444E6D17B6B002B71DDBB68D7F872
:10F3D00088109C1E2646FA69881ED7F88C10A2F168
:10F3E000020CD7F81880023903EB0C0500EB020E73
:10F3F00035F8023F36F8022F9B1A20F8023F31F908
:10F40000023F704593FBF8F30B80F1D1D7F88430BD
:10F41000991E0A46BB6803EB0C0534F9023F32F92A
:10F42000020F002BB8BF5B42984200DA1380A5425E
:10F43000F3D1BB68084663449C46FB690B441A46FB
:10F440003CF9023F30F9024F002BB8BF5B429C42AF
:10F45000B8BF03809042F3D16FF00044D7F89030EA
:10F460002646581E7B6B03449C46034604E09442A8
:10F47000A8BF14469C450AD013F8015F31F9022F4A
:10F48000ED07F4D49642A8BF16469C45F4D1D7F8B0
:10F49000842010F8015F118815F0010FA1EB04051D
:10F4A0000ABF891B15801180834202F10202F0D14C
:10F4B0005C37BD46BDE8F08F0024152505266FF4A6
:10F4C000247840F23E694FF0290AFB6C20460093F5
:10F4D00007942346CDE90586CDE90359CDE9015AC4
:10F4E0004FF0004248F26301FEF796FDCDE9066455
:10F4F000CDE90498CDE902A50195BB6C20460093A7
:10F500004FF00042234648F26301FEF785FD24E7F1
:10F51000002824DDF0B400258E1EAC464FF0FF37E6
:10F5200000E01D4636F9024F6B1C944203DD644532
:10F53000C4BFA4462F469842F3D17B1C11D07B0058
:10F5400031F917001FB1CA1832F9022C1044AF422A
:10F5500003DA1944B1F902301844F0BC70470020B6
:10F5600070470020F0BC70472DE9F04F80461D46E3
:10F57000460006F1080A2AF0070A91B006AFADEB83
:10F580000A0D3B6D06ACADEB0A0D06A8C7E90121DB
:10F590000092049301900B46CDE90245F860414684
:10F5A0001A220220D7F858B0D7F86890FFF7ECFD80
:10F5B0007A6DF9684046FFF7ABFF3B6EADEB0A0D85
:10F5C000B8F1000F18600DF1180A40F39A80AAF103
:10F5D00002031946023DA81935F9022F002AB8BFC7
:10F5E0005242854221F8022FF6D15A4651464046F2
:10F5F0003B60FFF78DFF00227B6E023E18601046D5
:10F600003B680AEB0605C9F8002033F9022F934541
:10F6100005DAD9F8001010440131C9F800109D42F4
:10F62000F3D1FB6E264418600023023C34F9022F0C
:10F630009342B8BF1346A642F8D1012404260621FE
:10F6400000254FF0020B386F354A03607B68CDE927
:10F65000014103922146424600966220F3F7E6F804
:10F66000304ABB68CDE9025259464246CDE90064B2
:10F670007220F3F7DBF82C4A534621460392CDE97A
:10F6800001454246CDF800B04E20F3F7CFF82748A9
:10F69000FB68424621460390CDE90145CDF800B014
:10F6A0004E20F3F7C3F82A4621496E20F3F70AF9F2
:10F6B0007A6E204B12682146BA61FA6E6E2012688B
:10F6C000FA61D9F800203A623A6F12687A623A6EAB
:10F6D000126803937A6107F1140305220096CDE9BD
:10F6E0000145F3F7A3F8FAF7C7FD3B6E2C371B680B
:10F6F000FF2BA8BFFF23DBB280F82430BD46BDE856
:10F70000F08F5A4651464046FFF702FF00227B6EBB
:10F71000F96E1860C9F8002013460A608DE700BF33
:10F72000C49E0100D09E0100DC9E0100F49E0100F9
:10F73000049F0100309F01002DE9F04F82461646DC
:10F74000524600258BB000AF8846386D520000212C
:10F750003C6E9946BB61C7F808A009F030F90AEB86
:10F76000DA7323F001030A3323F00703ADEB030D33
:10F77000C7F820D0AA45ADEB030D2561C7F81CD012
:10F7800025606560A560E56084F811A0257440F3EC
:10F79000F980504647F6FF7E7A6DCC46013A7A6092
:10F7A0009246321F02EB80037B613B6DAB46714694
:10F7B000A8F10408A3F102097D623C6611E07345DB
:10F7C000A8BF7346D7E9084524F81500A8BF184616
:10F7D0007C6A86467869013490427C620CF1010CA7
:10F7E00031D0B86952F8043F20B19CF8000000FB0A
:10F7F0000333DB1158F8040FBD6DC3EBA01347F6BC
:10F80000FF708342A8BF034661480E468342B8BFDB
:10F81000034618B229F8020F1AF8014F2C57002C92
:10F82000CDD18B42A8BF0B46FC691E4624F81B00B5
:10F83000A8BF184601467869734690420BF1010B48
:10F840000CF1010CCDD1D7E918429342A8BF134661
:10F850009642A8BF16461BB2524236B29342B8BF78
:10F8600013469642B8BF164632464FF0000C4FF092
:10F870000040FE60FE6D7968D6E900E9BE683B6134
:10F880000E44B346B7F9106012B27E61E0464E46B0
:10F8900063466FF00045BA617862D7F8509041E056
:10F8A0003A6A786932F91820002A5ADB002802DB0C
:10F8B0003869121A12B229F8132008F101087245AA
:10F8C00018DDB4F808A022680AF1010AA4F808A01B
:10F8D00039F913A094F91100AAEB0E0A52442260E0
:10F8E00094F910209842C8BF63749A42B8BF237439
:10F8F00039F9132096420ADD62896068013262811B
:10F9000039F91320A2EB060A8244C4F804A0786AED
:10F9100001339042B8BF10469542A8BF15468B45AB
:10F92000786227D011F8012FB86D8256002AB7D11E
:10F93000FA69B86932F91C20002A09DB002802DBC9
:10F94000F868121A12B229F813200CF1010CB6E76C
:10F950000028F5DA121A02EAE27212B229F813202C
:10F96000F3E70028A4DA121A02EAE27212B229F8C6
:10F970001320A2E72DB203B22C37A381E581BD4647
:10F98000BDE8F08F2B464FF000404FF0FF35F3E716
:10F990000080FFFF2DE9F047824686B00620DDE9B2
:10F9A00012781C460E4691461425F4F7B3FDF5F780
:10F9B00041F9159B31460493149B029003930F9BCE
:10F9C0004A46CDE9004305950E9B5046FFF7B4FE2D
:10F9D000002501210226154823460390524669203E
:10F9E000CDE901150096F2F721FFAA4528460EDD64
:10F9F000A31E03EB4A0A33F9021FCA1B002AC8BF21
:10FA0000AD18B1EB080148BF40185345F3D1109B26
:10FA1000AB4207DB119B8342D4BF0020012006B01C
:10FA2000BDE8F087012006B0BDE8F087C0A1010065
:10FA3000002820DDF0B48E1E06EB4006B14218D03F
:10FA4000571C38460B46B1F9004033F9025FAC420F
:10FA500007DD0D801C8092F9004090F90050157070
:10FA60000470B34200F10100EDD10231B1423A46D7
:10FA7000E6D1F0BC704770472DE9F04F8046450055
:10FA800005F1080485B000EBD07A24F007040730B4
:10FA90002AF0010A00AF20F00700ADEB040D08F1D9
:10FAA000090424F00704EB46ADEB000D0AF10A004F
:10FAB00020F007006E46ADEB040D6C46ADEB000D7B
:10FAC000E946C7E902210AF1020A08F102021F21F0
:10FAD00020467B6008F073FF52464846002108F03C
:10FAE0006EFFB8F1000F7B6807DD324606EB0800B9
:10FAF000911B02F8011B8242FAD14FF0FF3A2A46CD
:10FB0000F96858467B6008F04FFF59463246404638
:10FB1000FFF78EFF023D08F1FF3E7B6806EB0E010A
:10FB2000AB44013EB14218D03BF9025911F9012909
:10FB30009D4202F1010C10DBA05C22441F28927848
:10FB400060D01E2860D81E2A96BF4FF0FF3204F8FE
:10FB50000C0004F80C20B142E6D1B8F1020F04F118
:10FB6000010113DD0B46FF20A64402E0013373457B
:10FB70000CD05A781F2AF9D11A781E2AF6D89A780A
:10FB800001331E2A98BF18707345F2D1B8F1000FE7
:10FB90002EDDFB6804EB0806F96004E00134A642A0
:10FBA00003F1020323D06278FF2AF7D1257894F875
:10FBB00002C039F8150039F81CE08346704528BFAB
:10FBC000F346B3F90020B96B0A449345E6DA704571
:10FBD00038BF7046013465458CBF29F81C0029F8F0
:10FBE0001500A6420AF1FF3A03F10203DBD1F968DE
:10FBF0004246B86808F0D8FE0AF101001437BD4645
:10FC0000BDE8F08F1F2A06D01E2A88BF6FF0690258
:10FC100004F80C2086E70AF1010A04F80CA029F880
:10FC20001A507FE7FFF728BF004870477001002097
:10FC3000024B1A680260187D704700BF70010020F7
:10FC4000024B5A680260587D704700BF7001002067
:10FC500030B44FF0804300220E211F2020250F24B6
:10FC600083F8082183F80A2183F8090183F80B112E
:10FC70001A739A735873D9731D725C72DA7793F89A
:10FC8000211041F0010183F8211093F8211062F353
:10FC9000410183F8211030BC704700BF10B44FF011
:10FCA000804485B00DF1100C0CE90F00BDF8003058
:10FCB0002382BDF802306382BDF90430A382BDF90E
:10FCC0000630E382BDF808302383BDF80A30638331
:10FCD000BDF80C30A38305B010BC70474FF08043D3
:10FCE000988370474FF08043988B70474FF0804364
:10FCF00083F82000704700BF0123002110B50A4A95
:10FD00000A4C2377917210B94FF08042D3704FF0B4
:10FD100080430122987000211A700A2000F082F9B5
:10FD20000022024B1A7710BDCC2200200000105098
:10FD300001234FF08040102110B4034A034CA372FA
:10FD4000436010BC11607047D4080020CC22002012
:10FD500001234FF08040102110B4044A044C637218
:10FD6000C0F8043110BC1160704700BFD4080020F7
:10FD7000CC220020E0220021014808F020BE00BF74
:10FD800080010040F0B50546174B184885B06A1E43
:10FD900013F8011B834202F8011FF9D101242B46FD
:10FDA000002702262868124AC11782FB00C20244BB
:10FDB0001048C1EB222243F8242B2146224603900F
:10FDC000CDE9014700966220F2F730FD0A48CDE9FF
:10FDD00001470390009605F1260322462146622042
:10FDE000F2F724FD05B0F0BD2800004054000040AB
:10FDF0008988888830CA01006C9F010070B5E022B4
:10FE0000064600210B4808F0DAFD002401234FF0DC
:10FE10008042094D09492B770A208C729370214644
:10FE2000137000F0FFF82C773046BDE87040FFF704
:10FE3000A9BF00BF8001004000001050CC2200206C
:10FE400010B50446FFF79EFF2E234FF0804004F1CB
:10FE50004E0203F1600150F82110013B1F2B22F8E4
:10FE6000021DF6D14FF0804004F1960203F16001CB
:10FE700050F82110013B22F8021D591CF6D110BD8B
:10FE80004FF0804270B5037909B201FB03F1948B06
:10FE90008B11A342B8BF2346012500240221068806
:10FEA0009BB24380A2F80C61A2F80E31074E084BBA
:10FEB000357709205C7282F8035182F802112146DD
:10FEC000A2F8005100F0AEF8347770BD0000105079
:10FED000CC2200204FF0804393F81401704700BFFC
:10FEE0004FF0804393F81701704700BF0023094A81
:10FEF00082F832305064916472B6012382F8403047
:10FF000000BFB2F852309BB2002BFAD062B6B2F802
:10FF100050007047000010502DE9F047502210208B
:10FF2000202130244FF0400A4FF060094FF00108C3
:10FF30004FF4807E4FF4007C4FF480674FF40066EE
:10FF40000825104B83F8000383F8041383F8084353
:10FF500083F8034383F805A383F8092383F80A236E
:10FF600083F80B2383F80F93C3F80080186019609F
:10FF7000C3F800E0C3F800C01F601E601D60BDE84C
:10FF8000F08700BF00E100E04FF40042034BC3F8EC
:10FF90008020BFF34F8FBFF36F8F704700E100E009
:10FFA00000220121034BA3F86E20A3F86A20A3F8D6
:10FFB000681070470000105010B5174C84B094E8DA
:10FFC0000300029002A88DF80C1000F0ADF800F0CC
:10FFD000B5F8FFF7A1FF62B600F054FAA36804A8D1
:10FFE00040F80C3D00F048FA00F090FA00F0AAF951
:10FFF00000F000FB094B1A6922F004021A61BFF3FA
:020000021000EC
:100000004F8F0721064A82F824105A6942F01002E5
:100010005A6104B010BD00BFC48B010000ED00E0C8
:100020000000105008B500BF72B6084A135C3BB917
:1000300000BF30BF62B600BF72B6135C002BF7D0B2
:100040000023135401B1884762B608BDCC220020BA
:1000500000200A4B0A4913F8012B10448B42C0B20E
:10006000F9D1064B1A78AA2A01D000207047DB7B11
:10007000181AB0FA80F04009704700BF80004000B5
:100080008F0040002DE9F041142000F083FB002890
:10009000B8BF0730C51000234FF0A04001E08D42EB
:1000A00028DB027E0133591E002AF8D10126B04612
:1000B000194F00234FF0A04402E0A942267406DC49
:1000C000A27E0133591E002AF7D0BDE8F08172B636
:1000D000BFF34F8F4FF6FE724FF6FF733A877A8762
:1000E0007B873B87BFF34F8F00F0C2FE84F81180FF
:1000F00062B6DEE772B6BFF34F8F4FF6FE714FF672
:10010000FF72054B198759875A871A87BFF34F8F9C
:1001100000F0AEFE62B6C9E7000010504FF0A043F9
:1001200001225A74704700BF0246034B00681279DF
:1001300018601A71704700BFDC22002070B5FFF70D
:1001400087FF01220021334BD9705A72DA720028DE
:100150005CD0314AD278D2B21A72002201242F49DF
:100160002C4B8D789A725A731D734D780E781E75CC
:100170001D77CD78097983F8215083F820105A74BF
:100180009A741C749A7018B3234A51781A78C9B2B9
:10019000D2B28A4208D08A42B4BF013202F1FF32A1
:1001A000D0B28A421870F6D11B4B1A491A794B7893
:1001B000D2B2DBB29A420AD09A4203F1010096BF52
:1001C00003F1FF33C3B2DBB29A424B70F4D170BD7E
:1001D0001A78D2B2B02A08D0AF2AD4BF013202F1C5
:1001E000FF32D1B2B02A1970F6D10A4A5378DBB285
:1001F000082BECD0072B03F101018ABF03F1FF3379
:10020000CBB2DBB2082B5370F4D1E0E7E0221A72D4
:10021000A3E700BF0000105080004000DC22002057
:1002200007490B78DBB2834208D09842CCBF013338
:1002300003F1FF33DAB283420A70F6D1704700BF90
:100240000000105008B5FFF703FF18B1024B5878B3
:10025000C0B208BDB02008BD80004000014B187836
:10026000704700BF00001050084A5378DBB2834249
:100270000AD0984203F1010196BF03F1FF33CBB2DC
:10028000DBB283425370F4D1704700BF00001050BE
:10029000014B5878704700BF0000105010B504465D
:1002A000FFF73CFF4FF0A04320686168A26807C3D6
:1002B00010BD00BF38B54FF0A044E37DDBB2042B86
:1002C00028D0082B19D0022B09D00123184A13700B
:1002D00000BF4FF0A042137300BF537338BD154DDC
:1002E00015496079F9F766FE61792868F9F7CEFE5D
:1002F00062792B6813442B60E7E7104BD0E90512B5
:1003000059609A60236A5BBA0A4A18461360F9F783
:100310001BFEDAE7074D0A492079F9F729FE217912
:100320002868F9F763FE22792B6813442B60CCE729
:10033000CC220020E4220020200000509C19002044
:1003400024000050274B0022D3F8801041F0010117
:10035000C3F88010196C21F001011964196841F08B
:1003600001011960D3F8801021F00201C3F8801058
:10037000196C21F002011964196841F00201196039
:10038000D3F8801041F01001C3F88010196C41F0CF
:1003900010011964196841F010011960D3F8801038
:1003A00021F02001C3F88010196C21F0200119649C
:1003B000196841F020011960D3F8801021F0400144
:1003C000C3F88010196C21F040011964196841F0DC
:1003D00040011960C3F80821C3F80421C3F80021C3
:1003E000704700BF0000025038B572B64FF040545D
:1003F0000125642084F8245000F0F6F900F062F939
:1004000000234FF47A7084F8253084F8815000F08E
:10041000EBF900F057F962B638BD00BF10B572B6FF
:100420004FF040540123642084F8253000F0DCF9BB
:1004300000F048F9002384F8243084F8813062B653
:1004400010BD00BF0122002110B5094C86B02478F0
:10045000084806AB029103F8014DCDE90021039055
:1004600011466420F2F7E2F99DF8170006B010BDBE
:10047000B7004000809F01000268014B1A6070477E
:10048000E822002038B5FFF7E3FD0F23F0B94FF065
:1004900040524FF00104D9B2013B072B82F82B10D8
:1004A00082F8284082F82800F5D1042382F82F3002
:1004B0004FF040530121002283F8281083F82820B0
:1004C0004FF47A70BDE8384000F02EBA4FF040513A
:1004D000012500240C4806E081F82B20013B81F81F
:1004E000285081F82840027A0E2A8EBF0F22027A05
:1004F000D2B29342DAB2EFDA4FF04052024B5B7A5B
:10050000DBB282F82F30D3E780004000F8B5FFF768
:100510009FFD4FF0405401250026074684F82560D2
:100520004FF47A7084F8205084F8275000F0FCF9DA
:10053000642084F8255000F0F7F984F824506420F2
:1005400000F0F2F984F8256007BB06231C4D84F8FF
:100550002730EB7884F826302B7884F842304FF03F
:10056000405401230022697840F24C4084F8461040
:1005700084F8442084F8453084F8413084F84030D1
:1005800000F0D2F9AB7884F84430F8BDFFF75AFF99
:100590000C4B9B7A88B94FF04052DBB2084D84F87F
:1005A0002730E978074B82F82610DB7A29780B444C
:1005B0000B3BDBB282F84230D1E7053BEBE700BFF3
:1005C000E82200208000400020B9064A064B106057
:1005D0001860704703490548034B054A08601A60D4
:1005E000704700BFF0220020EC220020E903010048
:1005F0001D0401004FF04053F0B4062401220025F1
:100600000A26FF2083F8D64093F8D7100F2764F30B
:10061000030183F8D710042183F8D86083F84021C0
:1006200083F8D00083F87F5093F88C004FF0050CCE
:10063000104383F88C0093F88C00072640F00200EA
:1006400083F88C0093F8910064F30300032483F88B
:10065000910083F8901083F88D1083F8A02093F810
:10066000A10065F3010083F8A10083F8947093F86A
:100670008800104383F8880093F88900104383F8BA
:10068000890083F8F12083F8874083F88E4083F84F
:10069000D22083F8D52083F8ABC083F8AD5083F81F
:1006A000AC4083F8AE1083F8AF1093F88B1041F094
:1006B000700183F88B1083F8936083F8B020F0BC4E
:1006C000704700BF002382B000280193B8BF0730F5
:1006D000019BC010984206DD00BF019B01330193CE
:1006E000019B8342F8DB02B0704700BF10B572B6C1
:1006F0000023084C236062B6F9F7BEFD02E090F8D3
:1007000020302BB12368002BF9DD0122024B1A7037
:1007100010BD00BFF8220020F4220020054A06493F
:10072000937CD27801335B00934000FB03F091FB94
:10073000F0F070470000105000B4C404054A937AEA
:10074000D27ADBB20AB101339840034B93FBF0F04D
:10075000704700BF0000105040420F00054A937AD6
:10076000D27ADBB22AB10122134402FA03F390FBDE
:10077000F3F0704700001050054A00EB8000937CB6
:10078000D27801335B009340000190FBF3F0704797
:100790000000105041F28833124A00FB03F0137B33
:1007A0000001DBB25A1E062A0DD9082B12D0092BE4
:1007B00015D0A3F10B02032A0ED90F2B0CBF012376
:1007C0004FF0FF3300E00133064AD278934090FBAC
:1007D000F3F070470A23F7E7063B9B00F4E70C238E
:1007E000F2E700BF00001050124B00EB80001B7BB3
:1007F0000001DBB25A1E062A0DD9082B12D0092B94
:1008000015D0A3F10B02032A0ED90F2B0CBF012325
:100810004FF0FF3300E00133064AD278934090FB5B
:10082000F3F070470A23F7E7063B9B00F4E70C233D
:10083000F2E700BF00001050034B044A5B7C03F05A
:10084000010352F823301847000010508C9F01001C
:10085000134B1B7BDBB25A1E062A0DD9082B18D06E
:10086000092B1BD0A3F10B02032A14D90F2B0CBFA9
:1008700001234FF0FF3300E001330949094AC978E9
:100880008B4000FB03F382FB0320DB17C3EB6010FC
:1008900070470A23F1E7063B9B00EEE70C23ECE7E9
:1008A0000000105067666666034B044A5B7C03F0E9
:1008B000010352F82330184700001050849F0100B4
:1008C00038B50024064D21460320EC70FFF7AAFB43
:1008D00021460320EC70FFF7A5FB024B186838BDDA
:1008E000CC220020F822002070B50122002404262A
:1008F00086B00B4D06AB43F8040D1146CDE901243B
:10090000009603956420F1F791FF064B05985C7102
:1009100000F05EF821460520FFF784FB06B070BDAD
:10092000949F0100CC22002008B5FFF785FFBDE8A9
:100930000840FFF7D9BF00BF08B5FFF7B5FFBDE816
:10094000084000F015B800BF08B5FFF7ADFFBDE8DF
:10095000084000F025B800BF002000F069B800BFD3
:10096000012000F065B800BF00F04AB800F054B8AC
:10097000012830B44FF000024FF0020438BF0120CC
:100980000121054B054D1A702A719C709860DA6040
:100990005A70197030BC704700000850CC220020FB
:1009A000012830B44FF000024FF0020438BF01209C
:1009B0000121054B054D1A706A719C709860DA60D0
:1009C0005A70197030BC704700000950CC220020CA
:1009D00001284FF000024FF0010138BF012010B490
:1009E000054B064C1A70627199709860DA605A7003
:1009F000197010BC704700BF00000950CC220020C5
:100A0000012000220249034B08711A70704700BF91
:100A1000CC22002000000850012000220249034B94
:100A200048711A70704700BFCC22002000000950A6
:100A300010B40B4A0B4983B0CDE9001202AB03EBB3
:100A4000800353F8082C9378DBB2012B04D10021EA
:100A5000054C04302354117003B010BC704700BF24
:100A60000000095000000850CC220020034AD2F8B0
:100A7000803023F00103C2F880307047000002503C
:100A8000034AD2F8803043F00103C2F88030704747
:100A900000000250034BD3F88000C04300F0010077
:100AA000704700BF000002504FF48072DCF808303D
:100AB0001A617047002823DDF0B5DCE9013ED3F868
:100AC000013000241E7E0CE0DCF800703F5D07FB67
:100AD000055503FB05F35B1242F824300134A042B4
:100AE0000DD051F8045BDEF81030002EECD103FB82
:100AF00005F39B1042F824300134A042F1D1F0BD3F
:100B0000704700BF4FF48072DCF808301A617047FC
:100B1000002821DDF0B5DCE9013E00241E7E0CE05A
:100B2000DCF800703F5D07FB055503FB05F35B1226
:100B300042F824300134A0420DD051F8045BDEF8B5
:100B40001030002EECD103FB05F39B1042F824304B
:100B50000134A042F1D1F0BD704700BF4FF4807264
:100B6000DCF808301A617047002823DDF0B5DCE9B5
:100B7000013ED3F8013000241E7E0CE0DCF800704A
:100B80003F5D07FB055503FB05F35B1242F824307C
:100B90000134A0420DD051F8045BDEF81030002E75
:100BA000ECD103FB05F39B1042F824300134A04242
:100BB000F1D1F0BD704700BF4FF48072DCF808300F
:100BC0001A617047002823DDF0B5DCE9013ED3F857
:100BD000013000241E7E0CE0DCF800703F5D07FB56
:100BE000055503FB05F35B1242F824300134A042A3
:100BF0000DD051F8045BDEF81030002EECD103FB71
:100C000005F39B1042F824300134A042F1D1F0BD2D
:100C1000704700BFDCF80430F0B4D3F8013093F82B
:100C200021409CB900280FDD9B68DE889D8851F823
:100C3000043B013403FB06F393FBF5F3A0424FEAB8
:100C4000831342F8043BF2D1F0BC70470028FBDD6F
:100C50009B68DCF80040DF88013C9E88204414F843
:100C6000015F51F8043BA04205FB033307FB03F38C
:100C700093FBF6F34FEA630342F8043BEFD1F0BC79
:100C8000704700BF704700BF00280BDD10B4002480
:100C900051F8043B01349B01A04242F8043BF7D1D8
:100CA00010BC7047704700BFF0B50E4687B00221F8
:100CB000074601206546F3F775F900231946043805
:100CC00006F5F06406F5006C059350F8046FA4F582
:100CD000F062B60952F8803B9B1B94421944F9D14B
:100CE0000434A4450591F0D191FBF7F1AB6805916F
:100CF0001A88002A40D05888121A1202091A92FB48
:100D0000F1F1B1F5DC7FA8BF4FF4DC7119616A68BD
:100D10004FF0020CD2F8012000269068012284884E
:100D2000042701FB04F10912FF29A8BFFF21144683
:100D3000C1801348CDF800C011460390CDE901668B
:100D40006420F1F773FD0F4B224621460393CDE952
:100D5000014605AB00976420F1F768FDAB680A48CF
:100D6000CDE90146039000971033224621466420C6
:100D7000F1F75CFD07B0F0BD4FF480711961C6E773
:100D800080A001009CA00100A8A00100F3F720BCF6
:100D900008B5F3F74FFCBDE8084000210120F3F748
:100DA00001B900BF30B595B0202200210CA807F092
:100DB00006FE294C29492A4D2A48CDE90854CDE997
:100DC0000A01294A294B0E9293F8812002AC8DF832
:100DD0003C2093F881308DF83D30F5F78DFC8DF88F
:100DE0003E00F5F78FFC8DF83F00F5F791FC8DF88C
:100DF0004000F5F793FC8DF84100F5F795FC8DF870
:100E00004200F5F797FC1190F5F79AFC1290F5F770
:100E10009DFCADF84C0008A8F8F790FFF5F796FC9C
:100E2000F9F7EEFB002303220293A382C4E9013306
:100E3000C4E903338DF81D20FBF7F4FB06ABADF8D6
:100E40001E0093E803008DE8030094E80F00F8F714
:100E5000E5FE15B030BD00BF810A0100290901007F
:100E60006D0A0100950A01006E3816FA0000105054
:100E700070B5002301223F2148260825022484B0B2
:100E800001A8CDE9013303938DF807608DF8085070
:100E90008DF809208DF80F208DF80A408DF80D107F
:100EA000FFF7FCF904B070BD02FB01F21212FF2A39
:100EB000A8BFFF22028070472DE9F0432D4E95B068
:100EC0002D4D0FAC08AF904699460A9196E80F0059
:100ED00084E80F001CABC4E90275204613A91393E4
:100EE000EFF7CEF996E80F00244E0BAD85E80F0022
:100EF0002146C5E902762846EFF7C2F90520F3F747
:100F000009FB0521D0F801200990D2E902309A8826
:100F100014AEDA8006F8401D089031460120F3F740
:100F2000A9FA0221164B44F0010445F001050846D8
:100F3000CDE906450593CDF81090F3F733F8044654
:100F40008022002107F03BFD234631464046202207
:100F5000F5F702FC0625012104200A4A00900392BD
:100F60002346CDE9011520226420F1F75FFC15B07E
:100F7000BDE8F083D08B0100A90A0100B50A010089
:100F8000695F00000CBB01002DE9F0432D4E95B0C8
:100F90002D4D0FAC08AF904699460A9196E80F0088
:100FA00084E80F001CABC4E90275204613A9139313
:100FB000EFF766F996E80F00244E0BAD85E80F00B9
:100FC0002146C5E902762846EFF75AF90620F3F7DD
:100FD000A1FA0627D0F8013014AE9A6809939188D7
:100FE000DB68D18006F8407D314601200893F3F795
:100FF00041FA174B44F0010445F00105022103209A
:101000000593CDE90645CDF81090F2F7CBFF0446E5
:101010003C22002107F0D3FC2346314640460F22F4
:10102000F5F79AFB012104200A4ACDE90001039259
:10103000029723460F226420F1F7F8FB15B0BDE8B4
:10104000F08300BFD08B0100050B0100110B0100E4
:10105000915F00000CBB01002DE9F042214E90B0E1
:10106000214D0BAC04AF9946CDE9052196E80F0060
:1010700084E80F0016ABC4E9027520460FA90F9350
:10108000EFF7FEF896E80F00184E07AD85E80F0061
:10109000C5E9027621462846EFF7F2F8059B144F82
:1010A000D3F8013044F00104D3E90223918845F0DC
:1010B0000105D180169A0221042004930092CDE903
:1010C00002450197F2F76EFF8022002107F077FCBE
:1010D0002022034669464846F5F73EFB10B0BDE8BE
:1010E000F08200BFD08B01005D0B0100690B010095
:1010F0007D5F00002DE9F042214E90B0214D0BACF8
:1011000004AF9946CDE9052196E80F0084E80F0069
:1011100016ABC4E9027520460FA90F93EFF7B0F89C
:1011200096E80F00184E07AD85E80F00C5E9027676
:1011300021462846EFF7A4F8059B144FD3F8013059
:1011400044F00104D3E90223918845F00105D180E0
:10115000169A0221052004930092CDE902450197D9
:10116000F2F720FF3C22002107F029FC0F22034662
:1011700069464846F5F7F0FA10B0BDE8F08200BFC6
:10118000D08B0100B90B0100C50B0100A55F000069
:10119000054B0649013810F8012F013303F8012CE3
:1011A0008B42F8D1704700BF00008360E00183608C
:1011B0002DE9F041304E90B0304D0BAC04AF884675
:1011C000069096E80F0084E80F0016ABC4E902759C
:1011D00020460FA90F93EFF753F896E80F00284E1B
:1011E00007AD85E80F002146C5E902762846EFF7EE
:1011F00047F80120F3F78EF905900220F3F78AF9FA
:1012000002210020F2F7CEFE4FF4F06200210746E3
:1012100007F0D5FB0122059B10AED3F80130104634
:101220009B6906F8402D31460493F3F723F9059B9B
:10123000DFF864C0D3F8013031469A68114EB2F835
:1012400004E03B46A2F806E0404644F0010445F0C5
:1012500001054FF4F072CDE90245CDE900C6F5F77E
:101260007BFA094B09481B6909490A4A03610B616A
:10127000136110B0BDE8F081D08B0100A90C010012
:10128000150C0100953E0000BC0D0020F80A00205E
:10129000D80B0020900C0020D145000038B5054641
:1012A0000C4601200221F2F77DFED5F8013004F151
:1012B00080059B68D9889A8854F8043B03FB01F3A6
:1012C00093FBF2F3A54240F8043BF5D138BD00BFD3
:1012D0002DE9F041804684B00220F3F71BF902218A
:1012E00006460120F2F75EFE02220546D6F80130DE
:1012F00004AC9B68012099880E4FD98004F8102D0A
:101300002146F3F7B7F828468022002107F057FB63
:10131000094ADFF82CC0094E009221462B46404670
:101320002022CDE901C70396F5F716FA04B0BDE80F
:10133000F08100BF850C01008D0D0100890C0100BA
:10134000910D010083682DE9F04F9C880D4602FB4A
:1013500004F42412FF2CA8BFFF248968DC808A785B
:1013600091F800C08BB0ACEB420CCDF810C093F8F4
:1013700000E09A7847680646AEEB4202686805923C
:10138000BF788078B1F806A0874291F8089093F86A
:1013900008B040F0AA80306829680078097888424F
:1013A00040F0A380944500F0A98001224FF000088E
:1013B00002211746564806330091039011467120CA
:1013C000CDE90188F1F732FAB368524808333A465A
:1013D00039460390CDE9018871200097F1F726FA8C
:1013E00004204D4B3A46394600900393712005ABDB
:1013F000CDE90178F1F71AFA0222AB68474800926A
:1014000039463A4606330390CDE901887120F1F759
:101410000DFAAB68424808333A4639460390CDE9A5
:10142000018871200097F1F701FA04223D4B0092E8
:1014300003937120CDE901783A46394604ABF1F7C0
:10144000F5F9049800FB0AF0002854D0059BA4B2DB
:1014500003FB04F409F10E09A9EB0B0B04FA0BF4DE
:1014600094FBF0F402214046F2F79CFDE517061FBD
:1014700000F27C7C56F8040FC117CDE90801DDE9C4
:10148000088908FB05F7A8FB040104FB0977820B18
:10149000394442EA81428B13CDE90823DDE9082370
:1014A00066453260E6D102210120F2F77BFD061F7E
:1014B00000F17C0C56F8040FC117CDE90601DDE9F7
:1014C000068908FB05F7A8FB040104FB0977820BDA
:1014D000394442EA81428B13CDE90623DDE9062334
:1014E00066453260E6D1012005E0642000220E4905
:1014F000F1F7E8F902200BB0BDE8F08F00220B49AC
:101500006420F1F7DFF900200BB0BDE8F08F00BFD9
:10151000D09F0100F89F01001CA0010028A001003D
:1015200050A0010074A00100989F0100B49F010029
:1015300030B583B0FFF736FCF4F7A0FDFFF798FC59
:10154000FEF772FBFEF738FDFEF782FB00230B4926
:101550000B4C00931A4602200D680121A847FFF7A3
:10156000C5F800F02BFB2568FEF778FEA87024680C
:10157000FEF78EFEE07003B030BD00BFE0CA010090
:101580005C0600200246034B51680068926807C35E
:10159000704700BFFC2200202DE9F04F964683B033
:1015A000544E9DF834709DF830C0984600976346BD
:1015B0000D46B6F90620B6F90410044670469DF8AB
:1015C0003870FAF7FFFB3378800290FBF8F0002BBD
:1015D0004BD0A91C96F801904B002A4604EB030E51
:1015E00003F10208B9F1000F50D13EF8069C05F155
:1015F000FF3C24F80890A3F108053EF8043C25447C
:1016000024F811306189238961802380531ED2B36D
:101610001A4602F1010B4FEA4B0104EB010A0631B5
:1016200034F801903AF8028C34F81B30C84407FBB8
:1016300008F9BAF8048096F903B043440BFB039809
:10164000BAF8023096F90290624509FB03834FEA2B
:10165000A31300FB03F34FEA2343635246D0012A4E
:10166000D4D1E38800226380D3E765B1A91C04EBE1
:101670004101043431F8022D00FB02F28C424FEAA2
:1016800022428A80F6D103B0BDE8F08F0023638048
:10169000238024F8113024F80830002DF3D07F0087
:1016A00004EB450131F802E996F90350B1F808C09E
:1016B0000B88CA889C4538BF9C46964538BF9646DD
:1016C0000CFB07F36A000EFB02338D8896F90220AB
:1016D0008C4205FB02324FEAA21200FB02F24FEAF3
:1016E00022420A81DED103B0BDE8F08F2B88AEF82C
:1016F00000308BE7FC22002082B0F0B593B00546A5
:101700000E4608A818A981E80C00F8F7F9FA9DF828
:1017100026301BB19DF82730002B5FD03C4C189829
:10172000234619991A9A07C394F9033094F9027061
:10173000C3F12003E17AC7EB4307A37AC7F3470756
:101740006A6905F12C00CDE9011700930F212023D0
:10175000FFF722FF05F15200617A237A04466A6995
:10176000CDE90117009320210F23FFF715FFFEF7A6
:1017700001FB20462E234FF0804403F1600230F835
:10178000021D013B1F2B44F82210F6D14FF080447C
:1017900005F19A0232F8020D03F16001013B44F8B1
:1017A0002100591CF6D10120FEF7A6FA2846FEF7C3
:1017B000E9FAB4F84C301BB2336094F8503033720D
:1017C00094F85130737294F85230B37294F85330E5
:1017D000F37213B0BDE8F04002B07047B5F92430A1
:1017E000B3F5827F9ADA47F22E526B68A3F5EA438B
:1017F000313B934292D86B8BB42B8FD9054A044C62
:1018000005AB07CA83E8070084E807008CE700BF40
:10181000FC220020E08B010038B504220125124B88
:10182000124C1D712260FFF797F8F8F725FD837EB3
:101830002BB90F4B1B6813B10E4A157098470E4B0E
:10184000D3F80021120708D5002208250B480C49BF
:10185000C3F880510270C1F8402101211023094AC8
:10186000D160236038BD00BFCC220020D408002006
:10187000A40F0020600F002000E100E0D00800204D
:1018800000000250000008500122052138B50D4B20
:101890000D4C5A712160FFF763F80C4BD3F800210F
:1018A000120708D50022082509480A49C3F88051C3
:1018B0000270C1F8402101211023074AD160236042
:1018C00038BD00BFCC220020D408002000E100E099
:1018D000D0080020000002500000095030B4002061
:1018E00001251022044C0549054BE570C1F8400163
:1018F00030BC1A60704700BFCC22002000000250AC
:10190000D408002001234FF06050102110B4034A86
:10191000034CE372836210BC11607047D40800204E
:10192000CC2200200F21124A124B11605B6F84B051
:101930000193019B23F4FF6323F007030293019BB0
:1019400023F07F030393029BB3F5800F0AD0039A21
:10195000094B9A4206D0019A084B9A4202D20122C0
:10196000074B1A700122034BA3F86C2004B0704798
:10197000D40800200000105080FF010000FC01008E
:101980000823002008B5FFF7D3FD00F0BFFC0020BE
:1019900008BD00BF704700BF30B50A4D0A4C83B088
:1019A000294620464FF0CD32FCF76EFB4FF0CD328A
:1019B000204600922B46054A0549FCF7B7FB00205C
:1019C00003B030BDF83A0020F82E00200056002069
:1019D000F83A0020704700BF10B5084B084C1A6851
:1019E00021466320F0F76EFFF2F7EEFB054B214630
:1019F000BDE810401A686320F0F764BFA00400201F
:101A0000D8A00100A404002000210120F2F7CABAE6
:101A1000F0B5194B194C83B01A6821466320F0F7D2
:101A200051FFF2F7D9FA0220F2F774FD064601A839
:101A3000FEF7FEF802210120F2F7B4FA0746104B38
:101A400002A91B880F4D21F8083D0220F2F712FD74
:101A50000220FFF73DFC28460221FFF7A9FB2A6977
:101A600039463046FFF71AFC074B21461A686320B7
:101A7000F0F728FF03B0F0BDA0040020B8A00100DB
:101A8000EC8B0100BC0D0020A40400202DE9F043E4
:101A90000220A9B0F2F73EFD02210120F2F782FAFE
:101AA000002107460120F2F77DFA064607A8FEF757
:101AB000BFF80546274C80220021204606F07FFF14
:101AC000079AEDB218A80DF1200C0492CDE901C0DF
:101AD00003940097294633461A220220FDF754FB4F
:101AE0005DB1204604EB4502B0F90030002BB8BFD1
:101AF0005B4220F8023B9042F6D101244FF00409EA
:101B000006214FF00008144A3B46CDE901410392FB
:101B100021462A46CDF800906220F0F787FE0F4A52
:101B20003346CDE90282CDE900942A460221722093
:101B3000F0F77CFE02200A4B00900393CDE90148A8
:101B400021462A46034B6920F0F770FE014829B070
:101B5000BDE8F0838C250020C49E0100B0A10100E7
:101B6000BCA10100022300B583B002A901F8043D25
:101B70000120F2F77FFCF2F72BFDF2F75BFD03B0DB
:101B80005DF804FB30B5044685B0FEF75BFB01222F
:101B90000023084D084903340444CDE9013303917F
:101BA0002B460092114664202C70F0F73FFE05B0E2
:101BB00030BD00BFD4040020109301000148F6F7A7
:101BC000E9B900BFFC0500202DE9F04F8BB004AF50
:101BD000FEF738FB012400260425DFF838C207F1A0
:101BE000180343F8140D2246CDF80CC0CDE9014688
:101BF000214600956420F0F719FE0322784807F18A
:101C00001803DFF8149243F8102D21460390CDE914
